:100000000C94B3010C9436020C9436020C94360214
:100010000C9436020C9409180C948A160C9436022F
:100020000C9436020C9436020C9436020C94360270
:100030000C9436020C9436020C9436020C94CF0CBD
:100040000C9436020C9436020C94F1160C94511751
:100050000C9436020C9436020C9436020C94360240
:100060000C9436020C9436020C9436020C94360230
:100070000C9436020C9436020C94DC110C94411151
:100080000C9436020C9436020C9436026C706F702D
:100090007270757078707F70827085708870C070B3
:1000A000E570EA70EF70F470F970037116711971F0
:1000B00020712E719D719D719D719D713D71437176
:1000C0004C715E7161716D719D7170717671797134
:1000D0007F71827188718B71937172252E327820B5
:1000E000007C000A0077252E327820000A00722555
:1000F0002E32787C000A005445524D494E414C2026
:100100004552524F523A2063616E6E6F7420616C9B
:100110006C6F63206D656D6F72790A007265676937
:1001200073746572696E6720636D643A257320008D
:100130006661696C656421206E616D6520746F6F06
:10014000206C6F6E67210A0072656769737465724F
:10015000696E6720636D643A257320006661696C7F
:1001600065642120636D6473206275666665722024
:1001700066756C6C210A000A000A0009000A004238
:10018000544E5F5445524D494E414C3A20455252CF
:100190004F523A207768696C652072656164696EB8
:1001A000672066726F6D20756172740A000A20758F
:1001B0006172742072656164206572723A202564F0
:1001C0000A002563202563000A0025733A20636F27
:1001D0006D6D616E64206E6F7420666F756E640A5B
:1001E0000025632025630021214C494E4520544FB2
:1001F0004F204C4F4E4721210A002563006E757435
:100200003A206572726F723A2075736167653A0AB7
:10021000206E757420746872656164730A206E754F
:10022000742074696D6572730A206E757420686538
:1002300061700A004E75743A2048656170204176FD
:1002400061696C61626C65203D202575206279745E
:1002500065732E0A000A486E646C204E616D65203D
:10026000202020205072696F205374612051554521
:10027000202054696D722053746B5020467265655E
:100280004D656D0A002530345820252D3873202502
:1002900034752025732025303458202530345820DB
:1002A00025303458202535752025730A0025303433
:1002B0005820252D387320253475202573202530AE
:1002C00034582025303458202530345820253575B1
:1002D000202573002025303458004E757454687200
:1002E00065616457616B65004E75744576656E7423
:1002F00054696D656F75740041646472205469635C
:100300006B7320204C6566742043616C6C62616382
:100310006B0A002530345825366C7525366C7520EF
:10032000002530356C58002825303458290A00251E
:10033000303478202535640A00257520636F756E8A
:100340007465642C20627574202575207265706F49
:10035000727465640A00257520627974657320667D
:100360007265650A000085B7806885BF80916C0062
:10037000806880936C00BF9ABE9AC798C69880EC3C
:1003800085BFAF9AA79AAE9AA69A81EE8093008312
:1003900080E4809301832FE785B7822385BF80E0C7
:1003A00090E09D9B05C0019641F09D9BF8CFFBCF4F
:1003B000019619F09D99F3CFFBCF85B7806885BF73
:1003C00085B3822385BB84B3822384BBAE98A69871
:1003D00087E089B98093990011241FBECFEFD0E147
:1003E000DEBFCDBF14E1A0E0B1E0E6E4FCEF00E049
:1003F0000BBF02C007900D92AA30B107D9F715E1E3
:10040000AAE0B4E101C01D92A93EB107E1F78FEF68
:100410009FEF9EBF8DBF8FEF9FEF895E9541815803
:10042000914048F08FEF9EEF895E9541BC0189EEC7
:1004300095E10E9468090E947409892B59F0ADE882
:10044000B5E1EBE2F3E089E001900D928150E1F734
:100450000E94900920E831E040E050E060EF73E056
:1004600084E393E00E944E0B0C9400000C94000077
:10047000AF92BF92CF92DF92EF92FF920F931F93B2
:10048000CF93DF93CDB7DEB7CC54D0400FB6F894FE
:10049000DEBF0FBECDBF8E01075B1F4F80E091EE28
:1004A000A0E0B0E0F80180839183A283B3830E942F
:1004B000DF4A81E00E94374E40E060E070E08FE369
:1004C00093E00E943504409151045091520460E041
:1004D00071E081E493E00E94921880915104909120
:1004E00052040E942F18A80161E071E00E94831954
:1004F0000E94095183E091E09F938F930E94051918
:100500008DE391E00E941A1985E691E09F938F9305
:1005100083E791E09F938F930E94051981E991E011
:100520009F938F9388EC91E09F938F930E9405197E
:100530000E94510C5B016C010E945C0CDC01CB0140
:100540009F938F9350E4E52E52E4F52E5FE0052F44
:10055000112DC601B501A80197010E948C7DCA0129
:10056000B901A80197010E944E7DDC01CB01A601D3
:100570009501281B390B4A0B5B0BCA01B90124E614
:1005800030E040E050E00E948C7D3F932F93C60105
:10059000B501A80197010E948C7D3F932F938EECAB
:1005A00091E09F938F930E94051987EF91E09F93AD
:1005B0008F930E9405198FE292E00E941A190E94FF
:1005C0006F4B8BEB93E00E9496319093791580935B
:1005D00078154DE050E060E070E00E94A02ABE0176
:1005E0006F5F7F4F80917815909179150E94C02D93
:1005F0008A819927982F882729813327822B932B4B
:100600009F938F938C819927982F88272B8133274D
:10061000822B932B9F938F938E819927982F8827D6
:100620002D813327822B932B9F938F938CE492E021
:100630009F938F930E940519AE01495F5F4F60E061
:1006400070E080917815909179150E9452278D85E0
:100650009E859F938F938B859C859F938F938A858F
:1006600099279F938F93888599859F938F938F81E7
:1006700099279F938F9383E792E09F938F930E9494
:1006800005194DB75EB7485D5F4F0FB6F8945EBF72
:100690000FBE4DBFAE01415F5F4F60E070E08091E3
:1006A0007815909179150E94E0278E8999279F935C
:1006B0008F938D8999279F938F938C8999279F93E7
:1006C0008F938B8999279F938F938A8999279F93DB
:1006D0008F93898999279F938F93888999279F93CF
:1006E0008F938F8599279F938F9386E992E09F93AD
:1006F0008F930E9405198E01095E1F4F2EE1A801FC
:1007000060E070E080917815909179150E94182131
:100710001F930F938DEC92E09F938F930E94051986
:100720004FED52E060E070E080917815909179157E
:100730000E948C208BEE92E00E941A1989819927E1
:100740009F938F938A8199279F938F9380E193E062
:100750009F938F938E010B5C1F4F1F930F930E94EB
:100760002F19B80180915104909152040E940A54AB
:1007700080917815909179150E9496620E94746319
:100780000E94746A0E945F640E94B4648091510464
:10079000909152040E94156760E070E081E00E9431
:1007A00048588DB79EB74E960FB6F8949EBF0FBEB1
:1007B0008DBF80E090E0C45BDF4F0FB6F894DEBFE2
:1007C0000FBECDBFDF91CF911F910F91FF90EF90A2
:1007D000DF90CF90BF90AF90089580932503089548
:1007E0000E947E0420E033E040E050E068E372E0E5
:1007F00086E293E00E944E0B8EEF0E9406080E9454
:10080000B4070E94CC07209125032F3FC1F395B771
:100810009C7185B7837E822B85BF85B7806285BF3B
:10082000889585B78F7D85BF85B7837E892B85BFEA
:10083000E6CF0F931F93CF93DF938C01C0910B14DE
:10084000D0910C14209759F0B801CE0102960E9465
:10085000207D892B21F00990D881C02DF3CFCE01C6
:10086000DF91CF911F910F910895EF92FF920F9317
:100870001F93CF93DF93EC018FEFE82EF82E209794
:1008800009F16115710511F07D876C8741114E8763
:10089000CE0102960E9419048C01892B99F4EB89F0
:1008A000FC89309721F0CE010995892B59F480916C
:1008B0000B1490910C1499838883D0930C14C093DB
:1008C0000B147801C701DF91CF911F910F91FF9019
:1008D000EF90089580917C1590917D15A0917E15E3
:1008E000B0917F150196A11DB11D80937C15909349
:1008F0007D15A0937E15B0937F1508958AE694E048
:100900000E94010C87B7826087BF0895CF93DF9361
:10091000EC011B821A82E0917A15F0917B153097D9
:10092000D9F0288539854A855B8580859185A285A2
:10093000B385281739074A075B07D8F0281B390BFE
:100940004A0B5B0B288739874A875B87FB83EA83DF
:100950000190F081E02DE3CFF983E883309711F027
:10096000D383C283EA81FB81309761F0D183C08356
:100970000DC0821B930BA40BB50B80879187A287B8
:10098000B387EACFD0937B15C0937A15DF91CF91CF
:1009900008950FB6F8940F9280917C1590917D1573
:1009A000A0917E15B0917F150F900FBEBC01CD01B7
:1009B00008958F929F92AF92BF92CF92DF92EF9263
:1009C000FF920F93CF93DF936B017C015A01490192
:1009D00080E190E00E946408EC01892B39F10E94CB
:1009E000C904DC01CB018C0D9D1DAE1DBF1D2091E6
:1009F0000D1430910E1440910F1450911014821B5D
:100A0000930BA40BB50B88879987AA87BB8700FF38
:100A100005C01C821D821E821F8204C0CC82DD8222
:100A2000EE82FF82BD86AC869F868E86CE01DF91E8
:100A3000CF910F91FF90EF90DF90CF90BF90AF904C
:100A40009F908F900895CF92DF92EF92FF920F9335
:100A5000CF93DF936B017C01C701B6010E94D904DB
:100A6000EC01009711F00E948604CE01DF91CF9136
:100A70000F91FF90EF90DF90CF900895CF92DF928B
:100A8000EF92FF920F931F93DC01CB016A01790172
:100A9000BC01CD010E94610CDC01CB019701A601D4
:100AA000BC01CD010E9423051F910F91FF90EF9093
:100AB000DF90CF900895AF92BF92CF92DF92EF92E6
:100AC000FF920F935B016C01611571058105910522
:100AD000D9F162E875E180918415909185150E94A5
:100AE0002807E0918415F091851583E08787E090D1
:100AF0008415F090851501E0970149EA57E0C60199
:100B0000B5010E943E05F701968B858B892B19F064
:100B10000E9464071BC0E0918415F091851582E85E
:100B200095E1908F878B80918215909183159383A7
:100B3000828381E0878780918415909185159093B9
:100B400083158093821502C00E94B4070F91FF9015
:100B5000EF90DF90CF90BF90AF900895CF93DF9349
:100B6000EC01EA81FB8188819981309719F09183AA
:100B7000808304C090937B1580937A15E881F98176
:100B80003097A1F08A819B819383828380859185B0
:100B9000A285B385288539854A855B85820F931F99
:100BA000A41FB51F80879187A287B387CE010E94BB
:100BB000EA08DF91CF910895EF92FF920F931F9370
:100BC000CF93DF930E94C9049B01AC0180910D1467
:100BD00090910E14A0910F14B091101479018A0114
:100BE000E81AF90A0A0B1B0B20930D1430930E140C
:100BF00040930F1450931014C0917A15D0917B1527
:100C0000209709F461C0E114F1040105110509F40C
:100C10005BC088859985AA85BB85E816F9060A0711
:100C20001B0760F48E199F09A00BB10B8887998769
:100C3000AA87BB87EE24FF24870108C0E81AF90AB7
:100C40000A0B1B0B188619861A861B8688859985C0
:100C5000AA85BB850097A105B10551F5EC85FD85F9
:100C6000309721F06E857F85CE0109958C819D811D
:100C7000AE81BF8188879987AA87BB870097A10526
:100C8000B10521F4CE010E94AE0512C0E0917A15A3
:100C9000F0917B150190F081E02DF0937B15E093AE
:100CA0007A15309711F013821282CE010E948604C9
:100CB000C0917A15D0917B15209731F0E114F104A1
:100CC0000105110509F0A5CFDF91CF911F910F917B
:100CD000FF90EF900895EF92FF920F931F930E9461
:100CE000C9047B018C010E945C0C9B01AC01C80112
:100CF000B7010E948C7DCA01B9011F910F91FF902D
:100D0000EF9008956F927F928F929F92AF92BF92D1
:100D1000CF92DF92EF92FF920F931F930E94C9042C
:100D20005B016C010E945C0C9B01AC01C601B5012A
:100D30000E948C7D79018A010E945C0C9B01AC01B0
:100D4000C801B7010E944E7DDC01CB01A81AB90A87
:100D5000CA0ADB0A88EE682E83E0782E812C912C5B
:100D6000C801B701A40193010E944E7D7B018C0153
:100D7000C601B5010E944E7D5B016C010E945C0CB6
:100D80009B01AC01C601B5010E948C7DE20EF31EF1
:100D9000041F151FC801B7011F910F91FF90EF901D
:100DA000DF90CF90BF90AF909F908F907F906F908B
:100DB0000895CF93DF93DC019B01EC01788F6F8B5B
:100DC0001D821C820FB6F8940F92EB01E881F98125
:100DD0008FEFEF3FF80749F4E0E0F0E0ED018C81A0
:100DE0009D8101969D838C8316C03097A1F00F9052
:100DF0000FBE8289ED019A89981750F09F012E5FEE
:100E00003F4F0280F381E02D309711F08289F4CFBB
:100E10000FB6F8940F92ED01FB83EA83F901B183D9
:100E2000A083EA81FB81309771F084819581892BC1
:100E300051F08C819D8124813581820F931F9D8388
:100E40008C83158214820F900FBEDF91CF9108958D
:100E5000CF93DF939C01DB010FB6F8940F92ED91D5
:100E6000FC9111970F900FBE8FEFEF3FF80749F1FC
:100E7000309739F182819381E217F307E9F40FB6D5
:100E8000F8940F9211969C938E9384819581892B6F
:100E900059F0A281B381109729F084819581ED01E9
:100EA0009D838C83158214820F900FBEF9011382EB
:100EB0001282108E178A05C0DF011296FC01892B61
:100EC000C9F6DF91CF910895CF93DF93C09180153C
:100ED000D0918115209709F10FB6F8940F928C816B
:100EE0009D810F900FBE892BA1F0EF89F88D0FB671
:100EF000F8940F928C819D8101979D838C838081D2
:100F000091810F900FBE8F5F9F4F19F0CF010E940C
:100F1000690A0990D881C02DDDCF0E94DC05E091DF
:100F20008415F09185158091821590918315E817AD
:100F3000F90761F08785813011F482E087870FB669
:100F4000F8940F920E940F0B0F900FBEDF91CF917C
:100F50000895FB01168A158A82E0878762E875E1A9
:100F6000CF010E94D9060895E0918415F09185156E
:100F700082819381892B69F062E875E1CF010E943B
:100F8000280762E875E180918415909185150E948B
:100F9000D9060E9464070895E0918615F09187159F
:100FA000309741F0838994890E94EA08109287154E
:100FB0001092861508950F931F93CF93DF93C091DE
:100FC0008015D091811500E815E10E94CC0720978B
:100FD00081F0809184159091851528813981C817F9
:100FE000D90721F4F8013183208303C08E01E90180
:100FF000EECF8091841590918515909387158093FD
:101000008615DF91CF911F910F9108951F93CF9374
:10101000182FE0918415F0918515C28962E875E179
:10102000CF010E942807E0918415F0918515128B5D
:101030001F3F49F062E875E1809184159091851514
:101040000E94D90602C00E94DB07E0918415F0914E
:1010500085158091821590918315E817F90719F489
:1010600081E0878709C082E087870FB6F8940F92E6
:101070000E940F0B0F900FBE8C2F9927CF911F91BD
:1010800008958FEF0E94060808950F931F93CF9342
:10109000DF938C01C0918015D0918115209769F064
:1010A000B801CE0106960E94207D892B11F4CE0155
:1010B00006C00990D881C02DF1CF80E090E0DF918B
:1010C000CF911F910F910895CF93DF93AC01C0E0B2
:1010D000D0E0DE0180911114909112144817590745
:1010E00020F05FC0EF01DB0129C04A5F5F4F443051
:1010F000510510F444E050E0E0918815F091891515
:1011000068E875E1309709F44CC0208131812417DB
:10111000350760F02417350729F3209729F08881D7
:1011200099812817390710F4EF01DB01BF016E5FC9
:101130007F4F0280F381E02D309739F7209789F1B6
:10114000CA010A96288139816A817B8182179307B7
:1011500070F4FE01E40FF51F241B350B318320834F
:101160007383628359834883ED93FC9302C06D932C
:101170007C938091111490911214E881F9818E1B57
:101180009F0B9093121480931114EC0FFD1F349752
:101190008FEE9EEBADEABEED80839183A283B38395
:1011A0002296CE01DF91CF9108950F931F93CF9395
:1011B000DF938C010E946408EC01009729F0A801DC
:1011C00060E070E00E94167DCE01DF91CF911F910B
:1011D0000F910895EF92FF920F931F93CF93DF9398
:1011E0002EEFE22E2FEFF22EE80EF91ED7014D91D1
:1011F0005C91E0918815F091891508E815E1309728
:1012000009F44BC0B701640F751F808191819F0164
:10121000280F391F2E153F05D1F49C01240F351FCF
:1012200031832083DF01A20FB31F82819381A8172E
:10123000B90799F58D919C911197280F391F31832A
:101240002083ED018A819B819383828326C0EE16E1
:10125000FF06A0F4D801ED92FC926E177F0751F4BF
:10126000840F951FE70199838883828193819B83F3
:101270008A8313C0E701FB83EA830FC0E216F306FB
:1012800018F48FEF9FEF1DC08F010E5F1F4F02807C
:10129000F381E02D309709F0B8CF309731F4E701B2
:1012A000FB83EA83F801F182E0828091111490912E
:1012B0001214840F951F909312148093111480E0E0
:1012C00090E0DF91CF911F910F91FF90EF900895E3
:1012D000FC0161937193CF010E94EA080895809107
:1012E000111490911214089543E150E06AE875E1F9
:1012F00080E090E00E94010B9C01892B61F48091B9
:101300008A15833141F480918B158F3421F48091BB
:101310008C15833519F08FEF9FEF0895C90108955B
:1013200083E180938A158FE480938B1583E5809306
:101330008C1543E150E06AE875E180E090E00E949E
:10134000040B009711F08FEF9FEF0895CF93DF9379
:10135000AC01DB010FB6F8940F92CD91DC9111979F
:101360000F900FBE8FEFCF3FD80709F436C02097FC
:10137000A1F18D899E892A813B818417950741F5CA
:101380000FB6F8940F9211963C932E938C819D8109
:10139000892B81F0EA81FB81309729F08C819D8136
:1013A0009583848305C08FEF9FEF11969C938E9356
:1013B0001D821C820F900FBE82E08F8762E875E16C
:1013C000CE010E94D9068FEF9FEF9E8B8D8B05C0BB
:1013D000DE011296E901232B61F6DF91CF9108958A
:1013E000AF92BF92CF92DF92EF92FF920F93CF9383
:1013F000DF93EC015A016B010FB6F8940F928881CC
:1014000099810F900FBE8F5F9F4F51F40FB6F894E4
:101410000F92198218820F900FBE0E94B4073CC031
:1014200062E875E180918415909185150E942807E6
:10143000BE0180918415909185150E94D906E09196
:101440008415F091851583E08787E0908415F090EE
:101450008515A114B104C104D10461F001E09E011D
:1014600046EA59E0C601B5010E943E05F701968B98
:10147000858B03C0F701168A158A0E946407E091E4
:101480008415F0918515858996892FEF8F3F9207F6
:1014900019F4168A158A02C080E090E0DF91CF919E
:1014A0000F91FF90EF90DF90CF90BF90AF90089595
:1014B000FC010FB6F8940F92808191818F5F9F4F4E
:1014C00011F4118210820F900FBECF010E94F0091B
:1014D0000895CF93DF93DC010FB6F8940F92CD916E
:1014E000DC9111970F900FBE8FEFCF3FD80709F413
:1014F0003AC0209771F10FB6F8940F92EA81FB8100
:101500001196FC93EE938C819D81892B71F030971D
:1015100029F08C819D819583848305C08FEF9FEF97
:1015200011969C938E931D821C820F900FBE8D8905
:101530009E89009721F00E94AE051E8A1D8A82E0D6
:101540008F8762E875E1CE010E94D90681E090E0C4
:101550000CC00FB6F8940F928FEF9FEF11969C93EB
:101560008E930F900FBE80E090E0DF91CF910895B1
:101570000F931F930E94690A8C010E94B407C8014F
:101580001F910F9108950F931F93CF93DF93EC0159
:1015900000E010E00FB6F8940F92888199810F90C7
:1015A0000FBE2FEF8F3F920741F40FB6F8940F92C2
:1015B000198308830F900FBE13C0892B89F0CE01C9
:1015C0000E94690A080F191F0FB6F8940F928881BC
:1015D00099810F900FBE009719F08F5F9F4F79F799
:1015E000C801DF91CF911F910F9108950F931F9321
:1015F0000E94C30A8C010E94B407C8011F910F9179
:1016000008950E94CC1508950E94DC1508959F91BD
:101610008F910F900BBE0F900FBE1F9018952F92B9
:101620003F924F925F926F927F928F929F92AF9272
:10163000BF92CF92DF92EF92FF920F931F93CF93BF
:10164000DF938DB79EB7E0918415F0918515918B4E
:10165000808BE0918215F0918315F0938515E093CE
:10166000841581E08787E0918415F0918515808944
:1016700091898DBF9EBFDF91CF911F910F91FF90F8
:10168000EF90DF90CF90BF90AF909F908F907F9022
:101690006F905F904F903F902F900895AF92BF92C0
:1016A000CF92DF92EF92FF920F931F93CF93DF932E
:1016B0007C016B015A01E901C90149960E94640845
:1016C000FC01009709F478C08C010C0F1D1FB801B4
:1016D00067507040A8014B515040C801069628E061
:1016E000D7010D907D01EC010992CE012150C1F787
:1016F000E8012E8741505040598B488B4F5F5F4F18
:10170000FC8BEB8B8FEE9EEBADEABEED808391837D
:10171000A283B38384839583A683B78380879187CD
:10172000A287B38784879587A687B78780E48A8B4B
:101730008D2D9927FB018583C68280E883832283D0
:101740002483A1828B2D9927808327E03BE0832F80
:101750009927EA018A8B2B8B8091801590918115B6
:10176000F801918380831093811500938015C2E066
:10177000C787168A158A108E178A62E875E1C80134
:101780000E94D906E0918415F0918515309721F4D7
:101790000FB6F8940F925DCF8091821590918315CA
:1017A000E817F90741F0C7870FB6F8940F920E9427
:1017B0000F0B0F900FBEC801DF91CF911F910F91BA
:1017C000FF90EF90DF90CF90BF90AF9008951F9360
:1017D000182F8091131490911414A0911514B091A6
:1017E0001614BC01CD0120EA3FE040E050E00E9429
:1017F0008C7DE22FF32F3197F1F71A95D1F71F91D6
:101800000895BC0187B78D7F87BF80B7886080BF90
:1018100012BE82E083BF80B7992787709070892BB2
:10182000D1F781E086BF0FB6F8940F9281E090E087
:10183000A0E0B0E0B6B7B170E9F3B6BF0894811D7F
:10184000911DA11DB6B7B170C9F3BB270F900FBE94
:1018500027E0880F991FAA1FBB1F2A95D1F78093F5
:10186000131490931414A0931514B093161487B7FF
:101870008D7F87BF80B7886080BF12BE89E083BF3D
:101880008FE181BF80B7482F5527477050704115B1
:101890005105C1F782E086BF89E393E00E94CE71D3
:1018A00008958091131490911414A0911514B0917F
:1018B0001614BC01CD01089560E074E080E090E072
:1018C0000895EF92FF920F931F937B018C010E946A
:1018D0005C0C9B01AC01C801B7010E944E7DDC018C
:1018E000CB01BC01CD0128EE33E040E050E00E9486
:1018F0008C7D211531054105510521F421E030E0B1
:1019000040E050E0CA01B9011F910F91FF90EF90A4
:1019100008959C01FB0160E070E087B7482F5527D0
:101920004270507087B78D7F87BF20313105C1F07D
:10193000213131053CF42115310571F0213031059B
:1019400061F024C02231310541F12231310514F119
:1019500020323105B1F01AC0AB0182E086BF18C059
:1019600006B601FE05C081E090E09183808302C04D
:10197000718360834115510559F0808191818068A0
:1019800002C08EE090E09183808302C06FEF7FEF12
:10199000452B19F087B7826087BFCB0108951F924E
:1019A0000F920FB60F9211242F933F934F935F9393
:1019B0006F937F938F939F93AF93BF93EF93FF9317
:1019C00089E393E00E94C371FF91EF91BF91AF91C2
:1019D0009F918F917F916F915F914F913F912F9147
:1019E0000F900FBE0F901F901895559A89B78F7E54
:1019F00089BF0895CF93DF93DC01EC01EA81FB817D
:101A000020911814422F5527CA0180739070892B9A
:101A100089F044FF04C083E18CB9206403C081E1F4
:101A20008CB92F7B20931814809118148F7C80938D
:101A3000181454C027FF02C0559850C0ED018A8584
:101A40009B850097A9F180911B14882339F00C9B8A
:101A500005C0559889B7806189BF40C0ED018A856E
:101A60009B8501979B878A8780911914882311F0A1
:101A7000509A01C0509881918CB9ED018E819F815F
:101A8000E817F90711F4EC81FD81ED01FB83EA838E
:101A90002A853B858C859D8528173907F9F4E889C7
:101AA000F989309769F08FEFEF3FF807B9F011C06F
:101AB0005598ED019B878A87E889F989309729F441
:101AC0008FEF9FEF998B888B09C08FEFEF3FF8075F
:101AD00029F084819581019695838483DF91CF914C
:101AE0000895CF93DF93DC01809117149BB1892B6C
:101AF000809317143CB120911814222361F03331E4
:101B000019F45598206804C0313129F4559A2F777B
:101B1000209318145FC0ED014A855B8588859985FF
:101B20004817590730F08091171488608093171474
:101B300051C04F5F5F4F41305105A1F4ED01E8897D
:101B4000F989309729F48FEF9FEF998B888B2AC002
:101B50008FEFEF3FF80731F18481958101969583EE
:101B6000848320C0222399F0ED018E859F8548173C
:101B70005907C0F026FD16C05D9B05C083E18CB9F6
:101B800020642F7D01C02062209318140BC0809127
:101B90001A14882339F0FD0186859785481759075F
:101BA00008F01A9AED91FC91119731931196FC93DC
:101BB000EE932D913C911197ED018E819F81281715
:101BC000390729F48C819D8111969C938E93FD0198
:101BD00053874287DF91CF9108950FB6F8940F9203
:101BE00088EB8AB90F900FBE08950FB6F8940F9244
:101BF0005798569855980F900FBE8AE00E94E70BB1
:101C0000549853980895AF92BF92CF92DF92EF927B
:101C1000FF920F931F93CF93DF9389B1C82FDD27D6
:101C2000809190009927982F8827C82BD92B8091D5
:101C3000950086FF06C022E0A22EB12CC12CD12C2B
:101C40000DC0599B06C098E0A92EB12CC12CD12CF7
:101C500005C080E1A82EB12CC12CD12C0E94510CC2
:101C60007B018C019E01442755272F5F3F4F4F4F2B
:101C70005F4FC601B5010E944E7D9B01AC01C801BA
:101C8000B7010E948C7DCA01B901DF91CF911F91EC
:101C90000F91FF90EF90DF90CF90BF90AF9008959D
:101CA000EF92FF920F931F937B018C010E94F50D21
:101CB0008091950086FD11C0599B08C072E0EE0C22
:101CC000FF1C001F111F7A95D1F707C063E0EE0CCF
:101CD000FF1C001F111F6A95D1F70E94510CDC01F7
:101CE000CB01BC01CD01A80197010E948C7DDA01D6
:101CF000C9010196A11DB11DB695A7959795879528
:101D0000019789B9892F9927809390000E94ED0D42
:101D100080E090E01F910F91FF90EF900895529B0B
:101D200003C089E090E008958091950082FF0AC089
:101D30008091950081FF03C088E090E0089587E0DE
:101D400090E008958091950081FF03C086E090E0C7
:101D5000089585E090E00895CF93C82F0E94F50D77
:101D60005298809195008D7F809395008091950089
:101D70008B7F809395008C2F992787309105B1F048
:101D8000883091051CF4069739F015C0883091050C
:101D900041F0099729F00FC080919500826009C039
:101DA000529A809195008260809395008091950071
:101DB0008460809395000E94ED0D0E948F0E8C1719
:101DC00019F08FEF9FEF02C080E090E0CF9108956F
:101DD0008091950099279C012072307085FF0AC080
:101DE0008091950084FF03C081E090E0089582E037
:101DF00090E00895C9010895CF93C82F0E94F50D72
:101E00008C2F99278130910591F0823091051CF437
:101E1000892B21F01AC0029771F017C080919500AC
:101E20008F7E80939500809195008F7D0CC080916E
:101E30009500806103C0809195008F7E809395000E
:101E4000809195008062809395000E94ED0D0E9424
:101E5000E80E8C1719F08FEF9FEF02C080E090E042
:101E6000CF9108958091950083FF03C082E090E0B8
:101E7000089581E090E00895CF93C82F0E94F50D5A
:101E8000C13021F480919500877F05C0C23029F4CC
:101E9000809195008860809395000E94ED0D0E94CE
:101EA000320F8C1719F08FEF9FEF02C080E090E0A7
:101EB000CF91089520E030E040E050E08091171489
:101EC000992784FF04C021E030E040E050E083FD2A
:101ED000226082FD246080911814882321F086FD01
:101EE000426087FD48601A9B07C0326080911A14D7
:101EF000882319F0426001C031600C9B07C0386034
:101F000080911B14882319F0426001C0346041FFA6
:101F1000416043FF446080911914882311F04064AC
:101F200001C04068589B02C0406101C04062CA01C4
:101F3000B9010895EF92FF920F931F937B018C01DB
:101F4000809118148823D9F00FB6F8940F9200FFEF
:101F500002C08F7B03C001FF03C08064809318140C
:101F600002FF04C0809118148F7705C003FF05C0DD
:101F7000809118148068809318140F900FBE809180
:101F80001A14882321F001FD1A9A00FD1A98F1FC19
:101F90001A9AF0FC1A9806FF03C081E08093191486
:101FA00007FF02C01092191404FD589A05FD5898B5
:101FB000D801C70181709070A070B070892B29F092
:101FC000809117148F7E80931714E1FE05C08091D5
:101FD0001714877F80931714E2FE05C080911714B1
:101FE0008B7F809317140E945A0FDC01CB01887FEE
:101FF0008E159F05A007B10719F08FEF9FEF02C064
:1020000080E090E01F910F91FF90EF90089590E095
:102010008091950086FF09C091E0129993E080912C
:10202000950080FF04C0946002C0599990E2892F06
:1020300099270895CF93C82F0E94F50D8C2F9927CB
:1020400080FF13C081FF02C0129A01C0129882FF64
:1020500004C080919500816003C0809195008E7FBF
:102060008093950059985E9A0FC085FF02C0599AD7
:1020700001C05998809195008E7F80939500809142
:1020800095008F7B809395000E94ED0D0E940710B4
:102090008C1719F08FEF9FEF02C080E090E0CF9196
:1020A000089520E030E040E050E08091181488234B
:1020B00021F020E230E040E050E080911A148823C3
:1020C00011F0216001C02E7F80911B14882311F034
:1020D000226001C02D7FCA01B9010895EF92FF92DD
:1020E0000F931F937B018C0165FF0BC08091181427
:1020F000882371F40FB6F8940F9281E4809318143A
:1021000005C00FB6F8940F92109218140F900FBEDE
:10211000D801C70181709070A070B070892B31F028
:102120001A9A129A81E080931A1407C080911A14A7
:10213000882319F010921A141298E1FE10C040E0A2
:1021400050E065EF7CE089E494E00E94CE71892B39
:10215000E9F41C9A149881E080931B140EC08091BE
:102160001B14882351F010921B1440E050E0BA0178
:1021700089E494E00E94CE7114980E945110DC0111
:10218000CB018E159F05A007B10719F08FEF9FEFC8
:1021900002C080E090E01F910F91FF90EF900895B2
:1021A000559A0895909118149923A9F096FF13C099
:1021B0000FB6F8940F925D9B04C081E18CB99F7EAD
:1021C00001C0906190931814809118148F798093B6
:1021D00018140F900FBE80911A1481111A98089547
:1021E000CF93DF9344E853E061E77DE08DE394E033
:1021F0000E94CE71EC01892B81F442E753E06AEF33
:102200007CE083E494E00E94CE71009741F0AE013F
:10221000BE018DE394E00E94CE718FEF9FEFDF91BE
:10222000CF91089540E050E0BA018DE394E00E9420
:10223000CE7140E050E0BA0183E494E00E94CE7198
:1022400080911B14882351F010921B14149840E0C5
:1022500050E0BA0189E494E00E94CE7180911A1492
:10226000882319F010921A14129880E090E00895D3
:1022700080919A00806280939A0089B78F7D89BF90
:1022800008951F920F920FB60F9211242F933F9330
:102290008F939F93AF93BF93CF93DF93EF93FF936E
:1022A000AEEEB3E0E091F003F091F1032091F8037A
:1022B0003091F9032115310509F450C080912014A3
:1022C000882359F00D9B09C080919A008F7D8093DF
:1022D0009A0089B7806289BF60C08091F8039091AD
:1022E000F9030197ED019B878A8780911E1488234B
:1022F00021F080919A00816003C080919A008E7FC6
:1023000080939A00819180939C008091F403909136
:10231000F503E817F90721F4E091F203F091F303D4
:10232000ED01FB83EA832091F8033091F90380915A
:10233000FA039091FB032817390779F5E091FE0322
:10234000F091FF03309729F48FEF9FEF998B888BE3
:1023500024C08FEFEF3FF80701F11AC080919A0077
:102360008F7D80939A003093F9032093F803E091D6
:10237000FE03F091FF03309739F48FEF9FEF9093B6
:10238000FF038093FE0309C0CFEFEF3FFC0729F066
:1023900084819581019695838483FF91EF91DF91EC
:1023A000CF91BF91AF919F918F913F912F910F90BE
:1023B0000FBE0F901F9018951F920F920FB60F929D
:1023C00011242F933F934F935F936F938F939F931A
:1023D000AF93BF93EF93FF93A0E0B4E060E0209150
:1023E0001C1480919B00282B20931C1430919C007E
:1023F00040910A0450910B048091080490910904C3
:102400004817590708F045C04F5F5F4F41305105ED
:1024100011F461E00CC080911F14882341F0809179
:102420000E0490910F044817590708F0949AE09110
:102430000004F09101043193F0930104E09300044F
:1024400020910004309101048091060490910704CA
:102450002817390741F48091040490910504909362
:10246000010480930004FD015387428780919B0003
:1024700088230CF4B4CF6623C9F0E0911004F091E6
:102480001104309751F48FEF9FEFFD01918B808BFA
:102490000DC0286020931C1409C08FEFEF3FF80790
:1024A00029F084819581019695838483FF91EF9132
:1024B000BF91AF919F918F916F915F914F913F919C
:1024C0002F910F900FBE0F901F9018950FB6F89494
:1024D0000F9288EB80939A000F900FBE08950FB66D
:1024E000F8940F9280919A008F7780939A00809150
:1024F0009A008F7B80939A0080919A008F7D8093C1
:102500009A000F900FBE8AE00E94E70B80919A001C
:102510008F7E80939A0080919A00877F80939A00A3
:102520000895AF92BF92CF92DF92EF92FF920F93F6
:102530001F93CF93DF9380919900C82FDD2780915F
:1025400098009927982F8827C82BD92B80919D0018
:1025500086FF06C022E0A22EB12CC12CD12C0FC0C8
:1025600080919B0081FF06C098E0A92EB12CC12C60
:10257000D12C05C080E1A82EB12CC12CD12C0E94F9
:10258000510C7B018C019E01442755272F5F3F4F43
:102590004F4F5F4FC601B5010E944E7D9B01AC01BC
:1025A000C801B7010E948C7DCA01B901DF91CF91AA
:1025B0001F910F91FF90EF90DF90CF90BF90AF9061
:1025C0000895EF92FF920F931F937B018C010E945D
:1025D0006F1280919D0086FD13C080919B0081FF4A
:1025E00008C072E0EE0CFF1C001F111F7A95D1F796
:1025F00007C063E0EE0CFF1C001F111F6A95D1F7A6
:102600000E94510CDC01CB01BC01CD01A801970156
:102610000E948C7DDA01C9010196A11DB11DB695FC
:10262000A79597958795019780939900892F99276A
:10263000809398000E94661280E090E01F910F91B5
:10264000FF90EF90089580919A0082FF03C089E087
:1026500090E0089580919D0082FF0AC080919D00C6
:1026600081FF03C088E090E0089587E090E008953E
:1026700080919D0081FF03C086E090E0089585E091
:1026800090E00895CF93C82F0E946F1280919A0016
:102690008B7F80939A0080919D008D7F80939D0019
:1026A00080919D008B7F80939D008C2F9927873090
:1026B0009105D1F0883091051CF4069739F019C0C6
:1026C0008830910561F0099729F013C080919D0031
:1026D00082600DC080919A00846080939A008091FE
:1026E0009D00826080939D0080919D008460809316
:1026F0009D000E9466120E9423138C1719F08FEF21
:102700009FEF02C080E090E0CF91089580919D00FE
:1027100099279C012072307085FF0AC080919D002E
:1027200084FF03C081E090E0089582E090E0089586
:10273000C9010895CF93C82F0E946F128C2F99273B
:102740008130910591F0823091051CF4892B21F0A4
:102750001AC0029771F017C080919D008F7E809300
:102760009D0080919D008F7D0CC080919D008061B7
:1027700003C080919D008F7E80939D0080919D007D
:10278000806280939D000E9466120E9486138C17BF
:1027900019F08FEF9FEF02C080E090E0CF91089595
:1027A00080919D0083FF03C082E090E0089581E066
:1027B00090E00895CF93C82F0E946F12C13021F48A
:1027C00080919D00877F05C0C23029F480919D00D3
:1027D000886080939D000E9466120E94D0138C171F
:1027E00019F08FEF9FEF02C080E090E0CF91089545
:1027F00020E030E040E050E080911C14992784FFF5
:1028000004C021E030E040E050E083FD226082FD22
:10281000246080911D14882321F086FD426087FD8D
:102820004860949B07C0326080911F14882319F080
:10283000426001C031600D9B07C038608091201458
:10284000882319F0426001C0346041FF416043FFBA
:10285000446080911E14882311F0406401C04068D8
:1028600080919B0080FF02C0406101C04062CA01AC
:10287000B9010895EF92FF920F931F937B018C0192
:1028800080911D148823D9F00FB6F8940F9200FFA1
:1028900002C08F7B03C001FF03C0806480931D14BE
:1028A00002FF04C080911D148F7705C003FF05C08F
:1028B00080911D14806880931D140F900FBE80912D
:1028C0001F14882321F001FD949A00FD9498F1FCD7
:1028D000949AF0FC949806FF03C081E080931E1444
:1028E00007FF02C010921E1404FF05C080919B00D8
:1028F000816080939B0005FF05C080919B008E7FC7
:1029000080939B00D801C70181709070A070B07057
:10291000892B29F080911C148F7E80931C14E1FE7A
:1029200005C080911C14877F80931C14E2FE05C0B3
:1029300080911C148B7F80931C140E94F813DC017F
:10294000CB01887F8E159F05A007B10719F08FEF87
:102950009FEF02C080E090E01F910F91FF90EF90F9
:10296000089590E080919D0086FF09C091E0129942
:1029700093E080919D0080FF06C0946004C0809128
:102980009B0081FD90E2892F99270895CF93C82F4E
:102990000E946F128C2F992780FF1BC081FF02C0FD
:1029A000129A01C0129882FF04C080919D0081603C
:1029B00003C080919D008E7F80939D0080919B003D
:1029C0008D7F80939B0080919B00806480939B000F
:1029D00015C085FF04C080919B00826003C0809178
:1029E0009B008D7F80939B0080919D008E7F8093C4
:1029F0009D0080919D008F7B80939D000E946612B8
:102A00000E94B1148C1719F08FEF9FEF02C080E085
:102A100090E0CF91089520E030E040E050E08091D8
:102A20001D14882321F020E230E040E050E0809146
:102A30001F14882311F0216001C02E7F8091201483
:102A4000882311F0226001C02D7FCA01B9010895C9
:102A5000EF92FF920F931F937B018C0165FF0BC0D8
:102A600080911D14882371F40FB6F8940F9281E4BD
:102A700080931D1405C00FB6F8940F9210921D1488
:102A80000F900FBED801C70181709070A070B07018
:102A9000892B31F0949A8C9A81E080931F1407C09F
:102AA00080911F14882319F010921F148C98E1FE56
:102AB00010C040E050E068E371E187E394E00E94D9
:102AC000CE71892BE9F41D9A159881E0809320142A
:102AD0000EC080912014882351F01092201440E001
:102AE00050E0BA0187E394E00E94CE7115980E94ED
:102AF0000B15DC01CB018E159F05A007B10719F05E
:102B00008FEF9FEF02C080E090E01F910F91FF9048
:102B1000EF90089580919A00806280939A000895C2
:102B200090911D149923C1F096FF16C00FB6F8942A
:102B30000F9280919B0085FF05C081E180939C00EE
:102B40009F7E01C0906190931D1480911D148F7918
:102B500080931D140F900FBE80911F1481119498C3
:102B6000089580E090E0089580912014882351F02A
:102B700010922014159840E050E0BA0187E394E0E9
:102B80000E94CE7180911F14882319F010921F1497
:102B90008C9880E090E00895CF93DF93EA01DC0108
:102BA000FB01219724F00E94FC7D0192FACF80E086
:102BB00090E0DF91CF910895CF93DF93EC01FB017B
:102BC00060E070E06417750790F4DE01A60FB71F90
:102BD0009D010E94FC7D802D9081891721F0D901F3
:102BE000092E0E94047E31966F5F7F4FEBCF80E00D
:102BF00090E0DF91CF9108959C01FB01A0E0B0E04F
:102C000089B7482F55274072507089B78F7D89BF8B
:102C10002131310509F479C0223131056CF42130BC
:102C2000310519F1223031051CF4232BC1F069C0A4
:102C300020313105E9F065C02831310551F12931E4
:102C400031052CF42231310509F462C05AC0293112
:102C5000310589F12032310509F44EC052C08AB7DE
:102C60008B7F8ABF8AB7877F8ABF80E288BF4BC0CD
:102C700008B605FE05C081E090E09183808302C024
:102C8000B183A08341155105F1F180819181806864
:102C900035C08AB7982F987083FD2EC0943019F4F0
:102CA00087E090E02BC0983019F486E090E026C0D1
:102CB00081E090E023C0608171816130710519F479
:102CC0008AB78B7F05C06730710531F48AB784609D
:102CD0008ABF8AB7877F0EC06530710519F48AB73D
:102CE0008B7F05C06630710561F48AB784608ABF46
:102CF0008AB788608ABF07C085E090E091838083AF
:102D000002C0AFEFBFEF452B19F089B7806289BFD2
:102D1000CD0108951F920F920FB60F9211242F9399
:102D20003F934F935F936F937F938F939F93AF9353
:102D3000BF93EF93FF9387E394E00E94C371FF91E9
:102D4000EF91BF91AF919F918F917F916F915F9123
:102D50004F913F912F910F900FBE0F901F9018959C
:102D60009C01FB0160E070E08AB1482F5527407854
:102D70005070579820313105C1F0213131053CF4B4
:102D80002115310571F02130310561F023C0223168
:102D9000310529F1223131050CF120323105A9F03C
:102DA00019C0AB018CB18CB117C05F9B05C081E02D
:102DB00090E09183808302C0718360834115510547
:102DC00059F080819181806802C080E190E0918318
:102DD000808302C06FEF7FEF452B09F0579ACB013C
:102DE00008951F920F920FB60F9211242F933F93C5
:102DF0004F935F936F937F938F939F93AF93BF9303
:102E0000EF93FF938DE394E00E94C371FF91EF91E4
:102E1000BF91AF919F918F917F916F915F914F91F2
:102E20003F912F910F900FBE0F901F9018959C010E
:102E3000FB0160E070E08AB1482F55274072507066
:102E400055982131310551F1223131053CF42115DC
:102E5000310529F12031310541F01CC02231310505
:102E6000F1F02032310589F015C05D9B05C081E08D
:102E700090E09183808302C0718360834115510586
:102E800059F080819181806802C080E190E0918357
:102E9000808302C06FEF7FEF452B09F0559ACB017D
:102EA00008951F920F920FB60F9211242F933F9304
:102EB0004F935F936F937F938F939F93AF93BF9342
:102EC000EF93FF9383E494E00E94C371FF91EF912D
:102ED000BF91AF919F918F917F916F915F914F9132
:102EE0003F912F910F900FBE0F901F9018959C014E
:102EF000FB01A0E0B0E089B7482F55274071507022
:102F000089B78F7E89BF2131310509F47DC0223117
:102F100031056CF42130310519F1223031051CF4F2
:102F2000232BC1F06DC020313105E9F069C0283193
:102F3000310559F1293131052CF42231310509F4DB
:102F400066C05EC029313105A9F12032310509F48E
:102F500052C056C08AB78E7F8ABF8AB78D7F8ABF1C
:102F600080E188BF4FC008B604FE05C081E090E054
:102F70009183808302C0B183A0834115510509F478
:102F800041C080819181806838C08AB7982F927043
:102F900081FF03C085E090E030C0913019F487E0F4
:102FA00090E02BC0923019F486E090E026C081E0DA
:102FB00090E023C0608171816130710519F48AB796
:102FC0008E7F05C06730710531F48AB781608ABF92
:102FD0008AB78D7F0EC06530710519F48AB78E7F70
:102FE00005C06630710561F48AB781608ABF8AB70F
:102FF00082608ABF07C084E090E09183808302C032
:10300000AFEFBFEF452B19F089B7806189BFCD01C4
:1030100008951F920F920FB60F9211242F933F9392
:103020004F935F936F937F938F939F93AF93BF93D0
:10303000EF93FF9389E494E00E94C371FF91EF91B5
:10304000BF91AF919F918F917F916F915F914F91C0
:103050003F912F910F900FBE0F901F901895FC017C
:10306000808191810895CF92DF92EF92FF920F932A
:103070001F93CF93DF936C01CB010E94871D7C01CE
:103080008F5F9F4FC9F123E08091550490915604C2
:10309000892B61F0273050F52F5FE22FFF27EE0FCD
:1030A000FF1FE15BFB4F80819181F2CFC22FDD27B3
:1030B000CC0FDD1FC15BDB4F87E090E00E94031A5D
:1030C0008C0199838883009721F1B701C6010E9482
:1030D0009519F801918380838F5F9F4F81F48881D8
:1030E00099810E94101A1982188206C087E190E027
:1030F0009093E8158093E71580E090E00AC0E8819E
:10310000F981F382E2821482E881F98116821582C4
:10311000CF01DF91CF911F910F91FF90EF90DF9042
:10312000CF9008958F929F92BF92CF92DF92EF92AD
:10313000FF920F931F93CF93DF934C01CB01EA01D2
:103140000E94871D6C018F5F9F4F09F445C0BB240F
:1031500080914F04909150048C179D0769F0B394AF
:1031600087E08B1598F1EB2DFF27EE0FFF1FE15B3A
:10317000FB4F80819181F0CFEB2CFF24E701CE0D36
:10318000DF1DC15BDB4F87E090E00E94031A8C01DA
:1031900099838883009769F1B601C4010E9495194B
:1031A000F801918380838F5F9F4FC9F48881998153
:1031B0000E94101A22E02B1530F00894E11CF11C3B
:1031C000F982E88209C01982188206C089E090E07D
:1031D0009093E8158093E71580E090E00AC0E881BD
:1031E000F981D382C2821482E881F9811682158224
:1031F000CF01DF91CF911F910F91FF90EF90DF9062
:10320000CF90BF909F908F900895CF93DF93CDB7CD
:10321000DEB7E5E0F0E0EC0FFD1F81919191AF0189
:10322000BC0180915104909152040E944019DF9199
:10323000CF91089560915104709152040E94EB1D4A
:103240002FEF8F3F920751F060915104709152041B
:103250008AE090E00E94C31D80E090E00895CF9343
:10326000DF93CDB7DEB78F819885AE01475F5F4FA3
:10327000BC018D819E810E946219DF91CF910895DA
:10328000FC019A01AB016081718180EF99E10E949C
:103290003B1A0895EF92FF920F931F937C018A01CE
:1032A000F701808191810E94097DF70180819181E0
:1032B000800F911F91838083C8011F910F91FF9010
:1032C000EF900895CF93DF93CDB7DEB722970FB677
:1032D000F894DEBF0FBECDBF9A8389839A01AB01FC
:1032E000BE016F5F7F4F8AE499E10E943B1AE9813A
:1032F000FA81108222960FB6F894DEBF0FBECDBFC2
:10330000DF91CF910895CF93DF93EC01AA81BB8128
:10331000109719F4EB85FC8504C0ED01ED89FE8959
:10332000CD010995DF91CF910895CF92DF92EF9271
:10333000FF920F931F93CF93DF93CDB7DEB72997FB
:103340000FB6F894DEBF0FBECDBF7B018C0120E02D
:10335000DC018C91882381F08A3371F0FE01319673
:103360000F5F1F4F81932F5FD8018C91882321F02D
:103370008A3311F02830A0F3CE010196FC01E20F50
:10338000F11D10820E941904DC01892B49F482E0AE
:1033900090E09093E8158093E7158FEF9FEF11C0B1
:1033A000F80181918F018A3311F000E010E0FD01F6
:1033B000C58CD68C20E030E0A701B801CD01F60124
:1033C000099529960FB6F894DEBF0FBECDBFDF91E9
:1033D000CF911F910F91FF90EF90DF90CF900895C4
:1033E000CF93DF93DC01EC01EA81FB81309719F484
:1033F000EF81F88503C0018CF28DE02DCD01099598
:10340000DF91CF9108950E9464089C01892B31F4CB
:103410008CE090E09093E8158093E715C90108953A
:103420000E94EA080895CF92DF92EF92FF920F93E5
:103430001F93CF93DF936C017B018A01E901C131B6
:10344000D10544F040E150E0B801C701F60109950B
:103450006097F5CF1C161D062CF4AE01B801C7010C
:10346000F6010995DF91CF911F910F91FF90EF9099
:10347000DF90CF9008952F923F924F925F926F927C
:103480007F928F929F92AF92BF92CF92DF92EF92F4
:10349000FF920F931F93CF93DF93CDB7DEB76B9758
:1034A0000FB6F894DEBF0FBECDBF9B8B8A8B7D8B92
:1034B0006C8B2A0149011F8A1E8A6201F20107C032
:1034C000F5E23F1639F00894411C511CF20130809E
:1034D0003320B1F782010C191D0971F0A801B60162
:1034E0008C899D892A893B89F90109954E895F89D3
:1034F000400F511F5F8B4E8B332009F4EDC20894AF
:10350000411C511C2224298A198E188E80E090E0DB
:103510009B8F8A8F8FEF682E782EF20141912F01B9
:10352000342EF0E24F1721F489898823B1F703C0C4
:103530002BE2421711F4398AF0CF3DE2431719F418
:1035400044E0242AEACF53E2451719F481E0282AFF
:10355000E4CF90E3491719F4E0E12E2ADECFFCE630
:103560004F1719F428E0222AD8CF3AE74317A9F2D7
:103570005AE24517A1F4F40182E090E0880E991E0A
:103580000190F081E02DF98FE88FF7FFC6CF94E02E
:10359000292AF095E195FF4FF98FE88FBECFEEE233
:1035A0004E1791F5F20180818A3259F40894411C3A
:1035B000511CF40122E030E0820E931E6080718085
:1035C00020C06624772480538A3008F0A6CFC30138
:1035D00003E0880F991F0A95E1F7860D971D680E85
:1035E000791EF20181912F01992787FD9095680E30
:1035F000791E20ED3FEF620E731E808180538A306A
:1036000030F377FE8ACF86CF842F8153242F332740
:10361000893030F520533040398F288FF2012081D6
:10362000822F80538A3008F078CF888D998D13E0EF
:10363000880F991F1A95E1F7488D598D840F951FB2
:10364000480F591F822F992787FD9095480F591FC2
:1036500040535040598F488F0894411C511CDECF75
:103660002836310504F5253631050CF0A4C1203586
:10367000310509F444C0213531054CF425343105B8
:1036800009F499C12734310509F495C198C123364D
:10369000310549F1243631050CF076C02835310565
:1036A00009F427C18CC12037310509F422C1213723
:1036B00031054CF42936310509F466C02F36310541
:1036C00009F4D3C07CC12537310509F45CC0263725
:1036D000310524F42337310559F171C128373105FB
:1036E00009F407C16CC16E010894C11CD11CF4011E
:1036F00022E030E0820E931E8081898368C1F4014C
:1037000042E050E0840E951EC080D180C114D104E7
:1037100019F4B3E73B2E16C0C6010E94F37C019654
:103720000E94031A5C01B6010E94EC7C650107C08F
:10373000F40182E090E0880E991EC080D180C1140F
:10374000D10421F4AFE7CA2EA4E0DA2E77FC11C031
:10375000A30160E070E0C6010E94FC7C009739F094
:103760008C010C191D09601671060CF032C1830121
:1037700030C1F60101900020E9F78F01015010409F
:103780000C191D0926C1198A23FE0AC0F40124E080
:1037900030E0820E931EE080F1800281138115C01B
:1037A000C4010296453741F4F4014C0180819181B6
:1037B0007C010027112717C0F4014C018081918101
:1037C0007C010027F7FC0095102F453761F017FFAB
:1037D0000AC010950095F094E094E11CF11C011DC5
:1037E000111D8DE2898B7B8E6A8E77FC02C03FEEC5
:1037F0002322F1E1CF2ED12CCC0EDD1EE114F104F9
:103800000105110529F44A8D5B8D452B09F4CDC0C6
:103810005AE0E516F1040105110548F4E0E1CE2E69
:10382000D12CCC0EDD1E8E2D805D888BBEC0C801D4
:10383000B7012AE030E040E050E00E948C7DDC01DE
:10384000CB01805DF60182936F01C801B7012AE0C8
:1038500030E040E050E00E948C7D79018A01211522
:1038600031054105510519F7A0C023FE0AC0F40136
:1038700024E030E0820E931EE080F180028113810B
:103880000AC0F40142E050E0840E951E80819181CF
:103890007C0100271127198A7B8E6A8E77FC02C073
:1038A0005FEE252271E1C72ED12CCC0EDD1EE11476
:1038B000F1040105110529F48A8D9B8D892B09F4EA
:1038C00074C08E2D8770805DF60182936F0163E076
:1038D00016950795F794E7946A95D1F7E114F104EA
:1038E0000105110571F720FE60C0803309F45DC049
:1038F00058C0403779F4F40122E030E0820E931E84
:10390000808191817C010027112731E0232A58E72B
:10391000352E16C023FE0AC0F40144E050E0840EA8
:10392000951EE080F180028113810AC0F40182E0DB
:1039300090E0880E991E808191817C0100271127DB
:10394000198A7B8E6A8E77FC02C09FEE2922E8E5F9
:103950003E1629F446E8A42E44E0B42E04C037E90C
:10396000A32E34E0B32E21E1C22ED12CCC0EDD1ECD
:10397000F701EF70F070EA0DFB1D8081F601829374
:103980006F0194E016950795F794E7949A95D1F70F
:10399000E114F1040105110559F720FE06C0329229
:1039A0006F0180E3F60182936F018E010C191D09EE
:1039B0000F5E1F4F0FC024E030E0820E931E4423A1
:1039C00009F48AC06E010894C11CD11C498301E02E
:1039D00010E0198A78014A8D5B8D041715070CF4E5
:1039E0007A018989882319F00894E11CF11C622C62
:1039F000772484E1A82EB12CA620B720A114B1040D
:103A000069F4888D998D8E199F099C014FE654E0C9
:103A10006C897D898A899B890E94131A89898823E8
:103A200051F041E050E0BE016F5E7F4F8C899D896F
:103A3000EA89FB890995F0E1AF16B10469F4888D34
:103A4000998D8E199F099C014FE554E06C897D8901
:103A50008A899B890E94131A2A8D3B8D201B310B6A
:103A60003B8F2A8F4FE554E06C897D898A899B8939
:103A70000E94131A0115110539F0A801B6018C89AD
:103A80009D89EA89FB890995F0E53F1619F4C6017D
:103A90000E94101A62FE0DC0888D998D8E199F09A3
:103AA0009C014FE654E06C897D898A899B890E943C
:103AB000131A288D398D2E153F053CF04E895F89EC
:103AC000420F531F5F8B4E8BF8CC8E899F898E0DD2
:103AD0009F1D9F8B8E8BF1CC8E899F896B960FB625
:103AE000F894DEBF0FBECDBFDF91CF911F910F9134
:103AF000FF90EF90DF90CF90BF90AF909F908F900E
:103B00007F906F905F904F903F902F900895FC01B1
:103B100040E050E48081282F332727FD309522375D
:103B2000310579F02337310524F42136310539F098
:103B30001FC027373105E1F441E053E402C048E0FB
:103B400051E4319680818823E1F08081282F33274A
:103B500027FD30952B32310521F02236310529F031
:103B600007C04E7F42605360ECCF5F7B5068E9CF67
:103B700086E190E09093E8158093E7158FEF9FEF33
:103B80000895CA0108950F931F93CF93DF93CDB784
:103B9000DEB721970FB6F894DEBF0FBECDBF8C0104
:103BA000FB01898341E050E0BE01640F751F8081F5
:103BB00091810E94F019019711F00FEF1FEFC801DA
:103BC00021960FB6F894DEBF0FBECDBFDF91CF9127
:103BD0001F910F910895FC01CB01DF010D90002092
:103BE000E9F71197AE1BBF0BAD01BF01FC0180814E
:103BF00091810E94F01908952F923F924F925F9207
:103C00006F927F928F929F92AF92BF92CF92DF92EC
:103C1000EF92FF920F931F93CF93DF93CDB7DEB751
:103C20002E970FB6F894DEBF0FBECDBF6C017E8716
:103C30006D8729013A0147015801FCE62F2EF3E078
:103C40003F2E280E391E4196E1E0EE2EF12C03E0C6
:103C50009C01AB01BE016E0D7F1DC6010E94CF38D5
:103C60007C01F10180859185892B39F488E090E011
:103C70000E946408F10191878087F101A085B185D8
:103C80004D925D926D927C921397FD018482958294
:103C9000A682B78288E0F601848B858ABB27AB2D8C
:103CA0009A2D892D868BC501AA27BB27878B8B2D43
:103CB0009927AA27BB27808F418EBB27A72D962D3A
:103CC000852D828FC301AA27BB27838F872D992734
:103CD000AA27BB27848F0FEF1FEF2CE031E04D8523
:103CE0005E85B701C6010E941639DC01CB01BC011B
:103CF000CD012E960FB6F894DEBF0FBECDBFDF917B
:103D0000CF911F910F91FF90EF90DF90CF90BF90D8
:103D1000AF909F908F907F906F905F904F903F906B
:103D20002F900895AF92BF92CF92DF92EF92FF92C1
:103D30000F931F93CF93DF93CDB7DEB72C970FB6BA
:103D4000F894DEBF0FBECDBF6C015B01FC01EB5BE5
:103D5000FD4F1081112329F06BEF7EEF8FEF9FEF66
:103D60001BC081E08083C6014196A3E0EA2EF12CBE
:103D700003E09C01AB01BE016F5F7F4FC6010E9453
:103D8000CF38F601148B0FEF1FEF2CE033E0A501C5
:103D9000BC01C6010E9416392C960FB6F894DEBFFE
:103DA0000FBECDBFDF91CF911F910F91FF90EF908C
:103DB000DF90CF90BF90AF9008958F929F92AF9277
:103DC000BF92CF92DF92EF92FF920F931F93CF9308
:103DD000DF93CDB7DEB72C970FB6F894DEBF0FBEDA
:103DE000CDBF6C014B015A014196B5E0EB2EF12C91
:103DF00003E09C01AB01BE016F5F7F4FC6010E94D3
:103E0000CF387C01F501808199270196AC01B5017D
:103E1000C60144960E94097D0FEF1FEF2CE035E0AC
:103E2000A401B701C6010E941639DC01CB01BC0117
:103E3000CD012C960FB6F894DEBF0FBECDBFDF913B
:103E4000CF911F910F91FF90EF90DF90CF90BF9097
:103E5000AF909F908F9008952F923F924F925F92D4
:103E60006F927F928F929F92AF92BF92DF92EF926A
:103E7000FF920F931F93CF93DF93CDB7DEB78C885C
:103E80009D886E887F88D88C840104591C4F89E1F5
:103E9000E82EF12CEC0EFD1E5701F801868197816A
:103EA000892B39F48CE090E00E946408F801978334
:103EB0008683F801A681B781FD01D182BD016E5FC5
:103EC0007F4FF801A681B78181E08C938D2D8150C1
:103ED000823008F05BC082E090E0E80EF91EF70146
:103EE000D5018C91DB018D93BD019927813091051E
:103EF00071F0823091051CF4892B21F042C00297A9
:103F000071F13FC0F801A681B78182E038C02081FD
:103F10003181428153812D93BD01232E342E452EB4
:103F20005524DB012D92BD019A0144275527DB0161
:103F30002D9388E090E0E80EF91E248135814681BA
:103F400057812D93BD01BB27A52F942F832FFB01F4
:103F50008193CA01AA27BB278193BF010CC082E0CD
:103F600090E0E80EF91E0190F081E02D86E00190CE
:103F70000D928150E1F7F801A681B78188E08C931A
:103F800005C06EEE7FEF8FEF9FEF14C0F2E0DF16FB
:103F900051F4D7018C91FB018083F801A681B78190
:103FA0008C918F5F8C93F80146815781B301C401D6
:103FB0000E94DD1EDF91CF911F910F91FF90EF9036
:103FC000DF90BF90AF909F908F907F906F905F90A9
:103FD0004F903F902F900895AF92BF92CF92DF9273
:103FE000EF92FF920F931F93CF93DF93CDB7DEB77E
:103FF0002C970FB6F894DEBF0FBECDBF6C015B01EE
:10400000419629E0E22EF12C03E09C01AB01BE01B8
:104010006F5F7F4FC6010E94CF38F601148A0FEF01
:104020001FEF2CE039E0A501BC01C6010E94163942
:10403000DC01CB01BC01CD012C960FB6F894DEBF9C
:104040000FBECDBFDF91CF911F910F91FF90EF90E9
:10405000DF90CF90BF90AF9008958F929F92AF92D4
:10406000BF92CF92DF92EF92FF920F931F93CF9365
:10407000DF93CDB7DEB72C970FB6F894DEBF0FBE37
:10408000CDBF6C014B01142F4CE6A42E43E0B42E9F
:10409000A80EB91E41963AE0E32EF12C03E09C01F4
:1040A000AB01BE016F5F7F4FC6010E94CF387C011C
:1040B000F501808D918D892B39F481E090E00E948B
:1040C0006408F501918F808FF501A08DB18D1C934F
:1040D00081E0F601848B158B0FEF1FEF2CE03AE0A7
:1040E000A401B701C6010E941639DC01CB01BC0155
:1040F000CD012C960FB6F894DEBF0FBECDBFDF9179
:10410000CF911F910F91FF90EF90DF90CF90BF90D4
:10411000AF909F908F9008956F927F928F929F9211
:10412000AF92BF92CF92DF92EF92FF920F931F93C5
:10413000CF93DF93CDB7DEB72C970FB6F894DEBFE1
:104140000FBECDBF6C013B014A016CE6A62E63E0B9
:10415000B62EA80EB91E419653E1E52EF12C03E0D0
:104160009C01A301BE016F5F7F4FC6010E94CF3843
:104170007C01F50184899589892B59F489EF90E0B8
:104180000E946408DC01F501958B848BA850BF4F19
:104190001C92F50184899589F40101900020E9F7CA
:1041A0003197E819F909E83FF10520F4AF014F5FB5
:1041B0005F4F02C049EF50E0B4010E94097D88EFD3
:1041C000F601848B90E0D6015596F40180818D93A1
:1041D0008081882321F09F5F3196983FB8F3983F04
:1041E00009F49150F601E90FF11D158A0FEF1FEF49
:1041F0002CE033E1A301B701C6010E941639DC01AE
:10420000CB01BC01CD012C960FB6F894DEBF0FBEDA
:10421000CDBFDF91CF911F910F91FF90EF90DF9075
:10422000CF90BF90AF909F908F907F906F900895A8
:104230008F929F92AF92BF92CF92DF92EF92FF92B6
:104240000F931F93CF93DF93CDB7DEB72C970FB6A5
:10425000F894DEBF0FBECDBF6C014B015A01122F87
:10426000419674E1E72EF12C03E09C01A401BE010C
:104270006F5F7F4FC6010E94CF38BC01FC01B18641
:10428000A086812F9927AA27BB2784839583A6839D
:10429000B783F601148A0FEF1FEF2CE034E1A4017D
:1042A000C6010E941639DC01CB01BC01CD012C9660
:1042B0000FB6F894DEBF0FBECDBFDF91CF911F9137
:1042C0000F91FF90EF90DF90CF90BF90AF909F90B5
:1042D0008F900895AF92BF92CF92DF92EF92FF92AC
:1042E0000F931F93CF93DF93CDB7DEB72C970FB605
:1042F000F894DEBF0FBECDBF6C015B014196E5E1D6
:10430000EE2EF12C03E09C01AB01BE016F5F7F4FED
:10431000C6010E94CF38F601148A0FEF1FEF2CE080
:1043200035E1A501BC01C6010E941639DC01CB01B3
:10433000BC01CD012C960FB6F894DEBF0FBECDBFE9
:10434000DF91CF911F910F91FF90EF90DF90CF9071
:10435000BF90AF9008956F927F928F929F92AF928D
:10436000BF92CF92DF92EF92FF920F931F93CF9362
:10437000DF93CDB7DEB72C970FB6F894DEBF0FBE34
:10438000CDBF6C013B014A011CE6A12E13E0B12E0A
:10439000A80EB91E4196B6E1EB2EF12C03E09C016C
:1043A000AB01BE016F5F7F4FC6010E94CF387C0119
:1043B000F50182819381892B39F482E090E00E949B
:1043C0006408F50193838283F501A281B3818D9204
:1043D0009C9282E0F601848B858A892D9927868BB1
:1043E0000FEF1FEF2CE036E1A301B701C6010E94D9
:1043F0001639DC01CB01BC01CD012C960FB6F89427
:10440000DEBF0FBECDBFDF91CF911F910F91FF9007
:10441000EF90DF90CF90BF90AF909F908F907F9064
:104420006F900895AF92BF92CF92DF92EF92FF927A
:104430000F931F93CF93DF93CDB7DEB72C970FB6B3
:10444000F894DEBF0FBECDBF6C015B01419607E162
:10445000E02EF12C03E09C01AB01BE016F5F7F4FAA
:10446000C6010E94CF38F601148A0FEF1FEF2CE02F
:1044700037E1A501BC01C6010E941639DC01CB0160
:10448000BC01CD012C960FB6F894DEBF0FBECDBF98
:10449000DF91CF911F910F91FF90EF90DF90CF9020
:1044A000BF90AF9008956F927F928F929F92AF923C
:1044B000BF92CF92DF92EF92FF920F931F93CF9311
:1044C000DF93CDB7DEB72C970FB6F894DEBF0FBEE3
:1044D000CDBF6C013B014A013CE6A32E33E0B32E75
:1044E000A80EB91E419628E1E22EF12C03E09C01B2
:1044F000AB01BE016F5F7F4FC6010E94CF387C01C8
:10450000F50186899789892B39F482E090E00E9431
:104510006408F501978B868BF501A689B7898D9282
:104520009C9282E0F601848B858A892D9927868B5F
:104530000FEF1FEF2CE038E1A301B701C6010E9485
:104540001639DC01CB01BC01CD012C960FB6F894D5
:10455000DEBF0FBECDBFDF91CF911F910F91FF90B6
:10456000EF90DF90CF90BF90AF909F908F907F9013
:104570006F900895AF92BF92CF92DF92EF92FF9229
:104580000F931F93CF93DF93CDB7DEB72C970FB662
:10459000F894DEBF0FBECDBF6C015B01419649E1CF
:1045A000E42EF12C03E09C01AB01BE016F5F7F4F55
:1045B000C6010E94CF38F601148A0FEF1FEF2CE0DE
:1045C00039E1A501BC01C6010E941639DC01CB010D
:1045D000BC01CD012C960FB6F894DEBF0FBECDBF47
:1045E000DF91CF911F910F91FF90EF90DF90CF90CF
:1045F000BF90AF9008958F929F92AF92BF92CF924B
:10460000DF92EF92FF920F931F93CF93DF93CDB77B
:10461000DEB72C970FB6F894DEBF0FBECDBF6C018E
:104620004B01142F6CE6A62E63E0B62EA80EB91E21
:1046300041965AE1E52EF12C03E09C01A401BE0154
:104640006F5F7F4FC6010E94CF387C01F501828DDC
:10465000938D892B39F481E090E00E946408F50184
:10466000938F828FF501A28DB38D1C9381E0F601AB
:10467000848B158B0FEF1FEF2CE03AE1A401B701FB
:10468000C6010E941639DC01CB01BC01CD012C967C
:104690000FB6F894DEBF0FBECDBFDF91CF911F9153
:1046A0000F91FF90EF90DF90CF90BF90AF909F90D1
:1046B0008F900895AF92BF92CF92DF92EF92FF92C8
:1046C0000F931F93CF93DF93CDB7DEB72C970FB621
:1046D000F894DEBF0FBECDBF6C015B01419673E263
:1046E000E72EF12C03E09C01A501BE016F5F7F4F17
:1046F000C6010E94CF38F601148A0FEF1FEF2CE09D
:1047000033E2A501BC01C6010E941639DC01CB01D0
:10471000BC01CD012C960FB6F894DEBF0FBECDBF05
:10472000DF91CF911F910F91FF90EF90DF90CF908D
:10473000BF90AF9008954F925F926F927F928F9249
:104740009F92AF92BF92CF92DF92EF92FF920F9320
:104750001F93CF93DF93CDB7DEB72C970FB6F894A6
:10476000DEBF0FBECDBF6C012B0149015A010CE623
:10477000602E03E0702E680E791E419614E2E12E41
:10478000F12C03E09C01AB01BE016F5F7F4FC601BE
:104790000E94CF387C01F30182899389892B39F4F7
:1047A00084E090E00E946408F301938B828BF30114
:1047B000A289B3898D929D92AD92BC92139783E0AA
:1047C000F601848B858ABB27AB2D9A2D892D868B8C
:1047D000C501AA27BB27878B0FEF1FEF2CE034E220
:1047E000A201B701C6010E941639DC01CB01BC0150
:1047F000CD012C960FB6F894DEBF0FBECDBFDF9172
:10480000CF911F910F91FF90EF90DF90CF90BF90CD
:10481000AF909F908F907F906F905F904F90089592
:104820008F929F92AF92BF92CF92DF92EF92FF92C0
:104830000F931F93CF93DF93CDB7DEB72C970FB6AF
:10484000F894DEBF0FBECDBF6C014B01142F3CE6C8
:10485000A32E33E0B32EA80EB91E419621E3E22E1B
:10486000F12C03E09C01AB01BE016F5F7F4FC601DD
:104870000E94CF387C01F50182859385892B39F41C
:1048800081E090E00E946408F50193878287F5013A
:10489000A285B3851C9381E0F601848B158B0FEF05
:1048A0001FEF2CE031E3A401B701C6010E941639C5
:1048B000DC01CB01BC01CD012C960FB6F894DEBF14
:1048C0000FBECDBFDF91CF911F910F91FF90EF9061
:1048D000DF90CF90BF90AF909F908F9008952F92D0
:1048E0003F924F925F926F927F928F929F92AF9280
:1048F000BF92CF92DF92EF92FF920F931F93CF93CD
:10490000DF93CDB7DEB72D970FB6F894DEBF0FBE9D
:10491000CDBF6C011B014A012D8738012701ECE650
:10492000AE2EE3E0BE2EA80EB91E419673E3E72E2D
:10493000F12C03E09C01A101BE016F5F7F4FC60116
:104940000E94CF387C01F50184859585892B39F447
:1049500087E090E00E946408F50195878487F5015F
:10496000A485B58511969C928E928D85FD018283DA
:10497000F501A485B585FD01748263825682458266
:1049800087E0F601848B858A892D9927868B8D8512
:10499000878B608E872D9927818F428E852D992751
:1049A000838F0FEF1FEF2CE033E3A101B701C601A6
:1049B0000E941639DC01CB01BC01CD012D960FB64A
:1049C000F894DEBF0FBECDBFDF91CF911F910F9145
:1049D000FF90EF90DF90CF90BF90AF909F908F901F
:1049E0007F906F905F904F903F902F9008956F92BF
:1049F0007F928F929F92AF92BF92CF92DF92EF926F
:104A0000FF920F931F93CF93DF93CDB7DEB72C9711
:104A10000FB6F894DEBF0FBECDBF6C013B014A015B
:104A20000E94B9385C018FEFA8168FEFB80629F401
:104A30006DEF7EEF8FEF9FEF25C0C601419615E326
:104A4000E12EF12C03E09C0140E050E0BE016F5FDD
:104A50007F4FC6010E94CF3885E0F601848B81E04C
:104A6000858BA68A8B2D9927878B808E892D9927F8
:104A7000818F83012CE035E340E050E0BA01C601AC
:104A80000E9416392C960FB6F894DEBF0FBECDBF2C
:104A9000DF91CF911F910F91FF90EF90DF90CF901A
:104AA000BF90AF909F908F907F906F9008956F927E
:104AB0007F928F929F92AF92BF92CF92DF92EF92AE
:104AC000FF920F931F93CF93DF93CDB7DEB72C9751
:104AD0000FB6F894DEBF0FBECDBF6C013B014A019B
:104AE000BA010E94B9385C018FEFA8168FEFB806A3
:104AF00029F46DEF7EEF8FEF9FEF1DC0C601419649
:104B000026E3E22EF12C03E09C01A301BE016F5FBE
:104B10007F4FC6010E94CF38BC0182E0F601848B32
:104B2000A58A8B2D9927868B84012CE036E3A3017F
:104B3000C6010E9416392C960FB6F894DEBF0FBE40
:104B4000CDBFDF91CF911F910F91FF90EF90DF903C
:104B5000CF90BF90AF909F908F907F906F9008956F
:104B60004F925F926F927F928F929F92AF92BF927D
:104B7000CF92DF92EF92FF920F931F93CF93DF9329
:104B8000CDB7DEB72C970FB6F894DEBF0FBECDBF02
:104B90006C012B013A014901BA010E94B9385C014C
:104BA0008FEFA8168FEFB80629F46DEF7EEF8FEF29
:104BB0009FEF21C0C601419657E3E52EF12C03E09B
:104BC0009C01A201BE016F5F7F4FC6010E94CF38DA
:104BD000BC0184E0F601848BA58A8B2D9927868BF6
:104BE000878A892D9927808F83012CE037E3A201E2
:104BF000C6010E9416392C960FB6F894DEBF0FBE80
:104C0000CDBFDF91CF911F910F91FF90EF90DF907B
:104C1000CF90BF90AF909F908F907F906F905F905C
:104C20004F900895AF92BF92CF92DF92EF92FF9292
:104C30000F931F93CF93DF93CDB7DEB72C970FB6AB
:104C4000F894DEBF0FBECDBF6C015B01419664E4FA
:104C5000E62EF12C03E09C01A501BE016F5F7F4FA2
:104C6000C6010E94CF38F601148A0FEF1FEF2CE027
:104C700034E4A501BC01C6010E941639DC01CB0158
:104C8000BC01CD012C960FB6F894DEBF0FBECDBF90
:104C9000DF91CF911F910F91FF90EF90DF90CF9018
:104CA000BF90AF9008958F929F92AF92BF92CF9294
:104CB000DF92EF92FF920F931F93CF93DF93CDB7C5
:104CC000DEB72C970FB6F894DEBF0FBECDBF6C01D8
:104CD0004B01142FECE6AE2EE3E0BE2EA80EB91E5B
:104CE000419675E4E72EF12C03E09C01A401BE017E
:104CF0006F5F7F4FC6010E94CF387C01F50186852A
:104D00009785892B39F481E090E00E946408F501D1
:104D100097878687F501A685B7851C9381E0F60104
:104D2000848B158B0FEF1FEF2CE035E4A401B70146
:104D3000C6010E941639DC01CB01BC01CD012C96C5
:104D40000FB6F894DEBF0FBECDBFDF91CF911F919C
:104D50000F91FF90EF90DF90CF90BF90AF909F901A
:104D60008F900895AF92BF92CF92DF92EF92FF9211
:104D70000F931F93CF93DF93CDB7DEB72C970FB66A
:104D8000F894DEBF0FBECDBF6C015B014196F2E42B
:104D9000EF2EF12C03E09C01AB01BE016F5F7F4F52
:104DA000C6010E94CF38F601148A0FEF1FEF2CE0E6
:104DB00032E4A501BC01C6010E941639DC01CB0119
:104DC000BC01CD012C960FB6F894DEBF0FBECDBF4F
:104DD000DF91CF911F910F91FF90EF90DF90CF90D7
:104DE000BF90AF9008958F929F92AF92BF92CF9253
:104DF000DF92EF92FF920F931F93CF93DF93CDB784
:104E0000DEB72C970FB6F894DEBF0FBECDBF6C0196
:104E10004B01142FBCE6AB2EB3E0BB2EA80EB91E7F
:104E20004196A3E4EA2EF12C03E09C01AB01BE0104
:104E30006F5F7F4FC6010E94CF387C01F5018089EA
:104E40009189892B39F481E090E00E946408F50192
:104E5000918B808BF501A089B1891C9381E0F601CB
:104E6000848B158B0FEF1FEF2CE033E4A401B70107
:104E7000C6010E941639DC01CB01BC01CD012C9684
:104E80000FB6F894DEBF0FBECDBFDF91CF911F915B
:104E90000F91FF90EF90DF90CF90BF90AF909F90D9
:104EA0008F9008958F929F92AF92BF92CF92DF9290
:104EB000EF92FF920F931F93CF93DF93CDB7DEB79F
:104EC0002C970FB6F894DEBF0FBECDBF6C014B011F
:104ED0005A01419621E0E22EF12C04E09C01AB0145
:104EE000BE016E0D7F1DC6010E94CF38FC01B18648
:104EF000A0861482158216821782F601148A0FEF9B
:104F00001FEF20E131E0A401BC01C6010E94163967
:104F1000DC01CB01BC01CD012C960FB6F894DEBFAD
:104F20000FBECDBFDF91CF911F910F91FF90EF90FA
:104F3000DF90CF90BF90AF909F908F900895AF92E9
:104F4000BF92CF92DF92EF92FF920F931F93CF9376
:104F5000DF93CDB7DEB72C970FB6F894DEBF0FBE48
:104F6000CDBF6C015B01419632E0E32EF12C04E0F1
:104F70009C01AB01BE016F5F7F4FC6010E94CF381D
:104F8000F601148A0FEF1FEF20E132E0A501BC010A
:104F9000C6010E941639DC01CB01BC01CD012C9663
:104FA0000FB6F894DEBF0FBECDBFDF91CF911F913A
:104FB0000F91FF90EF90DF90CF90BF90AF9008954A
:104FC0008F929F92AF92BF92CF92DF92EF92FF9219
:104FD0000F931F93CF93DF93CDB7DEB72C970FB608
:104FE000F894DEBF0FBECDBF6C015B014A01419654
:104FF00043E0E42EF12C04E09C01AB01BE016F5FA5
:105000007F4FC6010E94CF38FC0191868086F60151
:10501000148A0FEF1FEF20E133E0A501BC01C601A8
:105020000E941639DC01CB01BC01CD012C960FB6D4
:10503000F894DEBF0FBECDBFDF91CF911F910F91CE
:10504000FF90EF90DF90CF90BF90AF909F908F90A8
:105050000895AF92BF92CF92DF92EF92FF920F939B
:105060001F93CF93DF93CDB7DEB72C970FB6F8948D
:10507000DEBF0FBECDBF6C015B01419654E0E52E53
:10508000F12C04E09C01AB01BE016F5F7F4FC601B4
:105090000E94CF38F601148A0FEF1FEF20E134E0B1
:1050A000A501BC01C6010E941639DC01CB01BC017F
:1050B000CD012C960FB6F894DEBF0FBECDBFDF91A9
:1050C000CF911F910F91FF90EF90DF90CF90BF9005
:1050D000AF900895AF92BF92CF92DF92EF92FF927E
:1050E0000F931F93CF93DF93CDB7DEB72C970FB6F7
:1050F000F894DEBF0FBECDBF6C015B01419665E049
:10510000E62EF12C04E09C01A501BE016F5F7F4FEC
:10511000C6010E94CF38F601148A0FEF1FEF20E17D
:1051200035E0A501BC01C6010E941639DC01CB01A6
:10513000BC01CD012C960FB6F894DEBF0FBECDBFDB
:10514000DF91CF911F910F91FF90EF90DF90CF9063
:10515000BF90AF9008958F929F92AF92BF92CF92DF
:10516000DF92EF92FF920F931F93CF93DF93CDB710
:10517000DEB72C970FB6F894DEBF0FBECDBF6C0123
:105180005B014A01419679E0E72EF12C04E09C0195
:10519000A501BE016F5F7F4FC6010E94CF38FC01A1
:1051A00091868086F601148A0FEF1FEF20E139E027
:1051B000A501BC01C6010E941639DC01CB01BC016E
:1051C000CD012C960FB6F894DEBF0FBECDBFDF9198
:1051D000CF911F910F91FF90EF90DF90CF90BF90F4
:1051E000AF909F908F9008956F927F928F929F9231
:1051F000AF92BF92CF92DF92EF92FF920F931F93E5
:10520000CF93DF93CDB7DEB72C970FB6F894DEBF00
:105210000FBECDBF6C013B014A01BA010E94B938F3
:105220005C018FEFA8168FEFB80629F46DEF7EEFC3
:105230008FEF9FEF1CC0C601419629E0E22EF12CB2
:1052400002E09C01A301BE016F5F7F4FC6010E9477
:10525000CF38BC01F601048BA58A8B2D9927868B4C
:10526000840128E039E0A301C6010E9416392C967A
:105270000FB6F894DEBF0FBECDBFDF91CF911F9167
:105280000F91FF90EF90DF90CF90BF90AF909F90E5
:105290008F907F906F9008958F929F92AF92BF9260
:1052A000CF92DF92EF92FF920F931F93CF93DF93F2
:1052B000CDB7DEB72C970FB6F894DEBF0FBECDBFCB
:1052C0006C014B015A01122FBA010E94B9388F5F4D
:1052D0009F4F29F46DEF7EEF8FEF9FEF23C0C60144
:1052E00041963BE0E32EF12C02E09C01A401BE01BB
:1052F0006F5F7F4FC6010E94CF387C0187E0F601C7
:10530000848BC6014596AC01B501C6010E94CE2D25
:10531000F601138F850128E03BE0A401B701C60127
:105320000E9416392C960FB6F894DEBF0FBECDBF83
:10533000DF91CF911F910F91FF90EF90DF90CF9071
:10534000BF90AF909F908F9008956F927F928F92B1
:105350009F92AF92BF92CF92DF92EF92FF920F9304
:105360001F93CF93DF93CDB7DEB72C970FB6F8948A
:10537000DEBF0FBECDBF6C013B014A01BA010E94E6
:10538000B9385C018FEFA8168FEFB80629F46DEFDE
:105390007EEF8FEF9FEF1CC0C60141965CE0E52ECB
:1053A000F12C02E09C01A301BE016F5F7F4FC6019B
:1053B0000E94CF38BC01F601048BA58A8B2D99275A
:1053C000868B840128E03CE0A301C6010E941639C7
:1053D0002C960FB6F894DEBF0FBECDBFDF91CF91F4
:1053E0001F910F91FF90EF90DF90CF90BF90AF9003
:1053F0009F908F907F906F9008954F925F926F92E1
:105400007F928F929F92AF92BF92CF92DF92EF9254
:10541000FF920F931F93CF93DF93CDB7DEB72C97F7
:105420000FB6F894DEBF0FBECDBF6C012B013A0161
:105430004901BA010E94B9385C018FEFA8168FEFBD
:10544000B80629F46DEF7EEF8FEF9FEF21C0C60104
:1054500041961DE0E12EF12C02E09C01A201BE016B
:105460006F5F7F4FC6010E94CF38BC0184E0F60118
:10547000848BA58A8B2D9927868B878A892D9927DE
:10548000808F830128E03DE0A201C6010E94163909
:105490002C960FB6F894DEBF0FBECDBFDF91CF9133
:1054A0001F910F91FF90EF90DF90CF90BF90AF9042
:1054B0009F908F907F906F905F904F900895AF92E4
:1054C000BF92CF92DF92EF92FF920F931F93CF93F1
:1054D000DF93CDB7DEB72C970FB6F894DEBF0FBEC3
:1054E000CDBF6C015B0141960EE0E02EF12C02E095
:1054F0009C01AB01BE016F5F7F4FC6010E94CF3898
:10550000F601148A0FEF1FEF28E03EE0A501BC0171
:10551000C6010E941639DC01CB01BC01CD012C96DD
:105520000FB6F894DEBF0FBECDBFDF91CF911F91B4
:105530000F91FF90EF90DF90CF90BF90AF900895C4
:105540006F927F928F929F92AF92BF92CF92DF9293
:10555000EF92FF920F931F93CF93DF93CDB7DEB7F8
:105560002C970FB6F894DEBF0FBECDBF6C013B0188
:105570004A013CE6A32E33E0B32EA80EB91E419695
:105580002FE0E22EF12C02E09C01AB01BE016F5F27
:105590007F4FC6010E94CF387C01F501848195813F
:1055A000892B39F482E090E00E946408F50195832C
:1055B0008483F501A481B5818D929C9282E0F601ED
:1055C000848B858A892D9927868B0FEF1FEF28E022
:1055D0003FE0A301B701C6010E941639DC01CB01EF
:1055E000BC01CD012C960FB6F894DEBF0FBECDBF27
:1055F000DF91CF911F910F91FF90EF90DF90CF90AF
:10560000BF90AF909F908F907F906F9008952F9252
:105610003F924F925F926F927F928F929F92AF9242
:10562000BF92CF92DF92EF92FF920F931F93CF938F
:10563000DF93CDB7DEB72C970FB6F894DEBF0FBE61
:10564000CDBF6C011B012A0149013801BA010E943A
:10565000B9385C018FEFA8168FEFB80629F46DEF0B
:105660007EEF8FEF9FEF25C0C6014196B1E0EB2E94
:10567000F12C02E09C01A101BE016E0D7F1DC6014F
:105680000E94CF38BC0186E0F601848BA58A8B2D61
:105690009927868B878A892D9927808F618E872D00
:1056A0009927828F820128E031E0A101C6010E9482
:1056B00016392C960FB6F894DEBF0FBECDBFDF9122
:1056C000CF911F910F91FF90EF90DF90CF90BF90FF
:1056D000AF909F908F907F906F905F904F903F9092
:1056E0002F9008952F923F924F925F926F927F92E8
:1056F0008F929F92AF92BF92CF92DF92EF92FF92E2
:105700000F931F93CF93DF93CDB7DEB760970FB69C
:10571000F894DEBF0FBECDBF5C017E876D87588BCE
:105720004F874901380127011601BA010E94B93893
:105730006C018FEFC8168FEFD80629F46DEF7EEF5E
:105740008FEF9FEF30C0C501419633E0E32EF12C7F
:1057500002E09C014D855E85BE016F5F7F4FC501F4
:105760000E94CF38BC018AE0F501848BC58A8D2D5B
:105770009927868B878A892D9927808F618E872D1F
:105780009927828F438E852D9927848F258E832D8F
:105790009927868F0F85188928E033E04D855E852F
:1057A000C5010E94163960960FB6F894DEBF0FBE91
:1057B000CDBFDF91CF911F910F91FF90EF90DF90C0
:1057C000CF90BF90AF909F908F907F906F905F90A1
:1057D0004F903F902F9008956F927F928F929F925B
:1057E000AF92BF92CF92DF92EF92FF920F931F93EF
:1057F000CF93DF93CDB7DEB72C970FB6F894DEBF0B
:105800000FBECDBF6C013B014A01BA010E94B938FD
:105810005C018FEFA8168FEFB80629F46DEF7EEFCD
:105820008FEF9FEF1CC0C601419654E0E52EF12C8E
:1058300002E09C01A301BE016F5F7F4FC6010E9481
:10584000CF38BC01F601048BA58A8B2D9927868B56
:10585000840128E034E0A301C6010E9416392C9689
:105860000FB6F894DEBF0FBECDBFDF91CF911F9171
:105870000F91FF90EF90DF90CF90BF90AF909F90EF
:105880008F907F906F9008952F923F924F925F92EA
:105890006F927F928F929F92AF92BF92CF92DF9240
:1058A000EF92FF920F931F93CF93DF93CDB7DEB7A5
:1058B0002C970FB6F894DEBF0FBECDBF6C011B0155
:1058C0002A0149013801BA010E94B9385C018FEF01
:1058D000A8168FEFB80629F46DEF7EEF8FEF9FEFDC
:1058E00025C0C601419605E0E02EF12C02E09C01A6
:1058F000A101BE016F5F7F4FC6010E94CF38BC017E
:1059000086E0F601848BA58A8B2D9927868B878A62
:10591000892D9927808F618E872D9927828F82010B
:1059200028E035E0A101C6010E9416392C960FB679
:10593000F894DEBF0FBECDBFDF91CF911F910F91C5
:10594000FF90EF90DF90CF90BF90AF909F908F909F
:105950007F906F905F904F903F902F9008956F923F
:105960007F928F929F92AF92BF92CF92DF92EF92EF
:10597000FF920F931F93CF93DF93CDB7DEB72C9792
:105980000FB6F894DEBF0FBECDBF6C013B014A01DC
:10599000BA010E94B9385C018FEFA8168FEFB806E4
:1059A00029F46DEF7EEF8FEF9FEF1CC0C60141968B
:1059B00026E0E22EF12C02E09C01A301BE016F5F04
:1059C0007F4FC6010E94CF38BC01F601048BA58A27
:1059D0008B2D9927868B840128E036E0A301C60130
:1059E0000E9416392C960FB6F894DEBF0FBECDBFBD
:1059F000DF91CF911F910F91FF90EF90DF90CF90AB
:105A0000BF90AF909F908F907F906F90089520E00F
:105A1000FC01E758FD4F8189853071F480819181C7
:105A20008617970749F4808982958F708370682F55
:105A300077278827992708952F5F77962A3058F37C
:105A40006DEF7EEF8FEF9FEF089520E0FC01E758A8
:105A5000FD4F81898530B1F4808191818617970748
:105A600089F483899489AA27BB272227382F492FB5
:105A70005A2F82899927AA27BB27282B392B4A2BF3
:105A80005B2B08C02F5F77962A3018F32DEF3EEF7F
:105A90004FEF5FEFCA01B901089520E0FC01E7581C
:105AA000FD4F8189853051F4808191818617970758
:105AB00029F4648575858685978508952F5F779687
:105AC0002A3078F36DEF7EEF8FEF9FEF089520E09F
:105AD000DC01A758BD4F39E0FD018189853079F49B
:105AE0006115710559F0E22FFF27EE0FFF1FE60F3A
:105AF000F71F8D919C911197918380832F5F315077
:105B0000579637FFE9CF822F9927AA27BB27BC01D9
:105B1000CD010895CF93DF93DB0120E0FC01E7582E
:105B2000FD4F8189853009F594818C919817E9F4AE
:105B30009581ED0189819817C1F496818A81981722
:105B4000A1F497818B81981781F490858C819817A7
:105B500061F491858D81981741F4808191819C0138
:105B600044275527CA01B90108C02F5F77962A300C
:105B7000C0F26DEF7EEF8FEF9FEFDF91CF91089531
:105B8000DB01FC01EA59FC4F86E001900D92815047
:105B9000E1F760E070E080E090E00895A0E09C0113
:105BA00023583D4FFC01E758FD4F8189853089F42A
:105BB000808191818617970761F4DA01F90186E007
:105BC00001900D928150E1F760E070E080E090E09C
:105BD0000895AF5F7796295E3F4FAA3030F36DEF9F
:105BE0007EEF8FEF9FEF089520E0FC01E758FD4F17
:105BF0008189853051F4808191818617970729F436
:105C000060E070E080E090E008952F5F77962A30A2
:105C100078F36DEF7EEF8FEF9FEF08950F931F9353
:105C20008B019A0141E050E0B9010E94F724C801BC
:105C30001F910F910895CB01089508950895CF9372
:105C4000DF93CDB7DEB72E970FB6F894DEBF0FBE49
:105C5000CDBF2C01AE01495F5F4FBE01655F7F4F35
:105C6000C2010E9428361C01009709F47EC0DC01A5
:105C70008C9199278330910509F452C084309105A5
:105C80001CF4029749F071C0049709F06EC0B1018D
:105C9000C2010E94AA3D69C0F1014281842F992767
:105CA0008F709070382F222781819927282B392BCC
:105CB00042954F70E3E07E2E7422142F16951695B0
:105CC000B901C2010E949338AC01F1018183292FEF
:105CD00033278281807F822B828363E1862E62E07C
:105CE000962E840C951CD201A75DBD4F27E232E0B1
:105CF000420E531EF2010190F081E02D29ED3DEF9F
:105D0000420E531EAF80B884C984DA84EB84FC84CD
:105D1000012F272DB1018D919C910995D40123C0AC
:105D2000F101828199278F709070982F88272181A7
:105D30003327822B932BBC01C2010E949338AC0104
:105D40008201095C1D4F23E432E0420E531ED20152
:105D5000ED91FC912DEB3DEF420E531E2B85B101D1
:105D6000C2010995D8018D939C9341E7C42E42E06E
:105D7000D42EC40CD51CF6018081882391F13DE717
:105D8000E32E32E0F32EE40CF51C820107571D4F81
:105D900029E0722EF2018785908918161906C4F43D
:105DA00083859485181619069CF4F8018181823048
:105DB00079F484E08183808182958F708370482F8D
:105DC000B701C2010E94AB46D6018C9181508C93E1
:105DD0007A94095E1F4FE7E1F0E0EE0EFF1E77FEBA
:105DE000D9CF92E7292E92E0392E240C351CD1010F
:105DF0008C91882309F467C077248DE7A82E82E070
:105E0000B82EA40CB51C620188249924F201878560
:105E10009089181619060CF048C0838594851816C9
:105E200019060CF042C02FE832E0C20ED31ED60194
:105E30008C91E1E7FDEFCE0EDF1E8823B1F584E003
:105E400090E09C878B87DE011196F50186E001903A
:105E50000D928150E1F787E190E0889E7001899E64
:105E6000F00C989EF00C1124E40CF51CF701E75897
:105E7000FD4F08EA14E02B85AE014F5F5F4F608154
:105E80007181C2010E94B047DC01CB010097A105DE
:105E9000B10559F42FE832E0E20EF31E83E0D7019A
:105EA0008C93F10180818150808373940894811CCC
:105EB000911C27E130E0C20ED31EA20EB31E39E0C2
:105EC000371508F0A3CF0E94B407C4CECF92DF925B
:105ED000EF92FF920F931F93CF93DF93EC010CE6A9
:105EE000C02E03E0D02EC80ED91E60E070E00E94E4
:105EF000921EF601A085B185109761F0FD01E48046
:105F0000F580068117812D913D914D915C9160E066
:105F100070E00DC01FEFE12E1FEFF12E1FEB012FE0
:105F20001FEF112F2FEF3FE140E050E0BD01CE0108
:105F30000E94FC1DF601068117810115110539F03B
:105F4000A80160E070E0CE010E94DD1E26C01F9314
:105F50000F9381E08F931F930F93DF93CF930E9452
:105F60002C1F82E090E09F938F931F930F9382E00A
:105F70008F931F930F93DF93CF930E942C1FCE59C3
:105F8000DC4F19830883C256D3408DB79EB7409625
:105F90000FB6F8949EBF0FBE8DBFF601A281B381EC
:105FA000109729F04D915C9160E070E003C040E4EF
:105FB0005FE1BD01CE010E94AB21F601A689B78940
:105FC000109729F04D915C9160E070E003C040E0D3
:105FD00050E2BD01CE010E945322F601A28DB38D85
:105FE000109721F04C9160E070E002C043E0BD01E9
:105FF000CE010E94FB22F601A285B385109721F005
:106000004C9160E070E002C040E0BD01CE010E9412
:106010001024F601A685B785109721F04C9160E019
:1060200070E002C041E0BD01CE010E945326F6019E
:10603000A089B189109721F04C9160E070E002C016
:1060400041E0BD01CE010E94F326F601A481B58195
:10605000109739F04D915C9160E070E0CE010E94A4
:10606000A02AF601A485B585109769F0FD01E580A9
:10607000F6800381148122814D915C9160E070E093
:10608000CE010E946F24F601A289B389109749F0CE
:106090002D913D914D915C9160E070E0CE010E94A8
:1060A0009B23F601448955894115510529F060E08B
:1060B00070E0CE010E948C20F601A08DB18D10976A
:1060C00031F04C9160E070E0CE010E942D20D601AD
:1060D000ED91FC91309711F0608101C063E0CE0139
:1060E0000E945D4960E070E0CE010E946A28DF9165
:1060F000CF911F910F91FF90EF90DF90CF90089577
:106100008F929F92BF92CF92DF92EF92FF920F9366
:106110001F93CF93DF93EC01FC01EA5BFD4F80817D
:106120009181892B19F08FEF9FEF8FC0809184159B
:106130009091851591838083CE010D960E946C4AC3
:106140002DE6E22E22E0F22EEC0EFD1EC7010E948B
:106150006C4A8E01085B1D4FC8010E946C4AC70142
:106160000E94854AC8010E94854AFE01EE59FC4FF3
:10617000808091808EE19EE2918380838A819B81E1
:106180000E942F1840E052EC61E070E00E947732EC
:1061900081E088870E94454BCF58DD4F19921882C5
:1061A000C257D24099E7E92E92E0F92EEC0EFD1E7F
:1061B0006E0189E0B82EF70181898823E1F18FEF24
:1061C0009FEF93838283808191818F5F9F4F89F1BD
:1061D00000E01FEF2FEF3FEFF701408151816FEF9C
:1061E0007FEFCE010E9404388C018F5F9F4F81F7B3
:1061F000F7018189853091F4FE01E958FD4FCB58B4
:10620000DD4FA881B981C557D24020813181F70186
:106210004081518168E083E0FD01099589E792E0C2
:10622000C80ED91EF6011183008387E89DEFC80EC2
:10623000D91EF701118ABA9487E190E0C80ED91EE1
:10624000E80EF91EB7FEB7CFC401DF91CF911F91C1
:106250000F91FF90EF90DF90CF90BF909F908F9025
:106260000895EF92FF920F931F93CF93DF93EC016A
:106270008B0136E4E32E32E0F32EE80EF91EF7012F
:1062800080819181892BA1F06F5F7F4F89F00E94FF
:10629000544BCE010E94662FCE59DC4F19830883E0
:1062A000CE01855593400E94854AF70111821082E4
:1062B000DF91CF911F910F91FF90EF9008950F9371
:1062C0001F93CF93DF938C010E948030EC018FEFFE
:1062D000CF3FD80751F068EE73E080E090E00E9475
:1062E0005B05BE01C8010E943131DF91CF911F9142
:1062F0000F910895FC01E95DFD4F61937193318326
:1063000020837697518340830895FC01ED5BFD4F18
:10631000718360833C97518340830895FC01EB585F
:10632000FD4F619371935183408308950F931F93A1
:10633000CF93DF938C0188E893E00E94D508EC01AD
:10634000009709F44DC01983088360E070E0815E16
:106350009D4F0E942D4A60E070E0CE01825C9D4F0F
:106360000E942D4A61E070E0CE01885B9D4F0E9443
:106370002D4ACE010E94A73281E090E090939E15B5
:1063800080939D15CE010E946C3720E030E0A9017A
:106390006EE07EE2CE010E947A3140E050E06BE197
:1063A0007EE2CE010E94853140E050E06DE17EE268
:1063B000CE010E948E3120E034E0AE016FE17EE23A
:1063C0008DEA94E00E944E0BCE010E94662FCE0112
:1063D0008A599C4FAC0160E070E0CE010E94AB286E
:1063E000CE01DF91CF911F910F910895AF92BF928F
:1063F000CF92DF92EF92FF920F931F93CF93DF9391
:106400006C01B42EA22E20E0FC01E758FD4F8081E4
:10641000918177968617970719F02F5F2A30B8F386
:106420002A30A1F0822F992727E130E0829FE001F6
:10643000839FD00D929FD00D1124CC0DDD1DC6572A
:10644000DD4F8881CA58D240853029F06DEF7EEF4C
:106450008FEF9FEF39C0C601815E9D4F0E946C4A4D
:10646000FE01E257FD4F80818F5F808382E0F7015C
:106470008083FE01E558FD4F8081E70189832181FA
:106480008B2D99278370907064E0880F991F6A950F
:10649000E1F7282B8A2D99278370907056E0880F9A
:1064A000991F5A95E1F7282B2A830B83812F99276F
:1064B0008C83B701C6010E94B8359C01442737FD83
:1064C0004095542FCA01B901DF91CF911F910F91CF
:1064D000FF90EF90DF90CF90BF90AF900895FC01B8
:1064E000EE59FC4F619371935183408308950F934C
:1064F0001F93CF93DF93CDB7DEB724970FB6F894F1
:10650000DEBF0FBECDBF8C0149835A836B837C8372
:1065100040E050E0BA010E94F01984E60E94E70BC7
:10652000AE014F5F5F4F61E071E0C8010E948319C7
:10653000009711F08FEF9FEF24960FB6F894DEBF0F
:106540000FBECDBFDF91CF911F910F910895AF92F4
:10655000BF92CF92DF92EF92FF920F931F93CF9350
:10656000DF93CDB7DEB724970FB6F894DEBF0FBE2A
:10657000CDBF6C0161E070E004960E942D4A40E0BE
:1065800060E070E0F601808191810E943504892BE2
:1065900009F027C1F6018081918165EB74E00296D4
:1065A0000E943318F601938382830E942F181816D5
:1065B00019060CF016C1F601828193810E942F18F2
:1065C00040E052EC61E070E00E947732892B09F0E4
:1065D00008C119821A821B821C82F6018281938172
:1065E0000E942F18AE014F5F5F4F65E071E00E947F
:1065F0008319892B09F0F5C088E090E0A0E0B0E0B5
:1066000089839A83AB83BC83F601828193810E9444
:106610002F18AE014F5F5F4F63E071E00E94831956
:10662000892B09F0DEC081E090E0A0E0B0E0898332
:106630009A83AB83BC83F601828193810E942F18D9
:10664000AE014F5F5F4F67E071E00E948319892BB5
:1066500009F0C7C019821A821B821C82F60182814E
:1066600093810E942F18AE014F5F5F4F63E171E08D
:106670000E948319892B09F0B4C083E090E0A0E068
:10668000B0E089839A83AB83BC83F60182819381D6
:106690000E942F18AE014F5F5F4F61E171E00E94D1
:1066A00083195C01892B09F09CC0F6011086828158
:1066B00093810E942F18A501B5010E94F67280E017
:1066C00092E0A0E0B0E089839A83AB83BC83F601BB
:1066D000828193810E942F18AE014F5F5F4F6BE163
:1066E00071E00E9483197C010027F7FC0095102FB0
:1066F000F601828193810E942F18AE014F5F5F4F98
:106700006DE171E00E948319AA2797FDA095BA2F29
:10671000E80EF91E0A1F1B1F84EF91E0A0E0B0E015
:1067200089839A83AB83BC83F601828193810E9423
:106730002F18AE014F5F5F4F62E271E00E94831934
:10674000AA2797FDA095BA2FE80EF91E0A1F1B1F56
:10675000F601828193810E942F18AE014F5F5F4F37
:1067600066E271E00E948319AA2797FDA095BA2FCF
:10677000E80EF91E0A1F1B1F82EC91E0A0E0B0E0BA
:1067800089839A83AB83BC83F601828193810E94C3
:106790002F18AE014F5F5F4F60E271E00E948319D6
:1067A000AA2797FDA095BA2FE80EF91E0A1F1B1FF6
:1067B000F601828193810E942F18AE014F5F5F4FD7
:1067C00064E271E00E948319AA2797FDA095BA2F71
:1067D000E80EF91E0A1F1B1FE114F1040105110543
:1067E00019F04FEF5EEF01C0A501CA0124960FB664
:1067F000F894DEBF0FBECDBFDF91CF911F910F91F7
:10680000FF90EF90DF90CF90BF90AF9008952F92C0
:106810003F924F925F926F927F928F929F92AF9230
:10682000BF92CF92DF92EF92FF920F931F93CF937D
:10683000DF93CDB7DEB7C954D0400FB6F894DEBFB2
:106840000FBECDBF3C012B016A01FC01A280B380C9
:1068500088249924DE011196E8EBF4E082E10190AE
:106860000D928150E1F7A3E1B0E0AC0FBD1FEAEC5F
:10687000F4E08FE001900D928150E1F7A2E2B0E0E8
:10688000AC0FBD1FE9EDF4E086E101900D9281505F
:10689000E1F788E3282E312C2C0E3D1ED101EFEEBE
:1068A000F4E08EE001900D928150E1F78C149D048C
:1068B00008F077C08601081919097201E80CF91C63
:1068C000C5010E942F18A801B7010E94F6728C0121
:1068D000FFEF8F3F9F0741F4BE016F5F7F4F8BE05B
:1068E0000E94FA58C80186C0880E991EC5010E94F0
:1068F0002F18AE014A5B5F4F6AE071E00E94831976
:10690000F30180858E010A5B1F4F882371F087E0B9
:1069100090E0A0E0B0E0F80180839183A283B3838C
:10692000C5010E942F18A80137C0F80120813181CC
:1069300042815381DA01C90187709070A070B070F4
:106940000097A105B10509F4B1CFDA01C901817041
:106950009070A070B070892B19F063E170E004C0F2
:1069600021FF05C062E270E06C0F7D1F03C022FFB3
:1069700004C0B1018BE00E94FA5887E090E0A0E0EB
:10698000B0E0F80180839183A283B383C5010E94A4
:106990002F18AE014A5B5F4F69E071E00E948319D6
:1069A00085CF80912714882319F100E010E00C15A1
:1069B0001D05B0F47201F70181917F0199279F9322
:1069C0008F938AED90E09F938F930E9456750F905E
:1069D0000F900F900F900F5F1F4F0C151D0558F370
:1069E00081EE90E09F938F930E9456750F900F90C9
:1069F00080E090E0C75BDF4F0FB6F894DEBF0FBEBC
:106A0000CDBFDF91CF911F910F91FF90EF90DF905D
:106A1000CF90BF90AF909F908F907F906F905F903E
:106A20004F903F902F9008956F927F928F929F92F8
:106A3000AF92BF92CF92DF92EF92FF920F931F938C
:106A4000CF93DF93CDB7DEB763970FB6F894DEBF71
:106A50000FBECDBF3C014B016A01AA24BB24DE015D
:106A60001196EDEFF4E083E101900D928150E1F792
:106A700080912714882341F083EE90E09F938F93B9
:106A80000E9456750F900F90AC14BD04A8F48601B7
:106A90000A191B097401EA0CFB1CC3010E942F1880
:106AA000A801B7010E94F0198C012FEF8F3F9207C8
:106AB00091F1A80EB91EE8CF80912714882319F10F
:106AC00000E010E00C151D05B0F47401F701819190
:106AD0007F0199279F938F9385EE90E09F938F93EB
:106AE0000E9456750F900F900F900F900F5F1F4FE1
:106AF0000C151D0558F38CEE90E09F938F930E9428
:106B000056750F900F90C3010E948272FFEF8F3F66
:106B10009F0749F40AC0BE016F5F7F4F8BE00E9460
:106B2000FA58C80102C080E090E063960FB6F8946E
:106B3000DEBF0FBECDBFDF91CF911F910F91FF90B0
:106B4000EF90DF90CF90BF90AF909F908F907F900D
:106B50006F90089504960E946C4A089504960E94CE
:106B6000854A0895FC01828193810E94143508951D
:106B7000EF92FF920F931F93CF93DF937C018B01D2
:106B8000FB01808199278230910531F18330910595
:106B90001CF4019739F037C08330910541F1049717
:106BA00061F131C0FB018381C82FDD2723969281DB
:106BB000892F86958695833049F5892F9927982FB7
:106BC000882721813327822B932B93700397F1F42D
:106BD00081E0F70180871AC0FB0184819927D82FB3
:106BE000CC2783819927C82BD92B24960FC0FB0172
:106BF0008381C82FDD27239609C0FB018281C82F1E
:106C0000DD27229603C08FEF9FEF1BC02196C7019F
:106C10000E94AA35AE01B801C7010E94B2358C01AD
:106C2000C7010E94AE358FEFF701818B812F992725
:106C300087FD9095809590958827990F881F9927B3
:106C40000197DF91CF911F910F91FF90EF900895E1
:106C5000AF92BF92CF92DF92EF92FF920F931F936A
:106C6000CF93DF93CDB7DEB7A1970FB6F894DEBF11
:106C70000FBECDBF7C015B018A01FC018281938143
:106C8000DE011196E0E1F5E020E201900D92215045
:106C9000E1F70E942F1841E050E0BE016F5D7F4F89
:106CA0000E94F672019709F0CAC0809127148823C8
:106CB00071F089A199279F938F938EEE90E09F9317
:106CC0008F930E9456750F900F900F900F9089A18F
:106CD000482F55274330510509F440C04430510531
:106CE00024F44230510531F0A0C04430510509F47C
:106CF0005FC09BC00E948206DC01CB01F80180834B
:106D00009183A283B38323E132E0E20EF31EF70105
:106D1000008111812DEE3DEFE20EF31E89A1F801F5
:106D2000819344E050E0BF01C7010E9407346C0129
:106D3000892B09F084C0F80184819927582F4427B2
:106D400083819927482B592BF501518340834115A5
:106D5000510509F477C0C801059622C027E332E047
:106D6000E20EF31EF7010081118129EC3DEFE20EE6
:106D7000F31EF8018193BF01C7010E9407346C0123
:106D8000892B09F05CC0F8018381482F5527F50154
:106D9000518340834115510509F454C0C80104963C
:106DA000BC01C7010E940734892B09F44BC020C0E5
:106DB00087010F5E1E4FF801819342E050E0BF0152
:106DC000C7010E9407346C01892BC9F5F801828143
:106DD000482F5527F501518340834115510551F046
:106DE000C8010396BC01C7010E940734892B11F02A
:106DF000C60135C0F7018085882321F1F801818122
:106E00008E3001F59581892F86958695D9F4892F45
:106E10009927982F882724813327822B932B9370CF
:106E2000892B81F4F70110860DC0F7018085882336
:106E300031F4BE016F5F7F4F8CE00E94FA5880E012
:106E400090E00DC080912714882341F085EF90E0F9
:106E50009F938F930E9456750F900F90C801A19633
:106E60000FB6F894DEBF0FBECDBFDF91CF911F915B
:106E70000F91FF90EF90DF90CF90BF90AF9008956B
:106E8000089520E0DC01A459BD4FFC01E45BFD4FF7
:106E900080819181009721F4718360832C93089500
:106EA0008617970719F48EEF9FEF08952F5F32969C
:106EB000203170F38FEF9FEF08959C01FC01E4599E
:106EC000FD4F80818F3F39F08FEF8083C901835957
:106ED0009D4F0E94854A08950F931F93CF93DF9390
:106EE000EC011FEF198B61E070E009960E942D4ABA
:106EF000CF5EDE4F1883C151D1409FE0FE01E45BBD
:106F0000FD4F11921192915097FFFBCF2FEF3FEF62
:106F1000FE01E758FD4F99E0118A318320833383C6
:106F2000228380898F7C808B9150779697FFF4CF56
:106F3000CF58DD4F1882C157D24061E070E0CE01DA
:106F40000D960E942D4A8E0103591D4F60E070E09E
:106F5000C8010E942D4AFE01E459FD4F80818F3FF8
:106F600029F08FEF8083C8010E94854AFE01ED5E03
:106F7000FD4FC75EDD4FD183C083C951D240CE01E2
:106F8000875C9D4FC95CDD4F99838883DF91CF91EA
:106F90001F910F910895FF920F931F93CF93DF934B
:106FA000EC01F62E062F1127000F111F080F191FD5
:106FB000045B1D4FD801ED91FC91248335834683FA
:106FC0005783CF010A960E94C30AD801ED91FC9124
:106FD00011978FEF9FEF938782871D921C92FE017E
:106FE000E459FD4F80818F1549F48F3F39F08FEFC1
:106FF0008083CE0183599D4F0E94854ADF91CF91B6
:107000001F910F91FF9008956F927F929F92AF9280
:10701000BF92CF92DF92EF92FF920F931F93CF9385
:10702000DF935C016B013A01780189012FEF3FEF9B
:107030009924EC01C45BDD4FE991F9913097B9F0E7
:10704000828193818615970591F48FEFC8168FEF93
:10705000D80629F0808191818C159D0541F4A80105
:107060009701692DC5010E94CB3720E030E0939451
:107070008FE0891508F7C901DF91CF911F910F911A
:10708000FF90EF90DF90CF90BF90AF909F907F9058
:107090006F900895FC019A01AB01E459FD4F6081A6
:1070A000EC56F2406F3F19F0CF010E94CB370895A4
:1070B00020E0DC01A45BBD4FED91FD91309761F0C4
:1070C000808191818617970739F482819381841793
:1070D000950711F4CF0108952F5F203168F380E008
:1070E00090E0089540E06FEF7FEF20E030E0FC019A
:1070F000E758FD4F9189992369F481E0818B80895C
:10710000806F808B7183608373836283958B968B92
:10711000C90108954F5F77962F5F3F4F4A3050F374
:107120008FEF9FEF0895CF93DF932FEF6F3F72079D
:1071300031F41BC0E758FD4F6081718116C020E01B
:10714000DC01A558BD4FFC01ED018F85853031F480
:107150008D919C9111978617970761F32F5F779612
:1071600057962A3088F36FEF7FEFCB01DF91CF91F5
:10717000089520E0FC01E758FD4F8189853041F4F6
:10718000808191818617970719F4828193810895F0
:107190002F5F77962A3088F38FEF9FEF08958F92B5
:1071A0009F92AF92BF92CF92DF92EF92FF920F9396
:1071B000CF93DF93EC014B015A016901CA5BDD4FAC
:1071C00028813981C654D2402115310539F080918A
:1071D0008415909185152817390721F0CE010D9659
:1071E0000E946C4A033021F485E3E816F10421F093
:1071F000CE0109960E946C4A81E0F6018083000F5F
:10720000000F0283E182A114B10411F4A40101C0B2
:10721000A501CA01DF91CF910F91FF90EF90DF9010
:10722000CF90BF90AF909F908F9008958F929F9234
:10723000AF92BF92CF92DF92EF92FF920F931F9384
:10724000CF93DF93EC017B014A016901672B39F190
:107250008DE6A82E82E0B82EAC0EBD1EC5010E94A0
:107260006C4AF701D182C08213830283138612868F
:10727000B701CE010E9441378C01009771F08F5FFA
:107280009F4F39F468EE73E080E090E00E945B0568
:10729000EFCF8FEF0E3F1807C9F1012B49F7CE0151
:1072A0004196BC01CE010E94B8358C01CA5BDD4F0E
:1072B00028813981C654D2402115310539F0809199
:1072C0008415909185152817390721F0CE010D9668
:1072D0000E94854A0115110531F0B801882777FD14
:1072E0008095982F23C0E114F104E1F08928D1F4AE
:1072F00040E050E060E070E0C7010A960E94F009AB
:10730000F701648175818681978110C0C5010E9453
:10731000854ACE010D960E94854A60E07FEF8FEF8F
:107320009FEF04C060E070E080E090E0DF91CF91DB
:107330001F910F91FF90EF90DF90CF90BF90AF9093
:107340009F908F9008952F923F924F925F926F92ED
:107350007F928F929F92AF92BF92CF92DF92EF92E5
:10736000FF920F931F93CF93DF93CDB7DEB72B9789
:107370000FB6F894DEBF0FBECDBF5C017B01442485
:10738000552432012FEF3FEF38872F83190131E069
:107390003987FB012581822F9927D82ECC2484811F
:1073A0009927C82AD92A8FEF93E0C822D922269597
:1073B0002695E22FFF27FB87EA87E330F10509F4E2
:1073C000C3C0E430F1055CF4E130F105B9F0E2301E
:1073D000F1050CF061C0EF2B09F41EC345C32A85EB
:1073E0003B852530310509F488C2253031050CF480
:1073F000CDC12F33310509F41FC336C338E0C3169E
:10740000D10409F431C389E0C816D10428F492E00C
:10741000C916D10451F028C3ECE0CE16D104C1F155
:10742000FDE0CF16D10419F11FC3B8E48B2EB2E0F2
:107430009B2E8A0C9B1CC4010E945E4A4F8158857A
:1074400064E071E0C5010E945838009761F0FC01CA
:1074500004811581268137814F81588564E071E070
:10746000C5010E940438C4010E94854AFDC24F81B3
:10747000588564E07DE0C5010E945838DE01119610
:10748000F701379665E081918D93615067FFFBCFDF
:10749000C5010E945D37E8C2FDE0CF16D10499F125
:1074A0002EE0C216D10448F439E0C316D10471F0BD
:1074B0008CE0C816D104A9F0D7C29EE0C916D10449
:1074C00089F1EFE0CE16D104E9F1CEC2FB0180854F
:1074D0009927382E222487819927282A392A8185BD
:1074E000FBC0FB0180859927382E222487819927AC
:1074F000282A392A8681882381F482859927982F22
:107500008827218518C0FB0180859927382E2224E1
:1075100087819927282A392A8681992790958195EC
:107520009F4FD2C0FB0186818823B9F780859927B8
:10753000982F882727813327822B932B2C016624B1
:10754000772492C2FB01E8CFF8E1CF16D10409F409
:107550008BC229E1C216D104E8F53AE0C316D10482
:1075600009F482C28BE0C816D104A8F493E0C916CE
:10757000D10409F45FC0E4E0CE16D10408F474C26B
:10758000F5E0CF16D10409F46FC229E0C216D10488
:1075900009F4A0C069C235E1C316D10409F472C070
:1075A00086E1C816D10458F493E1C916D10409F450
:1075B0005BC2E4E1CE16D10409F493C055C2F6E1F2
:1075C000CF16D10409F450C227E1C216D10409F440
:1075D00059C04AC233E3C316D10409F445C284E357
:1075E000C816D10478F493E2C916D10471F1E4E22B
:1075F000CE16D10408F038C2F9E1CF16D10409F44F
:1076000069C032C223E4C216D10409F42DC234E4A5
:10761000C316D10450F486E3C816D10409F443C05C
:1076200097E3C916D104A9F11FC2E4E4CE16D10430
:1076300049F11AC225E432E0A20EB31EF501108210
:107640002BEB3DEFA20EB31E0FC2FB0181859927E4
:10765000AA27BB273C015524442480859927AA27C3
:10766000BB27BA2FA92F982F8827482A592A6A2A78
:107670007B2A87819927AA27BB27482A592A6A2A61
:107680007B2AF2C1F70180859927982F88272781C7
:1076900018C0FB0180859927382E222487819927DD
:1076A000282A392AE1C1FB0180859927382E222416
:1076B00087819927282A392A82859927982F882710
:1076C00021853327822B932B2C01662457FC609451
:1076D000762CCAC1F7018781482E55246624772469
:1076E000C3C14F8158856CE074E1C5010E945838D0
:1076F0008C01FC018084918484819581A681B7816D
:10770000893F9105A105B10544F088EF90E0A0E024
:10771000B0E084839583A683B78360E0F801848119
:107720009581A681B781481659066A067B06D4F46E
:10773000E62FFF27DF01A80DB91DEE0DFF1D878184
:107740008C93882379F06F5F262F332744275527A2
:10775000F80184819581A681B781281739074A07E6
:107760005B0734F3262F332744275527F8018481FC
:107770009581A681B781281739074A075B0709F465
:107780006150860E911CF40110826EC1F3E0CF1699
:10779000D10409F451C024E0C216D10428F431E028
:1077A000C316D10489F060C185E0C816D10409F47C
:1077B00056C095E0C916D10408F456C1E9E0CE16CA
:1077C000D10409F487C050C14F81588560E171E050
:1077D000C5010E945838FC01A085B185F701878159
:1077E0008C938085282F332781859927982F882788
:1077F000282B392BFD0132832183F7018285FD017E
:107800008383F7018385282F332784859927982F31
:107810008827282B392BFD0135832483F7018585A3
:10782000282F332786859927982F8827282B392BAF
:10783000FD013783268318C14F81588560E173E0CD
:10784000C5010E945838FC01A085B185F701349626
:1078500067E081918D93615067FFFBCF05C123E203
:1078600032E0A20EB31EFB0180859927982F88274E
:1078700027813327822B932BF501918380832FE17E
:1078800030E0A20EB31EFB018185F50180832EEB53
:107890003DEFA20EB31EFB0183859927982F882701
:1078A00022853327822B932BBC01C501815E9D4F1E
:1078B0000E94934AF70185859927982F8827248568
:1078C0003327822B932BBC01C501825C9D4F0E9404
:1078D000934ACAC04F81588560E179E0C5010E9492
:1078E0005838FC01A085B185F701379665E0819194
:1078F0008D93615067FFFBCFB7C0F5E0CF16D10481
:1079000039F126E0C216D10428F433E0C316D104BD
:1079100031F082C087E0C816D104E1F17DC0FB01DF
:1079200080859927382E222487819927282A392A69
:10793000B101C5010E949338AC0164E173E0C50157
:107940000E945838FC01A085B185F701818572C07D
:10795000FB0180859927382E222487819927282AA0
:10796000392AB101C5010E949338AC0164E175E088
:10797000C5010E945838FC01A085B185F7018285B8
:107980009927982F882721853327822B932B8D9336
:107990009C936AC02F803884A10164E177E0C5011F
:1079A0000E945838FC01A085B185109729F0F70195
:1079B000858599278D939C93F70184859927AA271C
:1079C000BB27782E66245524442483859927AA272B
:1079D000BB27DC0199278827482A592A6A2A7B2A4B
:1079E00082859927AA27BB27BA2FA92F982F8827E6
:1079F000482A592A6A2A7B2A81859927AA27BB27E0
:107A0000482A592A6A2A7B2A42E0440C551C661CE3
:107A1000771C4A95D1F728C0198626C08F0162814C
:107A20007381C5010E94B9381C01F801A085B18598
:107A3000F70187818C9318C0FFE0CF16D104A1F025
:107A400022E1C216D10481F460E0D501A45BBD4FF0
:107A5000ED91FD91309729F0808191818C5F924169
:107A6000E9F26F5F6031A0F3F7018681882349F066
:107A70009927909581959F4F2C01662457FC60941F
:107A8000762CFFEF2F16FFEF3F0631F0B101C50155
:107A90000E94933898878F832985222391F09C2D0B
:107AA0008827EA85FB85EE0FFF1FEE0FFF1F8E2B49
:107AB0009F2B930182014F815885BC01C5010E9413
:107AC0000438F70183819927BC01C50109960E94FA
:107AD000934A2B960FB6F894DEBF0FBECDBFDF9151
:107AE000CF911F910F91FF90EF90DF90CF90BF90BB
:107AF000AF909F908F907F906F905F904F903F904E
:107B00002F9008950F931F93CF93DF93EC018B0178
:107B1000FB018381882321F4CE010E945D370DC0D3
:107B20009927909581959F4FAA2797FDA095BA2FE9
:107B3000AC01BD01CE010E944A38F8018481992729
:107B4000BC01CE0109960E94934ADF91CF911F910B
:107B50000F9108952F923F924F925F926F927F9272
:107B60008F929F92AF92BF92CF92DF92EF92FF924D
:107B70000F931F93CF93DF93CDB7DEB726970FB642
:107B8000F894DEBF0FBECDBF5C016B016FEF662EB8
:107B9000762E88249924F6018181992783319105D5
:107BA00009F4ADC4843191058CF58530910509F453
:107BB0002DC3863091059CF48230910509F484C070
:107BC0008330910524F4019709F452C019C683301B
:107BD000910509F49FC1049709F47AC211C68F3048
:107BE000910509F4FEC38031910544F48730910575
:107BF00009F47FC30E9709F4EFC302C680319105E3
:107C000009F416C6429709F4F1C3FAC58B31910500
:107C100009F40EC68C3191059CF48631910509F466
:107C200038C58731910524F4449709F4B6C4E8C5F2
:107C30008731910509F43DC5489709F4F9C5E0C5B8
:107C40008232910509F440C08332910544F48C31AD
:107C5000910509F43EC54D9709F465C5D1C58F3E20
:107C6000910509F4B1C58F3F910509F489C5C8C5CF
:107C7000F6016381662389F0862F99279095819577
:107C80009F4FAA2797FDA095BA2F8C019D01A301B4
:107C900064E071E0C5010E940438A30164E071E072
:107CA000C5010E945838FC01048115812681378165
:107CB000A30164E071E0C5010E940438C501885B3E
:107CC0009D4F0E94854AB4C54FEF5FEF64E071E0BD
:107CD000C5010E9458388C01FC01E084F184F60152
:107CE000838188249924882309F404C1B60154E0CF
:107CF000452E512C4C0C5D1CF80184819581880D1A
:107D0000991DFC0144E0EE0FFF1F4A95E1F7E81BC7
:107D1000F90BEE0DFF1DD20186E00D90019281500E
:107D2000E1F7F80184819581880D991DDC0134E02B
:107D3000AA0FBB1F3A95E1F7A81BB90BAE0DBF1DEB
:107D4000FB0192859F70FD018681807F892B868350
:107D5000F80184819581880D991DDC0124E0AA0F2A
:107D6000BB1F2A95E1F7A81BB90BAE0DBF1DFB0188
:107D700093859295907FFD0186818F70892B8683F4
:107D8000F6018181F80124813581FB01A585768486
:107D9000823209F053C0C901880D991D1C01B4E05D
:107DA000220C331CBA95E1F7281A390A2E0C3F1C15
:107DB0008485282F3327442755278A2F9927AA27D8
:107DC000BB27BA2FA92F982F8827282B392B4A2B6E
:107DD0005B2B872D9927AA27BB27DC0199278827AA
:107DE000282B392B4A2B5B2BF101278330874187C6
:107DF0005287F80184819581880D991DDC0134E05A
:107E0000AA0FBB1F3A95E1F7A81BB90BAE0DBF1D1A
:107E1000FB0180899927982F882727853327822B74
:107E2000932B9068FD0194878387FB0181899927B3
:107E300087FD9095FD01968785874CC0C901880D07
:107E4000991D1C01B4E0220C331CBA95E1F7281AE5
:107E5000390A2E0C3F1C2A2F332744275527872DFC
:107E60009927AA27BB27BA2FA92F982F8827282B15
:107E7000392B4A2B5B2BFB0187859927AA27BB2728
:107E8000DC0199278827282B392B4A2B5B2BF10102
:107E90002783308741875287F80184819581880D37
:107EA000991DDC0134E0AA0FBB1F3A95E1F7A81B2E
:107EB000B90BAE0DBF1DFB0181899927982F88272B
:107EC00020893327822B932B9068FD019487838729
:107ED000168615860894811C911C2EE030E0420E17
:107EE000531E620F731FF601838199278816990626
:107EF0000CF402CFF6012381F80184819581A681DB
:107F0000B781820F911DA11DB11D84839583A68326
:107F1000B7838EC4DE01119656E0E52EF12CEC0CF1
:107F2000FD1CF70186E001900D928150E1F7882455
:107F30009924A9817A816B813C812D819E81F501F3
:107F4000E358FD4FA5018585882391F080818A172C
:107F500079F48181871761F48281861749F48381DE
:107F6000831731F48481821719F48581891759F0B8
:107F70000894811C911C495E5F4F77968AE08816B1
:107F800091040CF30AC08A0107581D4FF801608064
:107F900071800115110509F03EC022E633E0A20E02
:107FA000B31EF501808191812EE93CEFA20EB31E34
:107FB000892B09F03DC4C5010E9472384C019923F8
:107FC0000CF436C487E190E0889E8001899E100DF4
:107FD000989E100D11240A0D1B1D07581D4FD80126
:107FE0001496F70186E001900D928150E1F784E04C
:107FF000F801818B80919D1590919E159C010196B1
:1080000090939E1580939D153183208380898F7C6A
:108010008061808B3901F8012189822F992703978C
:10802000F6016381029708F045C0662361F0F8010C
:10803000118A8FEF9FEF9183808393838283F60170
:108040008381992739C0233009F061E085E0F80188
:10805000818BF6018481282F332785819927982FDA
:108060008827282B392BF80133832283F601948546
:108070009F70F8018089807F892B808B128A9501FF
:1080800029583D4F85E792E0A80EB91EF501A08161
:10809000B1818BE89DEFA80EB91EF90120813181D5
:1080A000F8014081518182E0FD0109958301222779
:1080B00033270AC0862F9927909581959F4F8C0171
:1080C000222717FD2095322FA30164E075E054C3E9
:1080D00022E633E0A20EB31EF501808191812EE9E4
:1080E0003CEFA20EB31E892B09F4A2C3DE01119648
:1080F00033E0632E712C6C0C7D1CF30186E0019043
:108100000D928150E1F7F6018185E82EFF240027CA
:10811000112782859927AA27BB27BA2FA92F982F25
:108120008827E82AF92A0A2B1B2B83859927AA2757
:10813000BB27DC0199278827E82AF92A0A2B1B2B61
:10814000C5010E9472384C018F5F9F4F09F470C3C4
:1081500087E190E0889EF001899EF00D989EF00DD9
:108160001124EA0DFB1DE358FD4FD30146E00D90AD
:1081700001924150E1F787E190E0889E9001899E4D
:10818000300D989E300D112449018A0C9B1C85E806
:1081900092E0880E991EF401E082F182028313833B
:1081A0002BE73DEF820E931ED401A757BD4FF6017A
:1081B00094859F708C91807F892B8C9329E732E086
:1081C000820E931E80919D1590919E159C010196A3
:1081D00090939E1580939D15F4013183208321E1B6
:1081E00030E0820E931E82E0F40181938C918F7CAB
:1081F00080618C934083F501EF58FD4F56C2890191
:1082000007581D4FF8016080718020C0F6018581FC
:108210009927582F442784819927482B592B84016B
:10822000F501E558FD4F95018785882329F0808168
:1082300091818417950719F30894811C911C295E7C
:108240003F4F77968AE08816910474F39AE0891676
:1082500091040CF0EDC2F60183818823E1F5F80169
:10826000818B5FEFE52EF52EF382E282F182E082D0
:1082700080898F7C808B950129583D4F85E792E05E
:10828000A80EB91EF501A081B1818BE89DEFA80E63
:10829000B91EF90120813181A301F601668183E0D5
:1082A000FD010995F60183819927909581959F4F4E
:1082B000AA2797FDA095BA2F8C019D01A30164E028
:1082C00076E0C5010E94043806EF1EEF2FEF3FEF66
:1082D000A301B70151C29927909581959F4FAA2775
:1082E00097FDA095BA2F8C019D01A30164E076E073
:1082F00043C2A30164E079E1C5010E9458388C01B2
:10830000FC016084718484819581A681B781893F55
:108310009105A105B10544F088EF90E0A0E0B0E040
:1083200084839583A683B783F80184819581A68190
:10833000B781181619061A061B06F4F47301B60164
:10834000665F7F4FFB018191BF01F70181937F0140
:10835000882391F00894811C911C9401442737FDD7
:108360004095542FF80184819581A681B781281703
:1083700039074A075B0734F39401442737FD4095DA
:10838000542FF80184819581A681B7812817390778
:108390004A075B0719F4089481089108680C791C56
:1083A000F3011082F6016381662351F0862F99272D
:1083B000909581959F4FAA2797FDA095BA2F05C04C
:1083C000C401AA2797FDA095BA2F8C019D014FEFFC
:1083D0005FEF64E079E1D0C1B601C5010E94A33925
:1083E00027C2B601C5010E94823D22C2F601248146
:1083F000D501A358BD4F8C918217F1F4FD019181F5
:10840000F60185819817C1F4FD019281F6018681FC
:10841000981791F4FD019381F6018781981761F413
:10842000FD019481F6018085981731F4FD01958155
:10843000F6018185981741F00894811C911C57968C
:10844000FAE08F169104BCF22AE08216910409F436
:10845000EFC187E190E0889E7001899EF00C989EA4
:10846000F00C1124EA0CFB1C89E792E0E80EF91EDF
:10847000F7016080718027E83DEFE20EF31EF60100
:108480009380992019F0892D9927BDC0D701A7574E
:10849000BD4FF601928593709295907F8C918F7C61
:1084A000892B8C9382859927AA27BB278C019D0154
:1084B000A30168E07BE0C5010E9404382AE832E0AD
:1084C000E20EF31EF7018081853009F0B1C19501FC
:1084D00029583D4F85E792E0A80EB91EF501A0810D
:1084E000B1818BE89DEFA80EB91EF9012081318181
:1084F000A301692DF6018285FD01099599C1F60157
:1085000083819927881699060CF092C18601F8019B
:1085100087819927982F882726813327822B932BB1
:10852000BC01C501815E9D4F0E94A04A40E050E021
:10853000D501A257BD4FB50165587D4FF801858122
:108540009927382F222784819927282B392BFB0143
:1085500080819181695E7F4F8217930759F4F801FA
:1085600087819927382F22279681922B8C91891BFE
:108570008C9306C04F5F5F4F57964A305105F4F217
:108580000894811C911C0C5F1F4FF6018381992771
:10859000881699060CF4BBCF4BC1F601858199274B
:1085A000382F222784819927282B392B3F70F501FA
:1085B000E558FD4F8081918177968217930739F0B6
:1085C0000894811C911C8AE0881691049CF39AE01F
:1085D0008916910409F42CC187E190E0889ED001AE
:1085E000899EB00D989EB00D1124AA0DBB1DA758F1
:1085F000BD4F6D907C901197A957B240F6018381D1
:10860000882371F09927909581959F4FAA2797FD10
:10861000A095BA2F8C019D01A30168E07BE0ACC05E
:10862000A557BD4FF60186818D938681882359F029
:1086300080859927982F882727813327822B932B92
:108640008D939C9302C01D921C9287E190E0889EBE
:10865000F001899EF00D989EF00D1124EA0DFB1D8E
:10866000E457FD4F80819181AA27BB27BA2FA92FFC
:10867000982F8827F6012681332744275527822BF8
:10868000932BA42BB52B8C019D01A3016FEF7FEFE2
:1086900073C0DE011196F601339686E001900D92CB
:1086A0008150E1F7F501EE58FD4F80818F5F8083A7
:1086B000BFC0DE011196F601339686E001900D925F
:1086C0008150E1F7BE016F5F7F4FC5010E94654792
:1086D000AFC0F60185819927982F882724813327F9
:1086E000822B932BBC01C5010E9493383C01F601FB
:1086F0008381882329F09927909581959F4F09C000
:10870000F60187819927982F882726813327822B86
:10871000932BAA2797FDA095BA2F8C019D01A30149
:1087200064E07FE129C0F60185819927982F882789
:1087300024813327822B932BBC01C5010E949338DF
:108740003C01F6018381882329F099279095819532
:108750009F4F09C0F60187819927982F8827268186
:108760003327822B932BAA2797FDA095BA2F8C0134
:108770009D01A30164E07FE0C5010E94043858C058
:10878000F60182819927881699060CF051C086015E
:108790000D5F1F4FF80181918F0199279F938F9350
:1087A00080E395E09F938F930E9405190F900F909F
:1087B0000F900F900894811C911CF60182819927DB
:1087C000881699063CF334C001E0802E912CF60106
:1087D00082819927881699065CF586010C5F1F4FE8
:1087E000F80181918F0199270E94A0720894811C41
:1087F000911CF60182819927881699068CF318C07E
:10880000F601828188249924882391F086010D5FE6
:108810001F4FF80181918F0199270E94A07208943F
:10882000811C911CF60182819927881699068CF388
:1088300021E131E0A20EB31E8FEFF5018083269671
:108840000FB6F894DEBF0FBECDBFDF91CF911F9161
:108850000F91FF90EF90DF90CF90BF90AF909F90DF
:108860008F907F906F905F904F903F902F900895E2
:108870006F927F928F929F92AF92BF92CF92DF9230
:10888000EF92FF920F931F93CF93DF93CDB7DEB795
:108890002C970FB6F894DEBF0FBECDBF5C013B0135
:1088A000942E822E6801419621E0E22EF12C01E007
:1088B0009C01AB01BE016E0D7F1DC5010E94CF382A
:1088C0007C01C501885B9D4F0E946C4AF7011482B0
:1088D000158216821782D186C08685E0F501848BC9
:1088E00083E3858B8BE8868B8EE9878BF0E3F91524
:1088F00008F49F2EF501908E882011F481E0882ED7
:10890000F501818E0FEF1FEF24E031E0A301B701E5
:10891000C5010E941639DC01CB01BC01CD012C96AA
:108920000FB6F894DEBF0FBECDBFDF91CF911F9180
:108930000F91FF90EF90DF90CF90BF90AF909F90FE
:108940008F907F906F900895AF92BF92CF92DF92F9
:10895000EF92FF920F931F93CF93DF93CDB7DEB7C4
:108960002C970FB6F894DEBF0FBECDBF6C015B0134
:10897000419632E0E32EF12C01E09C01AB01BE01F7
:108980006F5F7F4FC6010E94CF38F601148A0FEF48
:108990001FEF24E032E0A501BC01C6010E94163998
:1089A000DC01CB01BC01CD012C960FB6F894DEBFE3
:1089B0000FBECDBFDF91CF911F910F91FF90EF9030
:1089C000DF90CF90BF90AF9008952F923F924F923B
:1089D0005F926F927F928F929F92AF92BF92CF924F
:1089E000DF92EF92FF920F931F93CF93DF93CDB758
:1089F000DEB72D970FB6F894DEBF0FBECDBF5C017A
:108A00001B014A0139010D8727011C2DBA010E9463
:108A10008A2DDC01CB018D5F9E4FAF4FBF4F29F0F8
:108A200069EF7EEF8FEF9FEFD4C020E030E0F401DC
:108A30004081D501A358BD4F8C91841731F5FD01BC
:108A40009181F4018181981701F5FD019281F40172
:108A500082819817D1F4FD019381F40183819817E5
:108A6000A1F4FD019481F4018481981771F4FD0152
:108A70009581F4018581981741F4FD018585833046
:108A800089F18230A1F1843091F12F5F3F4F5796E9
:108A90002A30310588F2CC24DD24F501E757FD4F5B
:108AA00029E030E08181853041F4808182958F70AA
:108AB000837019F40894C11CD11C21503040779662
:108AC00037FFF0CFF7E0CF16D1043CF4C5010E9488
:108AD00072386C018F5F9F4F79F46CEF7EEF8FEFF0
:108AE0009FEF77C068EF7EEF8FEF9FEF72C067EF69
:108AF0007EEF8FEF9FEF6DC0C501419665E0E62EDA
:108B0000F12C01E09C01A101BE016F5F7F4FC50107
:108B10000E94CF38BC018DE0F501848BD5015596BC
:108B2000F40126E001900D922150E1F7F501638EEA
:108B3000872D9927848F8D85858F268F478E852D4C
:108B4000992780A311A387E190E0C89EF001C99EF8
:108B5000F00DD89EF00D1124EA0DFB1DE358FD4FDA
:108B6000D40186E00D9001928150E1F787E190E019
:108B7000C89EF001C99EF00DD89EF00D1124EA0D9B
:108B8000FB1DE657FD4F83E08083EA58F240DF018A
:108B9000A758BD4F80919D1590919E159C010196FF
:108BA00090939E1580939D1511963C932E93E757B5
:108BB000FD4F1295110F110F107C80818F70812B4A
:108BC00080830D911C9124E035E0A101C5010E9434
:108BD00016392D960FB6F894DEBF0FBECDBFDF91CC
:108BE000CF911F910F91FF90EF90DF90CF90BF90AA
:108BF000AF909F908F907F906F905F904F903F903D
:108C00002F9008958F929F92AF92BF92CF92DF9252
:108C1000EF92FF920F931F93CF93DF93CDB7DEB701
:108C20002C970FB6F894DEBF0FBECDBF5C014B0191
:108C30006A01419678E0E72EF12C01E09C01A40145
:108C4000BE016F5F7F4FC5010E94CF38BC0186E037
:108C5000F501848BD5015596F60101900D92815056
:108C6000E1F70FEF1FEF24E038E0A401C5010E94F7
:108C70001639DC01CB01BC01CD012C960FB6F8945E
:108C8000DEBF0FBECDBFDF91CF911F910F91FF903F
:108C9000EF90DF90CF90BF90AF909F908F9008950E
:108CA0006F927F928F929F92AF92BF92CF92DF92FC
:108CB000EF92FF920F931F93CF93DF93CDB7DEB761
:108CC0002C970FB6F894DEBF0FBECDBF6C013B01F1
:108CD0004A01122FBA010E94B9385C018FEFA81621
:108CE0008FEFB80629F46DEF7EEF8FEF9FEF1EC078
:108CF000C6014196B6E0EB2EF12C01E09C01A301E8
:108D0000BE016F5F7F4FC6010E94CF38BC0183E078
:108D1000F601848BA58A8B2D9927868B178B84016E
:108D200024E036E0A301C6010E9416392C960FB646
:108D3000F894DEBF0FBECDBFDF91CF911F910F9191
:108D4000FF90EF90DF90CF90BF90AF909F908F906B
:108D50007F906F900895AF92BF92CF92DF92EF9283
:108D6000FF920F931F93CF93DF93CDB7DEB72C976E
:108D70000FB6F894DEBF0FBECDBF5C016B01142FA0
:108D8000419609E0E02EF12C01E09C0140E050E02A
:108D9000BE016F5F7F4FC5010E94CF3887E0F501AC
:108DA000848BD5015596F60186E001900D92815095
:108DB000E1F7F501138F0FEF1FEF24E039E040E0FA
:108DC00050E0BA01C5010E941639DC01CB01BC019B
:108DD000CD012C960FB6F894DEBF0FBECDBFDF914C
:108DE000CF911F910F91FF90EF90DF90CF90BF90A8
:108DF000AF9008956F927F928F929F92AF92BF92A1
:108E0000CF92DF92EF92FF920F931F93CF93DF9356
:108E1000CDB7DEB72C970FB6F894DEBF0FBECDBF2F
:108E20006C014B015A0139010E94B9388F5F9F4F85
:108E300029F46DEF7EEF8FEF9FEF32C0C6014196B0
:108E40002BE0E22EF12C01E09C0140E050E0BE015D
:108E50006F5F7F4FC6010E94CF3886E1F601848B99
:108E6000D6015596F50186E001900D928150E1F70B
:108E7000D6015B96F3019301225F3F4F80818D9372
:108E80008081882321F031962E173F07B8F784019F
:108E900024E03BE040E050E0BA01C6010E941639F0
:108EA0002C960FB6F894DEBF0FBECDBFDF91CF91E9
:108EB0001F910F91FF90EF90DF90CF90BF90AF90F8
:108EC0009F908F907F906F900895AF92BF92CF92B6
:108ED000DF92EF92FF920F931F93CF93DF93CDB763
:108EE000DEB72C970FB6F894DEBF0FBECDBF5C0186
:108EF0006B0141963CE0E32EF12C01E09C0140E047
:108F000050E0BE016F5F7F4FC5010E94CF3886E001
:108F1000F501848BD5015596F60101900D92815093
:108F2000E1F70FEF1FEF24E03CE040E050E0BA0132
:108F3000C5010E941639DC01CB01BC01CD012C9684
:108F40000FB6F894DEBF0FBECDBFDF91CF911F915A
:108F50000F91FF90EF90DF90CF90BF90AF9008956A
:108F60004F925F927F928F929F92AF92BF92CF92D9
:108F7000DF92EF92FF920F931F93CF93DF93CDB7C2
:108F8000DEB72C970FB6F894DEBF0FBECDBF6C01D5
:108F90002B015A01722E480141964DE0E42EF12C2E
:108FA00001E09C0140E050E0BE016F5F7F4FC601D1
:108FB0000E94CF38BC0187E1F601848BD60155961B
:108FC000F50186E001900D928150E1F7F601738E74
:108FD00040E050E0272D33274217530770F4D601A5
:108FE0005C96F40180818D938081882331F04F5FFE
:108FF0005F4F319642175307A8F3FB01B186A08655
:10900000820124E03DE040E050E0BA01C6010E9448
:109010001639DC01CB01BC01CD012C960FB6F894BA
:10902000DEBF0FBECDBFDF91CF911F910F91FF909B
:10903000EF90DF90CF90BF90AF909F908F907F90F8
:109040005F904F9008954F925F926F927F928F92B0
:109050009F92AF92BF92CF92DF92EF92FF920F93C7
:109060001F93CF93DF93CDB7DEB72C970FB6F8944D
:10907000DEBF0FBECDBF6C014B012A013901BA0121
:109080000E94B9385C018FEFA8168FEFB80629F45B
:109090006DEF7EEF8FEF9FEF22C0C6014196BFE0DC
:1090A000EB2EF12C01E09C01A401BE016F5F7F4F0C
:1090B000C6010E94CF38BC0184E0F601848BA58AEA
:1090C0008B2D9927868B678A872D9927808F820120
:1090D00024E03FE040E050E0C6010E9416392C96A3
:1090E0000FB6F894DEBF0FBECDBFDF91CF911F91B9
:1090F0000F91FF90EF90DF90CF90BF90AF909F9037
:109100008F907F906F905F904F9008950F931F9373
:109110008B0124E031E140E050E0BA010E941639B1
:10912000DC01CB01BC01CD011F910F9108955F922D
:109130006F927F928F929F92AF92BF92CF92DF9267
:10914000EF92FF920F931F93CF93DF93CDB7DEB7CC
:109150002C970FB6F894DEBF0FBECDBF4C015B015C
:109160003A01522E68011E2D419609E1E02EF12CA4
:1091700001E09C0140E050E0BE016F5F7F4FC40101
:109180000E94CF38BC01FC01D186C086812F99276F
:10919000AA27BB2784839583A683B7838AE0F4013B
:1091A000848BD4015596F50186E001900D92815093
:1091B000E1F7F401538E848F658E872D9927868F72
:1091C0000FEF1FEF24E039E140E050E0C4010E94BE
:1091D0001639DC01CB01BC01CD012C960FB6F894F9
:1091E000DEBF0FBECDBFDF91CF911F910F91FF90DA
:1091F000EF90DF90CF90BF90AF909F908F907F9037
:109200006F905F9008956F927F928F929F92AF922E
:10921000BF92CF92DF92EF92FF920F931F93CF9363
:10922000DF93CDB7DEB72C970FB6F894DEBF0FBE35
:10923000CDBF6C014B013A01BA010E94B9385C0103
:109240008FEFA8168FEFB80629F46DEF7EEF8FEF42
:109250009FEF1EC0C60141962FE1E22EF12C01E0E6
:109260009C01A401BE016F5F7F4FC6010E94CF38F1
:10927000BC0182E0F601848BA58A8B2D9927868B11
:10928000830124E03FE140E050E0C6010E9416392E
:109290002C960FB6F894DEBF0FBECDBFDF91CF91F5
:1092A0001F910F91FF90EF90DF90CF90BF90AF9004
:1092B0009F908F907F906F9008954F925F926F92E2
:1092C0007F928F929F92BF92CF92DF92EF92FF9206
:1092D0000F931F93CF93DF93CDB7DEB72C970FB6C5
:1092E000F894DEBF0FBECDBF6C01B62E8C010459C1
:1092F0001C4FD8018D919C91892B39F481E090E02D
:109300000E946408F80191838083D801ED91FC915B
:10931000B0826B2D77276230710561F16330710582
:109320003CF461157105C1F16130710561F170C0E6
:109330006430710579F064307105A4F06530710511
:1093400009F066C0412C8BE4582E612C712C03E08F
:10935000B02E2AC0412C16E9512E612C712CB4E09C
:10936000BB2E22C0412CA1EE5A2E612C712CF6E0AE
:10937000BF2E1AC0412CE2EC5E2EE1E06E2E712C65
:1093800078E0B72E11C0412C64E8562E63E0662EBB
:10939000712C5AE0B52E08C0412C48E0542E47E00D
:1093A000642E712C3CE0B32EC60141962FE0E22ED4
:1093B000F12C0FE39C0140E050E0BE016F5F7F4F56
:1093C000C6010E94CF384C0185E0F601848B83E012
:1093D000858B168A178AB08E118E0FEF1FEF2CEF38
:1093E0003FE0A401B401C6010E9416397B018C0143
:1093F000611571058105910559F4F601828193810A
:109400000E942F18B301A2010E947732892B29F004
:109410004FEF5EEF6FEF7FEF08C0B801A701C40107
:109420000A960E94F009B801A701CB01BA012C9657
:109430000FB6F894DEBF0FBECDBFDF91CF911F9165
:109440000F91FF90EF90DF90CF90BF909F908F9003
:109450007F906F905F904F9008950F931F93CF93DD
:10946000DF938C01F80111821082738362838091F3
:10947000281490912914009751F484E090E00E9400
:10948000D508FC01909329148093281410C0EC0196
:109490008A819B81892B21F00A80DB81C02DF8CF46
:1094A00084E090E00E94D508FC019B838A831183AD
:1094B0000083DF91CF911F910F910895FC0182816C
:1094C0009381009731F001979383828380E090E04D
:1094D00008958FEF9FEF0895CF93DF93EC018A817A
:1094E0009B81892B41F440E050E060E070E0CE01C8
:1094F0000E94F009F4CF8A819B8101979B838A8324
:1095000080E090E0DF91CF910895FC01828193810A
:10951000019693838283019719F4CF010E94690A0F
:1095200080E090E00895FC0122813381738362839F
:10953000232B19F4CF010E94C30A80E090E0089524
:10954000FC01CB0122813381820F931F938382839D
:10955000232B19F4CF010E94C30A80E090E0089504
:10956000CF93DF93C0912814D09129142097E9F06C
:10957000E881F981828193819F938F93888199817A
:109580009F938F9386E395E09F938F930E946E58ED
:109590000A80DB81C02D8DB79EB706960FB6F89472
:1095A0009EBF0FBE8DBF209719F7DF91CF91089511
:1095B00060EB7AE483E495E00E9452540895189A8F
:1095C000939A8B9A80E00E94ED0308950895882372
:1095D00021F087E00E94B24B089587E00E94A54BDE
:1095E000089584B7806884BF84BF089584B78F7757
:1095F00084BF84BF089580919A00877F80939A00EA
:109600008B9893988A9892988C98949815981D980E
:10961000809161008F7B80936100809162008F7BDD
:1096200080936200809161008F7D809361008091C2
:1096300062008F7D80936200809161008F7E8093B5
:109640006100809162008F7E809362000895809116
:109650009A00886080939A008B9A939A8A98929A3B
:109660008C9A15980895882321F086E00E94A54BD6
:1096700003C086E00E94B24B88E495E00E94FB4A5A
:1096800088E495E00E94F14A089588E495E00E94FC
:10969000FB4A88E495E00E94F14A80E00E94334B47
:1096A00081E00E94E74A089581E00E94334B64EF15
:1096B00071E080E090E00E945B0580E00E94E74A54
:1096C00088E495E00E94F64A88E495E00E94274BE2
:1096D00060ED77E080E090E00E945B0508950E94D5
:1096E000454B68EE73E080E090E00E945B050E94CD
:1096F000544B0895882321F085E00E94A54B0895DE
:1097000085E00E94B24B0895882321F084E00E94F6
:10971000A54B089584E00E94B24B0895282F0FB600
:10972000F8940F929927F82FEE2780818083C59AAD
:109730000000C5980F900FBE20932A140895BD9A7B
:1097400080912A140E948E4B089521E030E002C0DF
:10975000220F331F8A95E2F780912A14822B0E94F0
:109760008E4B089521E030E002C0220F331F8A950E
:10977000E2F7922F909580912A1489230E948E4BB4
:1097800008951F93CF93DF9310E0C0E0D0E0809165
:109790009F1599270C2E02C0959587950A94E2F79C
:1097A00080FF04C0812F0E94D77603C0812F0E94C2
:1097B000E5761F5F2196143050F3DF91CF911F9112
:1097C0000895CF93DF93C82FDD27C0FF04C080E04A
:1097D0000E94D77603C080E00E94E576C1FF04C0F6
:1097E00081E00E94D77603C081E00E94E576C2FF47
:1097F00004C082E00E94D77603C082E00E94E57632
:10980000C3FF04C083E00E94D77603C083E00E94B8
:10981000E576DF91CF910895562F622F9091B7157D
:10982000292F3327F901EE0FFF1FEE0FFF1FEF5512
:10983000FA4E8083518342836383C901019665E0B8
:1098400070E00E94797D8093B715982F8091A015C4
:10985000981749F4892F9927019665E070E00E94D6
:10986000797D8093A0150895C0E086E90E940608DE
:10987000E091A0158091B715E81719F41092B5156D
:1098800021C0FF27EE0FFF1FEE0FFF1FEF55FA4E0F
:1098900080818093B51510E0812F0E94E5761F5FCF
:1098A0001430D0F38091A015E82FFF27EE0FFF1F93
:1098B000EE0FFF1FEF55FA4E83818F3F11F081505D
:1098C0008383C2818091B51599278430910509F46D
:1098D0008DC08530910594F48130910509F457C00D
:1098E000823091051CF4892BC9F079C18230910531
:1098F00009F465C0039709F4A6C071C186309105CB
:1099000009F4E3C0863091050CF4C0C0873091059E
:1099100009F4FCC0089709F434C161C1809149057C
:10992000882359F10E948C6A7B018C0190914A0531
:109930008FE3989FC00111249C0144275527C8013B
:10994000B7010E948C7DDC01CB01CF97A105B10549
:10995000A0F460912B14662321F021E04091490589
:1099600007C080919F15882331F421E0422F622F98
:1099700084E00E940C4C1092B6158091B6158F5F52
:109980008093B6156FE370E080E090E025C1809190
:10999000A015E82FFF27EE0FFF1FEE0FFF1FEF555B
:1099A000FA4E81810E94E14B8FE3C89FC0011124D0
:1099B000AA2797FDA095BA2FBC01CD010DC18091BA
:1099C000A015E82FFF27EE0FFF1FEE0FFF1FEF552B
:1099D000FA4E81810E94E14B8FE3C89FC0011124A0
:1099E0007C010027F7FC0095102F22C080E00E9428
:1099F000E14B8FE3C89FC00111247C010027F7FCD5
:109A00000095102FC801B7010E945B058091B51524
:109A1000882309F4EFC08091A015E82FFF27EE0FEF
:109A2000FF1FEE0FFF1FEF55FA4E81810E94E14BA1
:109A3000C801B7010E945B058091B515882309F420
:109A4000D9C080E020C080E00E94E14B8FE3C89F36
:109A5000C00111247C010027F7FC0095102FC801DC
:109A6000B7010E945B058091B515882309F4C2C037
:109A70008091A015E82FFF27EE0FFF1FEE0FFF1FAD
:109A8000EF55FA4E81810E94E14BA4C080E00E9414
:109A9000D77610E08FE3C89FC00111246C01EE243B
:109AA000D7FCE094FE2CC701B6010E945B058091B3
:109AB000B515882341F1812F0E94E5761F5F812F24
:109AC0000E94D776133030F31EC083E00E94D77611
:109AD00013E08FE3C89FC00111246C01EE24D7FC72
:109AE000E094FE2CC701B6010E945B058091B5157C
:109AF000882349F0812F0E94E5761150812F0E9422
:109B0000D776112331F7C701B60166C080E00E9405
:109B1000D77610E08FE3C89FC00111249C01442731
:109B200037FD4095542FCA01B9010E945B05809111
:109B3000B515882349F0812F0E94E5761F5F812F9C
:109B40000E94D776133030F313E08FE3C89FC00133
:109B500011249C01442737FD4095542FCA01B901B7
:109B60000E945B058091B515882309F443C0812FBD
:109B70000E94E5761150812F0E94D776112329F794
:109B800039C080E00E94D77681E00E94D77682E0DB
:109B90000E94E57683E00E94E5768FE3C89FC001CE
:109BA00011247C010027F7FC0095102FC801B70194
:109BB0000E945B058091B5158823E1F080E00E944A
:109BC000E57681E00E94E57682E00E94D77683E028
:109BD0000E94D776C801B7010E945B050BC0809137
:109BE000A015E82FFF27EE0FFF1FEE0FFF1FEF5509
:109BF000FA4E13828091B515882309F439CE8091ED
:109C0000A015282F3327F901EE0FFF1FEE0FFF1FBE
:109C1000EF55FA4E8381882309F02ACEC9010196B7
:109C200065E070E00E94797D2091B7153327821797
:109C3000930711F40E94C14B8091A01599270196BA
:109C400065E070E00E94797D8093A01511CE80912F
:109C5000B7158093A0150E94C14B1092B5150895B9
:109C600080934A0560932B144093490508951F93F0
:109C7000182F0E94F3761092B7151092A015112399
:109C800051F020E034E040E050E064E37CE48BE419
:109C900095E00E944E0B1F910895CF93C82F80919D
:109CA000B515882319F48C2F0E94D77681E090E0B7
:109CB00002C0880F991FCA95E2F720919F15282BA3
:109CC00020939F15CF910895CF93C82F8091B515FC
:109CD000882319F48C2F0E94E57681E090E002C081
:109CE000880F991FCA95E2F7982F909580919F153C
:109CF000892380939F15CF910895CF93DF9380910F
:109D00004E1590914F152EEF30E0281B390B24177C
:109D1000350710F4E90101C0EA0180912C149091FB
:109D20002D140E944A5180914E1590914F158C0F21
:109D30009D1F90934F1580934E15CE01DF91CF91CB
:109D40000895EF92FF920F931F93CF93DF93CDB7B8
:109D5000DEB72B970FB6F894DEBF0FBECDBFFC88E1
:109D6000ED880E891F89EF2DFF27E45DFB4E828170
:109D7000282F33278E2D9927019702C035952795D7
:109D80008A95E2F720FF54C00E948C6ADC01CB0167
:109D90008D839E83AF83B88710924F1510924E1516
:109DA0009E01285E3F4FA80160E070E08DE79EE4D1
:109DB0000E943B1A00914E1510914F150E3F110550
:109DC00061F441E050E06FE475E080912C149091D3
:109DD0002D140E944A510F5F1F4F41E050E061E592
:109DE00075E080912C1490912D140E944A510F5FC0
:109DF0001F4F80915015909151159C0101969093A1
:109E00005115809350153A832983FB82EC821A877F
:109E100009874BE050E0BE016F5F7F4F80912C14AB
:109E200090912D140E944A5182E595E10E94C30A47
:109E30002B960FB6F894DEBF0FBECDBFDF91CF914A
:109E40001F910F91FF90EF90089580912C149091A5
:109E50002D140E948B5208956F927F928F929F9241
:109E6000AF92BF92CF92DF92EF92FF920F931F9328
:109E7000CF93DF93CDB7DEB72B970FB6F894DEBF45
:109E80000FBECDBF6C01762E642E49015801809122
:109E90002C1490912D140E9457528C01892B09F497
:109EA0003EC0EE24FF244BE050E0BE016F5F7F4FC9
:109EB000C8010E94CD51892B79F549855A856EE4F8
:109EC00074E1C8010E94CD51892B31F5772019F03A
:109ED0008B818715A9F4862D99272C813327215052
:109EE000304002C0959587952A95E2F780FF08C01B
:109EF000A501BE016F5F7F4F8EE494E1F4010995E7
:109F00000894E11CF11CC114D10419F0CE14DF0433
:109F100019F00E94B407C7CFC8010E947A522B964D
:109F20000FB6F894DEBF0FBECDBFDF91CF911F916A
:109F30000F91FF90EF90DF90CF90BF90AF909F90E8
:109F40008F907F906F9008957F928F929F92AF92A3
:109F5000BF92CF92DF92EF92FF920F931F93CF9316
:109F6000DF93CDB7DEB72B970FB6F894DEBF0FBEE9
:109F7000CDBF6C018B014A01590180912C14909145
:109F80002D140E9457527C01892BE9F1011511050E
:109F900019F00C0D1D1D06C00091501510915115A2
:109FA0000150104077244BE050E0BE016F5F7F4FBF
:109FB000C7010E94CD51892B19F589819A818C1591
:109FC0009D05F1F049855A856EE474E1C7010E9450
:109FD000CD51892BA9F489819A818017910719F4B1
:109FE00081E0782E02C0772041F0A501BE016F5FAD
:109FF0007F4F8EE494E1F40109950E94B407D3CF1A
:10A00000C7010E947A522B960FB6F894DEBF0FBE9E
:10A01000CDBFDF91CF911F910F91FF90EF90DF9017
:10A02000CF90BF90AF909F908F907F900895E82F32
:10A0300081508F3130F4FF27E45DFB4E82819927F8
:10A0400008958FEF9FEF0895E82F81508F3120F40E
:10A05000FF27E45DFB4E62830895CF93DF93CDB776
:10A06000DEB7CB50D1400FB6F894DEBF0FBECDBFE8
:10A0700088EC0E940608AA24BB2440E050E060E07F
:10A0800070E082E595E10E94F00980912C14909196
:10A090002D140E9457528C01C0905015D09051152C
:10A0A0000894C108D10880915A15882311F140E025
:10A0B00050E060E070E08BE595E10E94F009C80196
:10A0C0000E949D52882389F4A0905015B09051159C
:10A0D0000894A108B108C8010E947A5280912C14FA
:10A0E00090912D140E9457528C0182E595E10E94B7
:10A0F000690A4BE050E0BE016F5F7F4FC8010E94CC
:10A10000CD51892B09F042C089819A818A159B051E
:10A11000E9F18091561590915715892B79F18B8132
:10A12000E0915415F0915515E80FF11D8081282F0D
:10A1300033278C819927019702C0359527958A95F9
:10A14000E2F720FF1BC09CE0E92EF12CEC0EFD1E77
:10A1500049855A85B701C8010E94CD51892BB1F4B8
:10A16000E0915615F0915715409158155091591599
:10A17000BE016F5F7F4FC701099505C069857A856C
:10A18000C8010E9427520E94B4078DCF5601C80112
:10A190000E947A5280915015909151150197C816DE
:10A1A000D90609F072CF69CF9C0180915615909124
:10A1B0005715009719F08FEF9FEF089530935715BB
:10A1C0002093561570935915609358155093551553
:10A1D00040935415089510925715109256151092E9
:10A1E000591510925815109255151092541508953E
:10A1F00081E080935A15089510925A1580915B154D
:10A2000090915C15892B21F08BE595E10E94B80AAD
:10A210000895CF93DF93C4E5D5E1109251151092C4
:10A22000501510924F1510924E1510925315109212
:10A23000521510925A1510925C1510925B1540E061
:10A2400058EC60E074E082E090E00E94A7529093A6
:10A250002D1480932C148FEFFE01E652F140819370
:10A2600094E1ED34F907D9F3D0F31B821A821D82F1
:10A270001C82109255151092541520E034E040E0F5
:10A2800050E06DE270E583E595E00E944E0BDF91B2
:10A29000CF910895CF92DF92EF92FF920F931F9389
:10A2A000CF93DF93EC016B017A01488559854E15F8
:10A2B0005F0518F48EEF9FEF67C0CA018E199F09E2
:10A2C0002E813F818217930718F45F834E8304C069
:10A2D0002E0D3F1D3F832E8352E0FE01452F8089C6
:10A2E0008130A1F42E813F8188859985281739070F
:10A2F00069F4868597858E159F0520F4508B178607
:10A30000168604C08E199F09978786874150379615
:10A3100047FFE5CF088519852C813D81021B130B72
:10A320000E151F05B0F44427552788819981AA810D
:10A33000BB81820F931FA41FB51F9801AC01BD0103
:10A34000C6010E944A771D821C82E01AF10AC00EE3
:10A35000D11E8C819D819C0144275527888199813C
:10A36000AA81BB81820F931FA41FB51F9701AC0167
:10A37000BD01C6010E944A778C819D818E0D9F1D73
:10A380009D838C8380E090E0DF91CF911F910F91AE
:10A39000FF90EF90DF90CF900895CF92DF92EF92F1
:10A3A000FF920F931F93CF93DF93EC016B018A0110
:10A3B000E880F9808E81823019F48DEF9FEF3EC0E6
:10A3C0008C819D818417950728F482E08E838EEF1F
:10A3D0009FEF34C0841B950B9D838C832A813B8126
:10A3E0002417350788F4021B130BF70140815181B4
:10A3F00062817381C601800F911F0E94F777F70178
:10A40000808591859B838A838A819B81801B910BA8
:10A410009B838A839C0144275527F7018081918182
:10A42000A281B381820F931FA41FB51F9801AC01B5
:10A43000BD01C6010E94F77780E090E0DF91CF91E7
:10A440001F910F91FF90EF90DF90CF900895CF93E1
:10A45000DF93FC01A081B1818681823019F48DEFF8
:10A460009FEF22C0848195818617970728F482E0A8
:10A4700086838EEF9FEF18C0861B970B958384838E
:10A48000828193818617970738F4681B790BED0159
:10A49000888599859383828382819381861B970B1C
:10A4A0009383828380E090E0DF91CF910895CF93F2
:10A4B000DF93DC0190E09D01265F3F4FFD01808925
:10A4C000882369F4ED018C819D81958784878E8135
:10A4D0009F819787868781E0808BC90108C09F5F35
:10A4E0003796295F3F4F933050F380E090E0DF9143
:10A4F000CF910895DC01892B69F0ED91FC911197C2
:10A500003A9682E0EA17FB0709F4168281503796E3
:10A5100087FFF8CF0895DC0122E0FC01922F8089AB
:10A52000813009F4208B9150379697FFF8CFFD01C9
:10A5300015821482178216820895FC01868181306B
:10A5400019F481E090E0089580E090E00895CF92C2
:10A55000DF92EF92FF920F931F93CF93DF937B01D4
:10A560008C016A018FE190E00E94D508FC01E08235
:10A57000F18202831383D186C086158214821782EA
:10A580001682DC0182E0ED01FB87EA87188A8150A0
:10A59000179687FFF8CFCF01DF91CF911F910F91D1
:10A5A000FF90EF90DF90CF9008950F931F93CF937C
:10A5B000DF939C018C010D5F1B4FF801808191811D
:10A5C000CEEFD3E0C81BD90B4C175D0708F4EA01A6
:10A5D000820F931FAE0103960E94097DF8018081CE
:10A5E00091818C0F9D1F91838083CE01DF91CF914C
:10A5F0001F910F910895AC0120E030E0E091B81573
:10A60000F091B915E657FD4F808191818417950728
:10A6100011F4CF0108952F5F3F4FEB5FFB4F2230C6
:10A62000310590F380E090E008959F92AF92BF9241
:10A63000CF92DF92EF92FF920F931F93CF93DF930E
:10A640008C019924CC24DD245601E090B815F090BB
:10A65000B915F501EE0DFF1D83859485892B01F158
:10A66000EF0109900020E9F72197CE1BDF0BAE0127
:10A67000B801C7018C0D9D1D0E94317D892B81F48D
:10A68000FE01E00FF11F80818032A1F0F8010190FE
:10A690000020E9F73197E01BF10BCE17DF0751F0EF
:10A6A00093948DE090E0A80EB91EC80ED91E91E3D8
:10A6B000991558F6C2E39C1619F481E090E023C086
:10A6C000292D33278DE090E0289FD001299FB00DE0
:10A6D000389FB00D1124AE0DBF1DFD01019000206B
:10A6E000E9F73197EA1BFB0B0E0F1F1FF801808162
:10A6F000882311F00F5F1F4FED01EB85FC85C8012A
:10A70000099580E090E0DF91CF911F910F91FF902C
:10A71000EF90DF90CF90BF90AF909F9008950F93F0
:10A720001F93DC01FC0101900020E9F731970E2F07
:10A73000081B043108F003E111278091B8159091AE
:10A74000B915A801BD01805E924F0E943F7DE09146
:10A75000B815F091B915E00FF11FE05EF24F1082CD
:10A760001F910F9108950F931F938C018091B8153D
:10A770009091B9158C5C924F0E94F96C6091BA155A
:10A780007091BB15C8010E94EB1D8091B815909186
:10A79000B9158C5C924F0E94366D1F910F910895F0
:10A7A0008091B8159091B915805E924F0E94B35375
:10A7B0000895EF92FF920F931F93CF93DF93CDB73E
:10A7C000DEB709E010E00C0F1D1FF801E190F190D9
:10A7D0008F018091B8159091B9158C5C924F0E94B1
:10A7E000F96CA801B7018091BA159091BB150E9430
:10A7F0006B758C018091B8159091B9158C5C924F56
:10A800000E94366DC801DF91CF911F910F91FF908B
:10A81000EF900895CF93DF93EB019093BB15809356
:10A82000BA158FE99DE00E94D5089C019093B91557
:10A830008093B815892B49F487EF90E09F938F930D
:10A840000E94D9530F900F902AC0FE010190002062
:10A85000E9F731978E2F8C1B853108F084E1992719
:10A86000AC01BE01C901805E924F0E943F7D809184
:10A87000B8159091B915FC013B9621E31182108225
:10A880003D96215027FFFACF8C5C924F0E94F16CCD
:10A89000E091B815F091B915E65CF24F1082DF91A6
:10A8A000CF910895CF93DF93DC01EB0160E0FC01D1
:10A8B00001900020E9F73197E81BF90B3B9778F0FE
:10A8C0009F938F938CE191E09F938F930E94D95334
:10A8D0000F900F900F900F9080E391E01EC0409179
:10A8E000B8155091B915FA013B96808191813D963A
:10A8F000892B19F06F5F6233C0F36233A9F4BF9301
:10A90000AF9388E491E09F938F930E94D9530F9067
:10A910000F900F900F908CE591E09F938F930E9482
:10A92000D9530F900F9018C0262F33278DE090E059
:10A93000289FF001299FF00D389FF00D1124E40F9E
:10A94000F51FD487C3878DE0689FC0011124BD0126
:10A95000840F951F0E942A7DDF91CF910895EF9279
:10A96000FF920F931F937C01162F8091B815909141
:10A97000B9158C5C924F0E94F96C012F11278091C0
:10A98000BA159091BB150E942F18A801B7010E941B
:10A99000F0198091B8159091B9158C5C924F0E9476
:10A9A000366D1F910F91FF90EF9008950E94D05344
:10A9B000E091B815F091B915E25EF24F9081EE5139
:10A9C000FD4082E8989FC00111248E0F9F1FE15E19
:10A9D000F24F60818C56954F0E94AF5408952F928C
:10A9E0003F924F925F926F927F928F929F92AF921F
:10A9F000BF92CF92DF92EF92FF920F931F93CF936C
:10AA0000DF93CDB7DEB726970FB6F894DEBF0FBE43
:10AA1000CDBF5C01D62E49831B828FEFC82E8B8160
:10AA20008C838A83882499241401240134010091A1
:10AA3000B8151091B915F201E00FF11FFE83ED83F7
:10AA400083859485892B09F46BC08D2D9927780116
:10AA5000E20CF31CAC01B501C7010E94317D892BCA
:10AA600009F05EC0F981FF2361F18FEFC81619F07C
:10AA700091E09C8308C087E791E09F938F930E94A9
:10AA8000D9530F900F908091B8159091B915880DFA
:10AA9000991D0E94B353EB81EF5FEB838E2F65E02E
:10AAA0000E946D7D992319F489E791E002C08BE73C
:10AAB00091E09F938F930E94D9530F900F90CD2CCC
:10AAC0002FC0FFEFCF1681F4ED81FE8101900020B1
:10AAD000E9F73197CE2E8D81C81AB701C5010E94C2
:10AAE0002A7D1EC0C22E1CC091E09C832D2DDC143B
:10AAF000B8F48DE090E0689EF001699EF00D789EBC
:10AB0000F00D1124E00FF11FED0DF11DD501AD0D7C
:10AB1000B11D9D918191981729F72F5F2C15C8F3CE
:10AB2000EA81EF5FEA830894611C711C8DE090E07C
:10AB3000480E591E280E391E880E991EE23308F45D
:10AB400076CF9FEFC91619F48D2D992725C0EC817A
:10AB5000EE2331F4F501EC0DF11D80E28083C39406
:10AB6000F981FF2379F08DE791E09F938F930E9405
:10AB7000D9530E94D0536C2DC5010E94AF540F9041
:10AB80000F9008C08C2D8D19682FC5018D0D911D5A
:10AB90000E94AF548C2D992726960FB6F894DEBFED
:10ABA0000FBECDBFDF91CF911F910F91FF90EF901E
:10ABB000DF90CF90BF90AF909F908F907F906F90DD
:10ABC0005F904F903F902F900895AF92BF92CF9299
:10ABD000DF92EF92FF920F931F93CF93DF93CDB746
:10ABE000DEB723970FB6F894DEBF0FBECDBFCC24DF
:10ABF000AC2CBC2C86E90E9406080E94D654809199
:10AC0000BA159091BB150E942F1841E050E0BE018B
:10AC1000640F751F0E94F6727C018FEFE81639F4FD
:10AC20008FE791E09F938F930E94D953F8C191E0F1
:10AC3000E91629F78091BA159091BB150E942F183B
:10AC40000E94817B882369F099279F938F938DEAD7
:10AC500091E09F938F930E94D9530F900F900F9084
:10AC60000F9099819B3109F0CDC0BB24DB2C8D2D39
:10AC7000992787FD9095E2E0EE2EF12CE81AF90A6B
:10AC80008E010F5F1F4F080F191F8091BA15909109
:10AC9000BB150E942F18A701B8010E94F672D80EAA
:10ACA000A1E0AD1524F789818B35A1F58A81813426
:10ACB000D1F4E091B815F091B915E25EF24F8081C0
:10ACC00099272C2D3327821B930B059665E070E0A6
:10ACD0000E94797D0497F1F0AA2011F4CC20D1F0E4
:10ACE000C90104960EC0E091B815F091B9158234EF
:10ACF00071F4E25EF24F8081C81661F08C2D9927C5
:10AD0000019665E070E00E94797DC82E03C0E25E86
:10AD1000F24FC080E091B815F091B915E15EF24FA5
:10AD200080818823F1F0E091B815F091B915E15ECA
:10AD3000F24F80818150808388E090E09F938F93D1
:10AD40009F938F9382EC91E09F938F930E94D953AE
:10AD5000EDB7FEB736960FB6F894FEBF0FBEEDBF47
:10AD6000D9CFE091B815F091B915E25EF24F90811C
:10AD7000EE51FD40C91609F442CF82E8C89E800119
:10AD800011249F01200F311F2C56354F989FC00171
:10AD90001124E80FF91F42E850E0B901CF018C56A9
:10ADA000954F0E943F7D8091B8159091B915800F05
:10ADB000911F8C56954F0E94B3532091B815309136
:10ADC000B915225E324FD9018C912E513D40992701
:10ADD000FC01F695FE2FEE27F795E795E80FF91F92
:10ADE000E80FF91FE20FF31FEC56F54FDF010D904E
:10ADF0000020E9F71197AE1BBF0B215E324FF9011E
:10AE0000A083FDCE9A3019F09D3009F091C0BB248B
:10AE1000A091B815B091B915A15EB24F2C918E9149
:10AE2000AE51BD409927FC01F695FE2FEE27F79510
:10AE3000E795E80FF91FE80FF91FE20FF11DEA0F80
:10AE4000FB1FEC56F54FB08288EC91E09F938F93F7
:10AE50000E94D953E091B815F091B915E15EF24F17
:10AE60000F900F908081EF51FD40882309F45DC061
:10AE7000E25EF24F90818F010E511D4082E8989F53
:10AE8000C0011124080F191F0C56154FC8010E944C
:10AE90001553882361F01F930F938AEC91E09F93E1
:10AEA0008F930E94D9530F900F900F900F90E091C5
:10AEB000B815F091B915E25EF24F80818F5F808303
:10AEC000E091B815F091B915E25EF24F80818530BE
:10AED00011F4B082AE2CE091B815F091B915E25E94
:10AEE000F24FC190B08220E030E0A091B815B0914F
:10AEF000B915A25EB24F8C91AE51BD409927FC01AD
:10AF0000F695FE2FEE27F795E795E80FF91FE80F66
:10AF1000F91FE20FF31FEA0FFB1FEC56F54F1082EB
:10AF20002F5F3F4F2238310504F30E94D05367CE84
:10AF3000983019F09F3709F045C0BB24E091B8154F
:10AF4000F091B915E15EF24F8081882309F457CE64
:10AF500088E090E09F938F939F938F9381EE91E091
:10AF60009F938F930E94D953E091B815F091B91532
:10AF7000E15EF24F808181508083A091B815B0913D
:10AF8000B915A15EB24F2C918E91AE51BD4099275B
:10AF9000FC01F695FE2FEE27F795E795E80FF91FD0
:10AFA000E80FF91FE20FF11DEA0FFB1FEC56F54FFA
:10AFB000B0828DB79EB706960FB6F8949EBF0FBEAF
:10AFC0008DBF1DCEE091B815F091B9159930D1F42F
:10AFD0008F01015E124FE25EF24F9081EE51FD4013
:10AFE00082E8989FC0011124E80FF91F4B2DD8016A
:10AFF0006C91CF018C56954F0E94EF54F8018083DD
:10B00000B394FDCDE15EF24F80818F3759F487EE26
:10B0100091E09F938F930E94D9530E94D6540F9032
:10B020000F90EDCDBB24892F99279F938F938AEFA3
:10B0300091E09F938F930E94D953A091B815B0913E
:10B04000B915A15EB24F2C918E91AE51BD4099279A
:10B05000FC01F695FE2FEE27F795E795E80FF91F0F
:10B06000E80FF91FE20FF11DEA0FFB1FEC56F54F39
:10B0700089818083E091B815F091B915E15EF24FB6
:10B0800080818F5F80830F900F900F900F90B7CDCE
:10B090009B01882359F420503C4F40E050E069E583
:10B0A00078E58AE595E00E944E0B08950E94E555EB
:10B0B00008950E94E555FFCF8091B8159091B9157C
:10B0C0008C5C924F0E94F96C08958091B815909114
:10B0D000B9158C5C924F0E94366D08950F931F93A3
:10B0E000CF93DF93CDB7DEB70F811885809184159C
:10B0F000909185150E94FB52FC01892B61F08281A1
:10B10000882349F09E01275F3F4FA801BF0185EDCD
:10B1100092E50E943B1A0E945C58AE01475F5F4F68
:10B12000B8018091BA159091BB150E9440198C010D
:10B130000E946558C801DF91CF911F910F9108952A
:10B1400080E090E00E94FB52FC01892B69F0809125
:10B1500084159091851591838083ED5FFB4F11825B
:10B16000108280E090E0089581E090E00895809161
:10B170008415909185150E94FB52FC01892B49F0A2
:10B1800081E08283ED5FFB4F1182108280E090E0CE
:10B19000089581E090E0089580918415909185153F
:10B1A0000E94FB52DC01009779F0AD5FBB4FED913F
:10B1B000FC911197A350B440EA0FFB1F1382FD01CD
:10B1C0001282CD01039608950895E091B815F0918B
:10B1D000B915E256F24F24E641E0608182E00E9418
:10B1E0000C4C8091B8159091B915865C924F0E94D5
:10B1F000B35308950F931F93CF93DB01E091B815DC
:10B20000F091B915E65CF24FC081EA53FD40CC23C2
:10B2100019F5E256F24F8083FB0101900020E9F717
:10B2200031970E2F061B043608F003E61127809194
:10B23000B8159091B915A801BD01865C924F0E9486
:10B240003F7DE091B815F091B915E00FF11FE65C74
:10B25000F24FC0830E94E558CF911F910F9108953E
:10B26000FC01808199279F938F93818199279F93D8
:10B270008F93828199279F938F93838199279F939F
:10B280008F93848199279F938F93858199279F938B
:10B290008F9385E695E09F938F930E946E588DB7AC
:10B2A0009EB70E960FB6F8949EBF0FBE8DBF089541
:10B2B0000F931F93CF93DF93E091BC15F091BD15D1
:10B2C000EE55FF4F8081992787FD90959F938F932F
:10B2D00083E895E09F938F930E946E58E091BC1590
:10B2E000F091BD15EE55FF4F80810F900F900F909C
:10B2F0000F9087FF02C0108208C080E995E09F93FD
:10B300008F930E946E580F900F90E091BC15F091B2
:10B31000BD15EE55FF4F808100E010E018160CF0CF
:10B3200048C0E8011F930F9388EB95E09F938F939C
:10B330000E946E588091BC159091BD158C0F9D1F79
:10B340000E943059E091BC15F091BD15EC0FFD1F26
:10B35000858596859F938F93E091BC15F091BD15DF
:10B36000EC0FFD1F87819085A185B285BF93AF93B8
:10B370009F938F938FEB95E09F938F930E946E58CE
:10B380008DB79EB70C960FB6F8949EBF0FBE8DBFBB
:10B390000F5F1F4F2F96E091BC15F091BD15EE5534
:10B3A000FF4F8081992787FD9095081719070CF4A6
:10B3B000B9CFDF91CF911F910F9108958CEC95E05B
:10B3C0009F938F930E946E5886E796E09F938F938A
:10B3D0000E946E580F900F900F900F900895CF938A
:10B3E000DF93CDB7DEB724970FB6F894DEBF0FBE5C
:10B3F000CDBF9E012F5F3F4F3F932F939E012D5F47
:10B400003F4F3F932F9324EE36E03F932F939F932C
:10B410008F930E94A7722DB73EB7285F3F4F0FB69C
:10B42000F8943EBF0FBE2DBF029709F04EC08B812E
:10B430009C819F938F9389EE96E09F938F930E94B8
:10B440006E5829813A8180E496E0289FA001299FC7
:10B45000500D389F500D1124E091BC15F091BD1591
:10B46000EB53FF4F9A014B815C8160E070E080817B
:10B4700091810E94B0250F900F900F900F9097FF31
:10B480001BC022273327A901261B370B480B590B5A
:10B490005F934F933F932F938CE097E09F938F930D
:10B4A0000E946E584DB75EB74A5F5F4F0FB6F89473
:10B4B0005EBF0FBE4DBF0BC082E297E09F938F939C
:10B4C0000E946E580F900F9002C00E94DE59249681
:10B4D0000FB6F894DEBF0FBECDBFDF91CF910895B8
:10B4E000CF92DF92EF92FF920F931F93CF93DF9350
:10B4F000CDB7DEB722970FB6F894DEBF0FBECDBF33
:10B500008C0195E0E92EF12CFA82E98244E050E0CA
:10B5100066E377E0C8010E94317D6C01892B09F058
:10B520004DC0CE0101969F938F938BE397E09F933D
:10B530008F930C5F1F4F1F930F930E94A772E09190
:10B54000BC15F091BD15ED55FF4F89818083E091C9
:10B55000BC15F091BD15ED55FF4F8081992787FDF2
:10B5600090959F938F938EE397E09F938F930E9484
:10B570006E58E091BC15F091BD1582EAE82EF12CD1
:10B58000EE0EFF1EDF01AB53BF4F8F012AE0ED55DA
:10B59000FF4F4081B6018D919C910E943844DC019F
:10B5A000CB01F70180830E9458598DB79EB70A9648
:10B5B0000FB6F8949EBF0FBE8DBFCAC0A70161E64B
:10B5C00077E0C8010E94317D892B09F04DC0E091E0
:10B5D000BC15F091BD15EC55FF4F8081813019F4F9
:10B5E00087E697E0AFC0CE0101969F938F938BE3E0
:10B5F00097E09F938F930B5F1F4F1F930F930E94B2
:10B60000A772E091BC15F091BD15ED55FF4F8981F2
:10B6100080838FE897E09F938F930E946E58E0910C
:10B62000BC15F091BD15CF018A569F4FDF01AB537A
:10B63000BF4F8F012AE0ED55FF4F4081BC018D9136
:10B640009C910E943844E091BC15F091BD15EC55D9
:10B65000FF4F81E08083EDB7FEB738960FB6F894C0
:10B66000FEBF0FBEEDBF74C044E050E061EE77E076
:10B67000C8010E94317D892BC1F4E091BC15F09185
:10B68000BD15EC55FF4F8081E45AF040882319F135
:10B69000E056FF4F808191818F5F9F4F19F487EEB5
:10B6A00097E050C086EF97E04DC044E050E06EE078
:10B6B00078E0C8010E94317D892B09F041C00091DA
:10B6C000BC151091BD150C551F4FF8018081045A0F
:10B6D0001040882319F485E198E034C00D551F4FC0
:10B6E000F8018081992787FD9095A92FB92FBC017A
:10B6F000CD0128EE33E040E050E00E944E7DDC01B9
:10B70000CB01AC01BD01C80103970E94F009E09193
:10B71000BC15F091BD15E656FF4F808138968083A9
:10B7200087EE97E09F938F930E946E580E9458591E
:10B73000E091BC15F091BD15EC55FF4F108206C08D
:10B740008CE398E09F938F930E946E580F900F9018
:10B7500022960FB6F894DEBF0FBECDBFDF91CF911A
:10B760001F910F91FF90EF90DF90CF900895EF928F
:10B77000FF920F931F93CF93DF93CDB7DEB7A897B8
:10B780000FB6F894DEBF0FBECDBF8C018FEF9FEFD9
:10B7900098A78FA39EA38DA38091BC159091BD15F2
:10B7A0008B559F4F9F938F938091BC159091BD15A2
:10B7B00089559F4F9F938F938091BC159091BD1594
:10B7C00087559F4F9F938F938091BC159091BD1586
:10B7D00085559F4F9F938F938091BC159091BD1578
:10B7E00083559F4F9F938F938091BC159091BD156A
:10B7F00081559F4F9F938F938CEA98E09F938F93EF
:10B800001F930F930E94A7722DB73EB7205F3F4F43
:10B810000FB6F8943EBF0FBE2DBF069771F1CE0153
:10B8200085969F938F9384EC98E09F938F931F93BB
:10B830000F930E94A772EDB7FEB736960FB6F89435
:10B84000FEBF0FBEEDBF0197C1F0CE0187969F935B
:10B850008F938BE397E09F938F931F930F930E9497
:10B86000A7722DB73EB72A5F3F4F0FB6F8943EBF81
:10B870000FBE2DBF019709F0F9C02091BC15309182
:10B88000BD152E553F4FF9018081225A304099272E
:10B8900087FD90954FA158A5481759074CF088ECA3
:10B8A00098E09F938F930E946E580E945859E4C06D
:10B8B0004F5F5F4F09F00CF43EC08FEE98E09F930E
:10B8C0008F930E946E582FA138A5C90154E0880FAC
:10B8D000991F5A95E1F7821B930B2091BC1530916B
:10B8E000BD15820F931F0E94305981E099E09F930C
:10B8F0008F930E946E58A091BC15B091BD158FA179
:10B9000098A5FC0144E0EE0FFF1F4A95E1F7E81B04
:10B91000F90BEA0FFB1F86818F70AB53BF4F3EE1DF
:10B92000E32E8E01095F1F4F282F43855485BF01E9
:10B930008D919C9160C06DA17EA18FEF6F3F7807C4
:10B94000E9F0E4F02B533F4FAE014F5F5F4FF90139
:10B95000808191810E94CE2DDC01CB018D5F9E4FB5
:10B96000AF4FBF4F29F58DA19EA19F938F9383E089
:10B9700099E09F938F930E946E5873C018A61FA2E0
:10B98000A0E0B0E0AE014F5F5F4FFD01E40FF51F97
:10B99000AA0FBB1FA20FB31FAB55BF4F8C91808363
:10B9A0008FA198A5019698A78FA3DC0106976CF349
:10B9B0008FEE98E09F938F930E946E58CE01019670
:10B9C0000E94305981E099E09F938F930E946E58B6
:10B9D000E091BC15F091BD15EB53FF4F2EE1E22E27
:10B9E0008E01095F1F4F20E040E050E0BE016F5F15
:10B9F0007F4F808191810E9497487B018C010F903D
:10BA00000F900F900F9097FF1BC088279927DC019C
:10BA10008E199F09A00BB10BBF93AF939F938F9388
:10BA200088E299E09F938F930E946E582DB73EB79E
:10BA30002A5F3F4F0FB6F8943EBF0FBE2DBF1EC00A
:10BA40008DE399E09F938F930E946E586E2DCE01E7
:10BA500007960E94AF548BE499E09F938F930E94C6
:10BA60006E580F900F900F900F9008C08EE499E0E1
:10BA70009F938F930E946E580F900F90A8960FB6C9
:10BA8000F894DEBF0FBECDBFDF91CF911F910F9114
:10BA9000FF90EF900895CF92EF92FF920F93CF9384
:10BAA000DF93CDB7DEB728970FB6F894DEBF0FBE91
:10BAB000CDBF7C018FEF9FEF98878F838091BC155E
:10BAC0009091BD158B559F4F9F938F938091BC157F
:10BAD0009091BD1589559F4F9F938F938091BC1571
:10BAE0009091BD1587559F4F9F938F938091BC1563
:10BAF0009091BD1585559F4F9F938F938091BC1555
:10BB00009091BD1583559F4F9F938F938091BC1546
:10BB10009091BD1581559F4F9F938F938CEA98E02C
:10BB20009F938F93FF92EF920E94A7722DB73EB71B
:10BB3000205F3F4F0FB6F8943EBF0FBE2DBF069754
:10BB4000C1F0CE0107969F938F938BE397E09F936D
:10BB50008F93FF92EF920E94A7724DB75EB74A5F34
:10BB60005F4F0FB6F8945EBF0FBE4DBF019709F04F
:10BB7000D0C0E091BC15F091BD15EE55FF4F80810E
:10BB8000282F332727FD30958F81988582179307BB
:10BB90005CF081EA99E09F938F930E946E580E9417
:10BBA00058590F900F90B7C086EC99E09F938F93F0
:10BBB0000E946E582F8138850F900F905FEF2F3FB6
:10BBC0003507C1F1BCF1C90144E0880F991F4A95BE
:10BBD000E1F7821B930B2091BC153091BD15820FAC
:10BBE000931F0E94305981E099E09F938F930E94A8
:10BBF0006E58A091BC15B091BD158F819885FC0140
:10BC000004E0EE0FFF1F0A95E1F7E81BF90BEA0FBE
:10BC1000FB1F86818F70AB53BF4F71E0C72EE3844B
:10BC2000F484082F28E134E0AF0160E070E08D91EA
:10BC30009C913BC018861F82A0E0B0E0AE014F5F30
:10BC40005F4F2091BC153091BD15FD01E40FF51F2C
:10BC5000AA0FBB1FA20FB31FAB55BF4F8C918083A0
:10BC60008F819885019698878F83DC0106976CF306
:10BC7000CE0101960E94305981E099E09F938F9305
:10BC80000E946E58E091BC15F091BD15EB53FF4F2B
:10BC900061E0C62EEE24FF2400E028E134E0AE018E
:10BCA0004F5F5F4FB701808191810E94E5440F9003
:10BCB0000F9097FF1BC022273327A901261B370BA4
:10BCC000480B590B5F934F933F932F9383ED99E06C
:10BCD0009F938F930E946E584DB75EB74A5F5F4F38
:10BCE0000FB6F8945EBF0FBE4DBF15C09F938F93E4
:10BCF0007F936F9386EE99E09F938F930E946E5887
:10BD00008DB79EB706960FB6F8949EBF0FBE8DBF37
:10BD100002C00E94DE5928960FB6F894DEBF0FBE0F
:10BD2000CDBFDF91CF910F91FF90EF90CF9008950D
:10BD3000CF93DF93CDB7DEB728970FB6F894DEBF69
:10BD40000FBECDBF9E01295F3F4F3F932F932BE343
:10BD500037E03F932F939F938F930E94A7722DB745
:10BD60003EB72A5F3F4F0FB6F8943EBF0FBE2DBFC0
:10BD7000019709F076C0E091BC15F091BD15EB5329
:10BD8000FF4F6F817885808191810E94F42DDC01C5
:10BD9000CB010097A105B10539F08F8198859F935C
:10BDA0008F938BEF99E04BC0E091BC15F091BD15DE
:10BDB000EB53FF4FAE014F5F5F4F6F8178858081FE
:10BDC00091810E94CE2DDC01CB010097A105B10528
:10BDD00039F08F8198859F938F9381E29AE02FC0ED
:10BDE00081E59AE09F938F930E946E58CE01019651
:10BDF0000E94305981E099E09F938F930E946E5882
:10BE0000E091BC15F091BD15EB53FF4F23E14F813D
:10BE1000588560E070E0808191810E945046DC018D
:10BE2000CB010F900F900F900F900097A105B105D7
:10BE300079F08F8198859F938F9387E69AE09F93FF
:10BE40008F930E946E580F900F900F900F900BC021
:10BE500083EA9AE09F938F930E946E580F900F9001
:10BE600002C00E94DE5928960FB6F894DEBF0FBEBE
:10BE7000CDBFDF91CF910895CF93DF93CDB7DEB7DC
:10BE800024970FB6F894DEBF0FBECDBF9E012F5F83
:10BE90003F4F3F932F939E012D5F3F4F3F932F9333
:10BEA00024EE36E03F932F939F938F930E94A772C7
:10BEB0002DB73EB7285F3F4F0FB6F8943EBF0FBE79
:10BEC0002DBF029709F051C0E091BC15F091BD154E
:10BED000EB53FF4F29814B815C8160E070E08081F2
:10BEE00091810E944C2997FF1BC022273327A9016B
:10BEF000261B370B480B590B5F934F933F932F93A0
:10BF000082EB9AE09F938F930E946E584DB75EB775
:10BF10004A5F5F4F0FB6F8945EBF0FBE4DBF2DC096
:10BF20008B819C819F938F9385ED9AE09F938F9354
:10BF30000E946E58E091BC15F091BD15EB53FF4F78
:10BF40006B817C81808191810E94072D0F900F90E1
:10BF50000F900F90611571058105910519F484EF1B
:10BF60009AE005C08CEF9AE002C083E09BE09F93CB
:10BF70008F930E946E580F900F9024960FB6F894EE
:10BF8000DEBF0FBECDBFDF91CF910895CF93DF937A
:10BF9000CDB7DEB722970FB6F894DEBF0FBECDBF88
:10BFA0009E012F5F3F4F3F932F932BE337E03F934B
:10BFB0002F939F938F930E94A7722DB73EB72A5F4E
:10BFC0003F4F0FB6F8943EBF0FBE2DBF019761F5EE
:10BFD00089819A819F938F938FE39BE09F938F93A7
:10BFE0000E946E58E091BC15F091BD15EB53FF4FC8
:10BFF00069817A81808191810E94072DDC01CB01CA
:10C000000F900F900F900F900097A105B10519F4B4
:10C0100084EF9AE002C08CEF9AE09F938F930E9486
:10C020006E580F900F9002C00E94DE5922960FB6F4
:10C03000F894DEBF0FBECDBFDF91CF910895CF93AF
:10C04000DF93CDB7DEB722970FB6F894DEBF0FBEF1
:10C05000CDBF9E012F5F3F4F3F932F932BE337E0E0
:10C060003F932F939F938F930E94A7722DB73EB754
:10C070002A5F3F4F0FB6F8943EBF0FBE2DBF01970A
:10C0800021F489818093271402C00E94DE592296F0
:10C090000FB6F894DEBF0FBECDBFDF91CF910895EC
:10C0A000EF92FF920F931F93CF93DF93E091BC1514
:10C0B000F091BD15EB53FF4F0081118181E69BE0AC
:10C0C0009F938F930E946E580F900F905DE7E52E1F
:10C0D00052E0F52EE00EF11EE801C758DD4F09E0F1
:10C0E000888199819F938F938EE89BE09F938F9394
:10C0F0000E946E588A819B819F938F9382E99BE077
:10C100009F938F930E946E58C7010E94305989896E
:10C1100099279F938F9388E99BE09F938F930E9429
:10C120006E58888982958F70837099279F938F931B
:10C130008EE99BE09F938F930E9405198DB79EB760
:10C1400040960FB6F8949EBF0FBE8DBF8A8999277F
:10C150008130910579F0823091051CF4892B39F0FA
:10C1600012C08230910549F0039751F00CC082EA69
:10C170009BE00BC08AEA9BE008C080EB9BE005C017
:10C1800087EB9BE002C08DEB9BE09F938F930E9417
:10C190006E580F900F9081E099E09F938F930E94CB
:10C1A0006E580F900F900150679687E190E0E80E6F
:10C1B000F91E07FF95CFDF91CF911F910F91FF904F
:10C1C000EF9008950F931F93CF93DF93CDB7DEB712
:10C1D0006E970FB6F894DEBF0FBECDBF8C0143E063
:10C1E00050E066EC7BE00E94317DBC01892BC9F4F4
:10C1F0000C5F1F4FE091BC15F091BD15EB53FF4F45
:10C20000A801808191810E948C20DC01CB010097E4
:10C21000A105B10519F08AEC9BE035C085EE9BE0E5
:10C2200032C043E050E066EF7BE0C8010E94317D00
:10C23000BC01892B31F5E091BC15F091BD15EB5394
:10C24000FF4F2EE1AE014F5F5F4F808191810E94D1
:10C250001821DC01CB010097A105B10519F08AEF87
:10C260009BE011C0CE0101969F938F9384E19CE0E7
:10C270009F938F930E946E580F900F900F900F9086
:10C2800008C086E29CE09F938F930E946E580F90A7
:10C290000F906E960FB6F894DEBF0FBECDBFDF9144
:10C2A000CF911F910F910895EF92FF920F931F93DB
:10C2B000CF93DF93CDB7DEB724970FB6F894DEBFE8
:10C2C0000FBECDBF8C0143E050E066EC7BE00E94E6
:10C2D000317D7C01892BB9F5CE0101969F938F9317
:10C2E00086E59CE09F938F930C5F1F4F1F930F93E6
:10C2F0000E94A7722DB73EB72A5F3F4F0FB6F89442
:10C300003EBF0FBE2DBF0197D9F4E091BC15F0914F
:10C31000BD15EB53FF4F29813A814B815C81B701F9
:10C32000808191810E949B23DC01CB010097A105B4
:10C33000B10519F08AE59CE035C084E79CE032C085
:10C3400084E89CE02FC043E050E066EF7BE0C8014A
:10C350000E94317DBC01892B19F5E091BC15F0914B
:10C36000BD15EB53FF4F808191810E945A23DC0160
:10C37000CB0189839A83AB83BC83BF93AF939F9395
:10C380008F9383EB9CE09F938F930E946E588DB7A1
:10C390009EB706960FB6F8949EBF0FBE8DBF08C01D
:10C3A00087EC9CE09F938F930E946E580F900F90A4
:10C3B00024960FB6F894DEBF0FBECDBFDF91CF91AC
:10C3C0001F910F91FF90EF90089585EF9CE09F9350
:10C3D0008F930E946E58E091BC15F091BD15EB5300
:10C3E000FF4F808191818A599C4F0E94305981E092
:10C3F00099E09F938F930E946E580F900F900F902B
:10C400000F900895CF93DF93CDB7DEB728970FB67F
:10C41000F894DEBF0FBECDBFE091BC15F091BD1505
:10C42000EB53FF4FAE014F5F5F4F60E070E08081E4
:10C4300091810E9452278F8198859F938F938D8140
:10C440009E819F938F938C8199279F938F938A814D
:10C450009B819F938F93898199279F938F9385E0E9
:10C460009DE09F938F930E946E588DB79EB70C9658
:10C470000FB6F8949EBF0FBE8DBF28960FB6F894E6
:10C48000DEBF0FBECDBFDF91CF910895CF93DF9375
:10C49000CDB7DEB728970FB6F894DEBF0FBECDBF7D
:10C4A000E091BC15F091BD15EB53FF4FAE014F5F0E
:10C4B0005F4F60E070E0808191810E94E027888575
:10C4C00099279F938F938F8199279F938F938E8125
:10C4D00099279F938F938D8199279F938F938C8119
:10C4E00099279F938F938B8199279F938F938A810D
:10C4F00099279F938F93898199279F938F9383E3A4
:10C500009DE09F938F930E946E588DB79EB7429681
:10C510000FB6F8949EBF0FBE8DBF28960FB6F89445
:10C52000DEBF0FBECDBFDF91CF9108950F931F9354
:10C530008C0187EC90E00E94D508FC019093BD151A
:10C540008093BC15ED55FF4F85E08083E091BC15CD
:10C55000F091BD15EB53FF4F118300831F910F9195
:10C560000895CF93DF93EC0144E050E06AE77DE06B
:10C570000E94317D892B19F40E94E561B2C048E028
:10C5800050E06FE77DE0CE010E94317D892B19F4E8
:10C590000E945060A6C049E050E068E87DE0CE010E
:10C5A0000E94317D892B29F4CE010A960E941F60DA
:10C5B00098C049E050E062E97DE0CE010E94317D03
:10C5C000892B29F4CE010A960E94EF598AC043E0D4
:10C5D00050E06CE97DE0CE010E94317D892B29F489
:10C5E000CE0104960E944B5D7CC046E050E060EABC
:10C5F0007DE0CE010E94317D892B29F4CE01079682
:10C600000E94985E6EC047E050E067EA7DE0CE0190
:10C610000E94317D892B29F4CE0108960E94705A20
:10C6200060C044E050E06FEA7DE0CE010E94317DC1
:10C63000892B29F4CE0105960E94E26052C043E0A6
:10C6400050E064EB7DE0CE010E94317D892B29F41E
:10C65000CE0104960E94546144C045E050E068EB6E
:10C660007DE0CE010E94317D892B29F4CE01069612
:10C670000E94B75B36C047E050E06EEB7DE0CE0134
:10C680000E94317D892B29F4CE0108960E943C5FDF
:10C6900028C044E050E066EC7DE0CE010E94317D90
:10C6A000892B29F4CE0105960E94C65F1AC048E086
:10C6B00050E06BEC7DE0CE010E94317D892B19F4B6
:10C6C0000E9446620EC047E050E064ED7DE0CE017E
:10C6D0000E94317D892B19F40E94026202C00E94DF
:10C6E000DE59DF91CF91089561EB72E68CED9DE00C
:10C6F0000E94525408958AE090E00E94CD759C01FA
:10C70000E8EEF3E0BF010E94797D6AE070E00E94EC
:10C71000797D7F936F93C901BF010E94797D7F93DB
:10C720006F938FED9DE09F938F930E946E588DB70E
:10C730009EB706960FB6F8949EBF0FBE8DBF0895A4
:10C74000AF92BF92CF92DF92EF92FF920F931F931F
:10C75000CF93DF93CDB7DEB72A970FB6F894DEBF3D
:10C760000FBECDBF8C011A8219825E010894A11CF4
:10C77000B11CBF92AF92CE0103969F938F9395E029
:10C78000C92ED12CCC0EDD1EDF92CF92CE010796A2
:10C790009F938F938CEF9DE09F938F931F930F93A5
:10C7A0000E94A7722DB73EB7245F3F4F0FB6F89493
:10C7B0003EBF0FBE2DBF03973CF02D814F81698195
:10C7C0008B810E940C4C6AC04AE050E06CE07EE035
:10C7D000C8010E94317D892B19F40E94274E5EC04A
:10C7E00089E0E82EF12CEC0EFD1EFF92EF9287E11E
:10C7F0009EE09F938F931F930F930E94A7722DB774
:10C800003EB72A5F3F4F0FB6F8943EBF0FBE2DBF15
:10C81000019721F489850E944D4E40C0FF92EF920E
:10C820008CE19EE09F938F931F930F930E94A772BA
:10C830002DB73EB72A5F3F4F0FB6F8943EBF0FBEED
:10C840002DBF019721F489850E94644E27C0DF9295
:10C85000CF92FF92EF92BF92AF9282E29EE09F93BF
:10C860008F931F930F930E94A7722DB73EB7265F39
:10C870003F4F0FB6F8943EBF0FBE2DBF039731F464
:10C880004D81698589810E94304E08C08BE29EE00F
:10C890009F938F930E946E580F900F902A960FB619
:10C8A000F894DEBF0FBECDBFDF91CF911F910F91E6
:10C8B000FF90EF90DF90CF90BF90AF90089560EA27
:10C8C00073E685EC9EE00E9452546BE773E689ECB8
:10C8D0009EE00E94525408958DEF91E09F938F93B4
:10C8E0000E94D9530F900F900895CF93DF93EC01DE
:10C8F00047E050E06DEC7EE00E94317D892B39F4F9
:10C900008091BA159091BB150E94456B2AC046E0F4
:10C9100050E065ED7EE0CE010E94317D892B39F437
:10C920008091BA159091BB150E94E06B1AC044E04B
:10C9300050E06CED7EE0CE010E94317D892B79F4D0
:10C940000E946F099F938F9384E392E09F938F934C
:10C950000E94D9530F900F900F900F9002C00E9429
:10C960006C64DF91CF91089565E774E681EE9EE0F7
:10C970000E9452540895EF92FF920F931F937C01EF
:10C980008B010E945C58F8018381E82FFF27EE0F8E
:10C99000FF1FEB51F14F808191819F938F93F8019D
:10C9A000828199279F938F9384819581A681B781F6
:10C9B000BF93AF939F938F93808191819F938F9328
:10C9C00087E09FE09F938F938091BE159091BF1554
:10C9D0009F938F930E948F726091BE157091BF15C7
:10C9E000C7010E94EB1D0E9465588DB79EB70E9639
:10C9F0000FB6F8949EBF0FBE8DBF1F910F91FF9091
:10CA0000EF9008958BE19FE09F938F930E946E5863
:10CA100087E29FE09F938F930E946E588BE49FE084
:10CA20009F938F930E946E588CE79FE09F938F9304
:10CA30000E946E5883E89FE09F938F930E946E58E8
:10CA40008DE99FE09F938F930E946E588BEA9FE041
:10CA50009F938F930E946E5887EC9FE09F938F93D4
:10CA60000E946E5888ED9FE09F938F930E946E58AE
:10CA70008AEE9FE09F938F930E946E588DB79EB76A
:10CA800044960FB6F8949EBF0FBE8DBF08950F93C6
:10CA90001F93CF93DF93CDB7DEB724970FB6F894EB
:10CAA000DEBF0FBECDBF8C011C821B828FEF90E0DA
:10CAB0009A83898342E050E069EF7FE0C8010E94D9
:10CAC000317DBC01892B71F440EC55E18BEB94E690
:10CAD0000E94D450892B19F48CEF9FE02CC08BE07E
:10CAE00090E129C044E050E063E370E1C8010E9496
:10CAF000317D892B29F40E94EB5087E390E11BC024
:10CB000043E050E067E470E1C8010E94317D892B69
:10CB100029F40E94F8508DE490E10DC045E050E00A
:10CB200060E670E1C8010E94317D892B59F40E94B2
:10CB3000FC5087E690E19F938F930E946E580F9070
:10CB40000F9054C0CE0101969F938F93CE01039610
:10CB50009F938F938BE790E19F938F931F930F93F6
:10CB60000E94A7722DB73EB7285F3F4F0FB6F894CB
:10CB70003EBF0FBE2DBF82309105A1F4EB81FC8139
:10CB8000CF0101974F9728F4E254FA4E89818283AE
:10CB90000CC080E890E19F938F930E946E580F9095
:10CBA0000F9003C018161906FCF4EB81FC81CF012D
:10CBB00001974F97C8F4E254FA4E828199279F93C8
:10CBC0008F938B819C819F938F9389E990E19F93B1
:10CBD0008F930E946E588DB79EB706960FB6F89445
:10CBE0009EBF0FBE8DBF02C00E94026524960FB685
:10CBF000F894DEBF0FBECDBFDF91CF911F910F9193
:10CC00000895EF92FF920F931F93CF93DF93CDB7C9
:10CC1000DEB728970FB6F894DEBF0FBECDBF8C01EC
:10CC20001C821B828FEF90E09A8389831E821D8273
:10CC300018861F8244E050E064EC70E1C8010E9455
:10CC4000317D7C01892B49F5CE0101969F938F930D
:10CC5000CE0103969F938F93CE0105969F938F935A
:10CC600089EC90E19F938F930C5F1F4F1F930F935D
:10CC70000E94A77287012BEB34E649816B818D817D
:10CC80009E810E942C4F2DB73EB7265F3F4F0FB6B7
:10CC9000F8943EBF0FBE2DBFA4C043E050E060ED4E
:10CCA00070E1C8010E94317D7C01892B61F5CE01C4
:10CCB00001969F938F93CE0103969F938F93CE01FE
:10CCC00005969F938F93CE0107969F938F9384ED44
:10CCD00090E19F938F930D5F1F4F1F930F930E94BF
:10CCE000A77297014BEB54E66D817E818F81988509
:10CCF0000E94A44F8DB79EB70C960FB6F8949EBFB6
:10CD00000FBE8DBF6EC045E050E06DED70E1C80113
:10CD10000E94317D892B19F40E94254F62C047E0A3
:10CD200050E063EE70E1C8010E94317D892B09F06B
:10CD300048C0CE0101969F938F93CE0103969F9397
:10CD40008F938BE790E19F938F93095F1F4F1F9302
:10CD50000F930E94A7722DB73EB7285F3F4F0FB6C3
:10CD6000F8943EBF0FBE2DBF8230910529F4698132
:10CD70008B810E94245003C01816190684F58B81FC
:10CD80000E9417509A8389838B819C819F938F93F4
:10CD90008BEE90E19F938F930E946E580F900F90AF
:10CDA0000F900F9089819A819F938F938AEF90E1E2
:10CDB0009F938F930E946E580F900F900F900F903B
:10CDC00010C049E050E061E171E1C8010E94317D8D
:10CDD000892B29F4C8010A960E94476502C00E9467
:10CDE000026528960FB6F894DEBF0FBECDBFDF9167
:10CDF000CF911F910F91FF90EF90089540EC55E176
:10CE000060E070E08BEB94E60E94D4500895E82F28
:10CE100081508F3138F4FF27E254FA4E628380E06C
:10CE200090E008958FEF9FEF08959093BF15809342
:10CE3000BE15E0ECF5E1119285E1EF3DF807D9F37D
:10CE4000D0F361E076E68BE191E10E9452540895BF
:10CE50008FE191E19F938F930E946E580F900F90F6
:10CE600008950F931F93CF93DF93CDB7DEB7249729
:10CE70000FB6F894DEBF0FBECDBF9E012F5F3F4FB0
:10CE80003F932F939E012D5F3F4F3F932F932DE8AC
:10CE900031E13F932F939F938F930E94A7722DB7F9
:10CEA0003EB7285F3F4F0FB6F8943EBF0FBE2DBF71
:10CEB000029709F052C0E091BC15F091BD15EB53FB
:10CEC000FF4F09811A8198014B815C8160E070E01D
:10CED000808191810E94072B9B01AC012F3F8FEF36
:10CEE00038078FEF48078FEF5807E9F0E4F0BB27CA
:10CEF00057FDBA95A52F942F832F9F938F93C90128
:10CF000090709F938F9382E991E19F938F930E94FA
:10CF10006E582DB73EB72A5F3F4F0FB6F8943EBF0D
:10CF20000FBE2DBF22C088279927DC01821B930BDF
:10CF3000A40BB50BBF93AF939F938F9387EB91E1B6
:10CF40009F938F930E946E588DB79EB706960FB62B
:10CF5000F8949EBF0FBE8DBF08C08AED91E19F93EC
:10CF60008F930E946E580F900F9024960FB6F894EE
:10CF7000DEBF0FBECDBFDF91CF911F910F910895FE
:10CF8000CF92DF92EF92FF920F931F93CF93DF9395
:10CF9000CDB7DEB728970FB6F894DEBF0FBECDBF72
:10CFA0009E012F5F3F4F3F932F939E012D5F3F4F79
:10CFB0003F932F939E012B5F3F4F3F932F939E01F3
:10CFC000295F3F4F3F932F9324E032E13F932F930C
:10CFD0009F938F930E94A7722DB73EB7245F3F4F58
:10CFE0000FB6F8943EBF0FBE2DBF8130910519F0EA
:10CFF0008430910519F5E091BC15F091BD150197AC
:10D0000059F4EB53FF4F4F81588560E070E0808109
:10D0100091810E94EC2B1BC0EB53FF4FC980DA803B
:10D02000EB80FC800D811E8198014F81588560E066
:10D0300070E0808191810E94722B09C08DE092E1A5
:10D040009F938F930E946E580F900F9040C09B014A
:10D05000AC012F3F8FEF38078FEF48078FEF58074E
:10D06000E9F0E4F0BB2757FDBA95A52F942F832F45
:10D070009F938F93C90190709F938F9386E592E160
:10D080009F938F930E946E582DB73EB72A5F3F4FF4
:10D090000FB6F8943EBF0FBE2DBF19C08827992741
:10D0A000DC01821B930BA40BB50BBF93AF939F9333
:10D0B0008F9387EB91E19F938F930E946E588DB76A
:10D0C0009EB706960FB6F8949EBF0FBE8DBF2896EA
:10D0D0000FB6F894DEBF0FBECDBFDF91CF911F9189
:10D0E0000F91FF90EF90DF90CF9008950F931F93D3
:10D0F000CF93DF93CDB7DEB724970FB6F894DEBF9A
:10D100000FBECDBF9E012F5F3F4F3F932F939E01D8
:10D110002D5F3F4F3F932F932DE831E13F932F93A6
:10D120009F938F930E94A7729C0101974DB75EB7A2
:10D13000485F5F4F0FB6F8945EBF0FBE4DBF0297BA
:10D1400000F5E091BC15F091BD152130310559F481
:10D15000EB53FF4F4B815C8160E070E080819181F7
:10D160000E94AF2C17C0EB53FF4F09811A81980121
:10D170004B815C8160E070E0808191810E94442C51
:10D1800009C08CE792E19F938F930E946E580F9095
:10D190000F9040C09B01AC012F3F8FEF38078FEFFE
:10D1A00048078FEF5807E9F0E4F0BB2757FDBA9521
:10D1B000A52F942F832F9F938F93C90190709F93D6
:10D1C0008F9386EB92E19F938F930E946E584DB799
:10D1D0005EB74A5F5F4F0FB6F8945EBF0FBE4DBF9C
:10D1E00019C088279927DC01821B930BA40BB50B70
:10D1F000BF93AF939F938F938BED92E19F938F9308
:10D200000E946E588DB79EB706960FB6F8949EBFD3
:10D210000FBE8DBF24960FB6F894DEBF0FBECDBFF4
:10D22000DF91CF911F910F910895CF93DF93CDB7E9
:10D23000DEB724970FB6F894DEBF0FBECDBF9E01B8
:10D240002F5F3F4F3F932F939E012D5F3F4F3F93A3
:10D250002F932DE831E13F932F939F938F930E945B
:10D26000A7722DB73EB7285F3F4F0FB6F8943EBF69
:10D270000FBE2DBF0297D1F48B819C810297B0F431
:10D2800089819A81029790F48981880F9B81890F07
:10D29000E091BC15F091BD15EB53FF4F482F60E0B6
:10D2A00070E0808191810E94FB2208C080E093E1C0
:10D2B0009F938F930E946E580F900F9024960FB6F5
:10D2C000F894DEBF0FBECDBFDF91CF910895FC0172
:10D2D000E081E03379F4E091BC15F091BD15EB539A
:10D2E000FF4F808191810E94803090935E158093E2
:10D2F0005D150895E13379F4E091BC15F091BD1509
:10D30000EB53FF4F60915D1570915E1580819181A7
:10D310000E94313108950E9428670895E091BC155C
:10D32000F091BD15EB53FF4F808191810E945F31D9
:10D330000895CF93DF93EC018881882309F462C0BC
:10D340008AE090E00E94A072E091BC15F091BD15BA
:10D35000EB53FF4F0190F081E02D81E0818BE09154
:10D36000BC15F091BD15EB53FF4F0190F081E02DFE
:10D370008CEF838BE091BC15F091BD15EB53FF4F03
:10D380000190F081E02D86E0828BE091BC15F09158
:10D39000BD15EB53FF4FA081B181FE01019000202C
:10D3A000E9F73197EC1BFD0B8E2F8F5FFD01848B0E
:10D3B000E091BC15F091BD15EB53FF4F0190F0814A
:10D3C000E02D84899927AC01BE01CF0145960E94CA
:10D3D0003F7DE091BC15F091BD15EB53FF4F2081CF
:10D3E0003181C9014196BC01C9010E94B83568E884
:10D3F00073E180E090E00E945B058AE090E00E948B
:10D40000A07208C08FE493E19F938F930E946E589F
:10D410000F900F90DF91CF910895CF93DF93EC01A0
:10D4200044E050E06CE773E10E94317D892B29F4E0
:10D43000CE0105960E94316754C045E050E061E896
:10D4400073E1CE010E94317D892B29F4CE0106962D
:10D450000E94C06746C044E050E067E873E1CE0137
:10D460000E94317D892B29F4CE0105960E947668B1
:10D4700038C044E050E06CE873E1CE010E94317D99
:10D48000892B29F4CE0105960E9415692AC046E031
:10D4900050E061E973E1CE010E94317D892B29F4CE
:10D4A000CE0106960E9467691CC045E050E068E91D
:10D4B00073E1CE010E94317D892B19F40E948E699F
:10D4C00010C047E050E06EE973E1CE010E94317D6B
:10D4D000892B29F4CE0108960E94996902C00E9406
:10D4E0002867DF91CF910895E091BC15F091BD15AB
:10D4F000EB53FF4F80819181892B31F06DE07AE60B
:10D5000086EA93E10E94525408950E948206DC014B
:10D51000CB01BC01CD0108958091E015813089F4E3
:10D520000E9482069B01AC0180915F15909160156D
:10D53000A0916115B0916215280F391F4A1F5B1F1A
:10D5400010C00E9482069B01AC0180915F159091F2
:10D550006015A0916115B0916215281B390B4A0B1B
:10D560005B0BCA01B9010895DC01CB0180935F1503
:10D5700090936015A0936115B09362154093E015E8
:10D5800008950F931F93CF93DF938C01EB012FEF3F
:10D590006F3F720731F4BC0182EC93E10E94EB1DF6
:10D5A0006FC0672B09F46CC0EB89FC898081918185
:10D5B000A281B3818F5E9E4BAD4ABE4DF1F0848156
:10D5C0009581A681B7818F5E9E4BAD4ABE4DA9F075
:10D5D00080859185A285B3858F5E9E4BAD4ABE4DF9
:10D5E00061F084859585A685B7858F5E9E4BAD4A93
:10D5F000BE4D19F08CEC93E102C081ED93E19F9355
:10D600008F93888999892B893C89821B930B9F93DF
:10D610008F93888999899F938F938D899E899F93F2
:10D620008F938F89988D9F938F938F85E82FFF27F6
:10D63000EE0FFF1FE654FC4E808191819F938F93E4
:10D640008A8999279F938F932696DF93CF93269766
:10D65000DF93CF9385E892E09F938F931F930F936F
:10D660000E9431750A80DB81C02D8DB79EB746962A
:10D670000FB6F8949EBF0FBE8DBF209709F094CFD0
:10D68000DF91CF911F910F910895EF92FF920F9329
:10D690001F93CF93DF937C01BC0185E592E00E944C
:10D6A0004275C0918015D0918115209709F481C0F1
:10D6B000EB89FC8980819181A281B3818F5E9E4B31
:10D6C000AD4ABE4D19F08CEC93E102C081ED93E1BF
:10D6D0009F938F93888999892B893C89821B930B0F
:10D6E0009F938F93888999899F938F938D899E8922
:10D6F0009F938F938F89988D9F938F938F85E82F1A
:10D70000FF27EE0FFF1FE654FC4E808191819F930F
:10D710008F938A8999279F938F932696DF93CF9330
:10D720002697DF93CF938DEA92E09F938F93FF929A
:10D73000EF920E9431758DB79EB746960FB6F8945A
:10D740009EBF0FBE8DBF8F89988D892B39F1EF89D0
:10D75000F88D008111819FEF0F3F190731F4B70158
:10D7600084ED93E10E94EB1D19C001151105B1F084
:10D770001F930F9384ED92E09F938F93FF92EF920C
:10D780000E943175F801028113818DB79EB706960C
:10D790000FB6F8949EBF0FBE8DBFE7CFB7018AE0EA
:10D7A00090E00E94C31D0990D881C02D209709F0F8
:10D7B0007FCFDF91CF911F910F91FF90EF90089550
:10D7C0000F931F93CF93DF938C01C0917A15D09163
:10D7D0007B15209709F471C0BC0188EF92E00E948C
:10D7E000427588859985AA85BB85BF93AF939F9322
:10D7F0008F938C819D81AE81BF81BF93AF939F93A7
:10D800008F93DF93CF9383E193E09F938F931F9345
:10D810000F930E9431758C859D852DB73EB7225F91
:10D820003F4F0FB6F8943EBF0FBE2DBF37E0893A89
:10D83000930721F4B8018AED92E007C029E0863A07
:10D84000920731F4B80188EE92E00E9442751AC046
:10D85000AA27BB27880F991FAA1FBB1FBF93AF938F
:10D860009F938F9381E293E09F938F931F930F93E6
:10D870000E9431758DB79EB708960FB6F8949EBF7B
:10D880000FBE8DBF8E859F859F938F9387E293E018
:10D890009F938F931F930F930E9431750990D881A6
:10D8A000C02D2DB73EB72A5F3F4F0FB6F8943EBF4D
:10D8B0000FBE2DBF209709F094CFDF91CF911F911C
:10D8C0000F910895009721F09093E2158093E11550
:10D8D0008091E1159091E215892B19F06093E5157F
:10D8E00008951092E5150895EF92FF920F931F93FC
:10D8F000CF93DF938C01EE24FF24BC018AE090E0FB
:10D900000E94C31DC0918815D0918915209719F1E7
:10D9100088819981E80EF91E9F938F93DF93CF93AF
:10D920008FE293E09F938F931F930F930E94317523
:10D93000CE01805690402DB73EB7285F3F4F0FB6BF
:10D94000F8943EBF0FBE2DBF805A9F4720F40A8037
:10D95000DB81C02DDBCF0E946F098E159F05A9F0DA
:10D960009F938F93FF92EF9289E393E09F938F931E
:10D970001F930F930E9431758DB79EB708960FB60F
:10D98000F8949EBF0FBE8DBF13C09F938F9386E503
:10D9900093E09F938F931F930F930E9431752DB740
:10D9A0003EB72A5F3F4F0FB6F8943EBF0FBE2DBF64
:10D9B000DF91CF911F910F91FF90EF900895009705
:10D9C00021F09093E4158093E3158091E3159091F5
:10D9D000E415892B19F06093E61508951092E61569
:10D9E0000895FC0113821282158214821182108222
:10D9F0000895CF93DF93EC012A813B8180918415B8
:10DA0000909185152817390761F08C819D81892BAC
:10DA100041F040E050E060E070E0CE010E94580A22
:10DA2000F4CF80918415909185159B838A838C8196
:10DA30009D8101969D838C83DF91CF910895FC0198
:10DA400084819581892B61F02281338180918415B5
:10DA5000909185152817390719F08FEF9FEF0895DA
:10DA6000CF010E94F96C80E090E00895FC012281D2
:10DA7000338180918415909185152817390719F005
:10DA80008FEF9FEF0895848195810197958384831B
:10DA9000892B19F4CF010E94B80A80E090E0089524
:10DAA000FC0184819581009771F0228133818091FE
:10DAB0008415909185152817390719F480E090E0B6
:10DAC00008958FEF9FEF08950F931F93CF93DF93E8
:10DAD000FC01C189D289EDA9FEA909958C01892B88
:10DAE00049F4CF5BDF4FE881F98160E072EC81E0BF
:10DAF00090E00995C801DF91CF911F910F91089592
:10DB0000AF92BF92CF92DF92EF92FF920F931F934B
:10DB1000CF93DF938C017B016A015901FC01C48121
:10DB2000D581808591850FB6F8940F921186108665
:10DB30000F900FBE8617970799F0892B29F0209731
:10DB400019F0CE010E94101AE114F10449F0C70146
:10DB50000E94031AEC01892B19F48FEF9FEF1DC06F
:10DB6000E114F104C1F0F801D583C483D183C083EB
:10DB7000D383C283CE0DDF1DD783C683D586C486EB
:10DB8000B786A686138612860FB6F8940F92F18692
:10DB9000E0860F900FBE80E090E0DF91CF911F9163
:10DBA0000F91FF90EF90DF90CF90BF90AF900895CE
:10DBB0006F927F928F929F92AF92BF92CF92DF929D
:10DBC000EF92FF920F931F93CF93DF939B013A0144
:10DBD000882499247B01EC01EA81FB810189128967
:10DBE000E801A296688579856115710519F48FEFB2
:10DBF0009FEFA5C0232B69F42E853F854C855D855D
:10DC0000CE010E94806DE801EBADFCAD0995C40129
:10DC100096C00FB6F8940F92AA84BB840F900FBEE3
:10DC2000A114B10491F4F80183AD94ADFC01099500
:10DC3000F8014085518562857385CE0140960E942A
:10DC4000F009892B31F3C5017AC0F801808187FF83
:10DC500039C0CC24DD24C614D70408F06FC05AE0C4
:10DC60008A149B0408F051C0EA81FB814191FB8337
:10DC7000EA832A813B818E819F812817390721F40D
:10DC80008C819D819B838A830894811C911C4D30DB
:10DC900011F04A3059F4F80184A9882311F084174F
:10DCA00069F4F80144ABF701519304C0F80114AAD8
:10DCB000F70141937F010894C11CD11CC614D704FD
:10DCC00078F223C06301A614B70408F46501882420
:10DCD00099248C149D0490F5EA81FB818191FB834A
:10DCE000EA83F70181937F012A813B818E819F81A5
:10DCF0002817390721F48C819D819B838A8308949E
:10DD0000811C911C8C149D0438F381149104B1F092
:10DD10000FB6F8940F928A859B85881999099B877D
:10DD20008A870F900FBE2A853B858C859D85281795
:10DD3000390720F4E801EBADFCAD0995C601DF9190
:10DD4000CF911F910F91FF90EF90DF90CF90BF90F8
:10DD5000AF909F908F907F906F900895CF92DF92B9
:10DD6000EF92FF920F931F93CF93DF937C016A0191
:10DD70008C01005F1F4F0FB6F8940F92F801828557
:10DD80009385860F971F93878287C285D3850F90CF
:10DD90000FBECC16DD06A8F4F70181AD92ADFC01F3
:10DDA0000995F7014485558566857785C8014096B4
:10DDB0000E94F009892B29F40FB6F8940F92F8010C
:10DDC000E4CFCE01DF91CF911F910F91FF90EF90A3
:10DDD000DF90CF9008956F927F928F929F92AF9233
:10DDE000BF92CF92DF92EF92FF920F931F93CF9348
:10DDF000DF93FB014A013901EC01E988FA88E70168
:10DE0000609688859985892B19F48FEF9FEF87C0DD
:10DE10006115710529F4AB01C7010E94AE6E7FC088
:10DE2000D7012D913D914D915C9131FF03C041E0AF
:10DE3000A42E01C0AA24D7018C91807819F031E07A
:10DE4000B32E01C0B82E0FB6F8940F924A855B85A9
:10DE50000F900FBE8F01CC24DD24B601C814D90465
:10DE60000CF05CC09A01260F371F8E859F852817FE
:10DE7000390770F04C855D85C7010E94AE6EAC011C
:10DE800060E070E08C859D858417950708F446C096
:10DE90006114710419F0F801849102C0D8018C91C9
:10DEA000B1E0BB1649F48A3061F422E0B22E8DE075
:10DEB000AB1661F4AB2C0AC0E2E0BE1611F491E09F
:10DEC000B92E0F5F1F4F0894C11CD11CE881F98146
:10DED0008193F983E883288139818E819F81281776
:10DEE000390721F48C819D81998388836F5F7F4FEF
:10DEF000C814D9040CF4B6CF6115710579F00FB6CA
:10DF0000F8940F928A859B85860F971F9B878A8737
:10DF10000F900FBEE701E9ADFAAD0995C601DF919B
:10DF2000CF911F910F91FF90EF90DF90CF90BF9016
:10DF3000AF909F908F907F906F90089520E030E099
:10DF4000FC01828193810E94EB6E089521E030E014
:10DF5000FC01828193810E94EB6E0895CF93DF9341
:10DF6000DC01EC01EA81FB81C189D289892B21F096
:10DF70008FEFAF3FB80719F48FEF9FEF15C0CD01BA
:10DF80000E94101A20E030E0A901B901CE014096AC
:10DF90000E94806D20E030E0A901B901CE01829697
:10DFA0000E94806D80E090E0DF91CF910895CF9244
:10DFB000DF92EF92FF920F931F93CF93DF936C0149
:10DFC0007A01FC01C189D289CA0183709070892BC2
:10DFD00061F02EE130E044E150E060E270E0CE011B
:10DFE00040960E94806D892B19F5C701837090704F
:10DFF000019779F02EE130E044E150E060E270E01A
:10E00000CE0182960E94806D892B19F08C899D89A2
:10E010000DC086E090E00E94031A8C01892B59F410
:10E020008C899D890E94101A8EA19FA10E94101AAE
:10E030008FEF9FEF23C0C7018070907C28813981CA
:10E040004A815B818050904811F42F7701C020688D
:10E05000288339834A835B83F80111821082D3823B
:10E06000C28215821482F3E0EF22FF2461E0E616FB
:10E07000F10419F0EBADFCAD0995C801DF91CF912A
:10E080001F910F91FF90EF90DF90CF900895AF9286
:10E09000BF92CF92DF92EF92FF920F931F93CF9395
:10E0A000DF936A01AA24BB24DA01ED90FD900D9163
:10E0B0001C912E2DFC01C189D289615071406732BB
:10E0C000710508F03AC16A5B7F4FFB01EE0FFF1F3D
:10E0D0000590F491E02D0994CF5BDF4F4BC0CD5BF1
:10E0E000DF4FA8C0CB5BDF4F05C0C95BDF4FCDC0A2
:10E0F000C75BDF4FE881F981822F0995ECC0C55BD2
:10E10000DF4FC3C0C35BDF4FF5CFC15BDF4FBDC087
:10E11000E6FE11C0FE01B2962685378544855585F9
:10E1200060857185CF010E94806D5C01892B19F497
:10E13000EBADFCAD0995E7FE0FC0FE017096A11492
:10E14000B10451F4268537854485558560857185F0
:10E15000CF010E94806D5C01A114B10409F0F0C0F0
:10E16000CF5ADF4F8FE39FEFAFEFBFEFE822F922E7
:10E170000A231B23E881F981C801B7010995ABC0C7
:10E18000CD5ADF4FE881F981C355D04009959B01F5
:10E19000AC01D6016D937D938D939C9313978CA5C1
:10E1A0009DA5892B31F42064F601208331834283BD
:10E1B00053838A8D9B8D892B09F0C2C0F601808123
:10E1C0009181A281B3818068B3C0E886F9860A870D
:10E1D0001B87B6C088859985AA85BB85A8C0EC86B3
:10E1E000FD860E871F87ACC08C859D85AE85BF855B
:10E1F0009EC088819981AA81BB81EE2011F0806444
:10E2000028C08F7B26C088819981AA81BB819C010F
:10E21000AD01207430704070507086FD22C0D60170
:10E220002D933D934D935C9313978AC0EDADFEAD56
:10E23000A3CFEF96E881F9810995DC01CB0177C086
:10E2400088819981AA81BB81EE2011F0806801C08C
:10E250008F7788839983AA83BB8372C0888187FF65
:10E2600005C081E090E0A0E0B0E061C0DA011D925D
:10E270001D921D921C92139763C0CB5ADF4FE88109
:10E28000F9818E2D3ACFC95ADF4FE881F98109957E
:10E290009927AA27BB274BC0FE0170962685378594
:10E2A00044855585B701CF010E94806D5C01892BA3
:10E2B00009F046C0EBADFCAD099542C0888D998D43
:10E2C00034C0FE01B2962685378544855585B70151
:10E2D000CF010E94806D5C0133C08AA59BA525C03B
:10E2E0000FB6F8940F92FD8EEC8E1AC08C8D9D8D1A
:10E2F0001CC00FB6F8940F92FF8EEE8E11C08E8D5B
:10E300009F8D13C00FB6F8940F92FFA6EEA608C01B
:10E310008EA59FA50AC00FB6F8940F92F9AAE8AA95
:10E320000F900FBE0DC088A999A9AA27BB27F60197
:10E3300080839183A283B38303C05FEFA52EB52EA4
:10E34000C501DF91CF911F910F91FF90EF90DF906A
:10E35000CF90BF90AF900895CF93DF93EC01EA8107
:10E36000FB810188F289E02DB2960FB6F8940F92E6
:10E3700082859385AA27BB270F900FBEBC01CD01D4
:10E38000DF91CF910895FC01228133812115310560
:10E3900021F080819181F90109950895EF92FF9212
:10E3A0000F931F93CF93DF93EC017B018A0180E0F1
:10E3B00090E0EC81FD81309711F0BC010995198343
:10E3C0000883FB82EA82DF91CF911F910F91FF902A
:10E3D000EF900895CF93DF932FEF3FEFEC01EC81A7
:10E3E000FD81309731F060E070E081E190E00995C7
:10E3F0009C01C901DF91CF910895CF93DF932FEF57
:10E400003FEFEC01EC81FD81309731F060E070E08E
:10E4100082E190E009959C01C901DF91CF910895B7
:10E420000F931F93CF93DF93CDB7DEB724970FB62B
:10E43000F894DEBF0FBECDBF8C017C836B838FEF62
:10E440009FEFF8012481358121153105B9F0BE0116
:10E450006F5F7F4F80E290E0F9010995009771F4BA
:10E46000F80124813581BE016D5F7F4F81E290E02C
:10E47000F9010995009711F489819A8124960FB6C4
:10E48000F894DEBF0FBECDBFDF91CF911F910F91EA
:10E4900008950F931F93CF93DF93CDB7DEB72497E3
:10E4A0000FB6F894DEBF0FBECDBF8C017C836B83AB
:10E4B0008FEF9FEFF8012481358121153105B9F0E7
:10E4C000BE016F5F7F4F88E190E0F90109950097E9
:10E4D00071F4F80124813581BE016D5F7F4F89E1C0
:10E4E00090E0F9010995009711F489819A812496A9
:10E4F0000FB6F894DEBF0FBECDBFDF91CF911F9155
:10E500000F910895FC0140E050E0BA0180819181B3
:10E510000E94F019009711F08FEF9FEF0895CF93AD
:10E52000DF93CDB7DEB78F819885AE01475F5F4F30
:10E53000BC018D819E810E944019DF91CF91089589
:10E5400060915104709152040E94C31D0895CF93AD
:10E55000DF93CDB7DEB78F819885AE01475F5F4F00
:10E56000BC018D819E810E94D872DF91CF91089568
:10E57000CF93DF93DC01EB0120E030E012C0ED919E
:10E58000FC9111978081882379F0ED91FC9111978E
:10E5900081911196FC93EE938993415050402F5FE7
:10E5A0003F4F4115510559F7C901DF91CF910895AA
:10E5B000CF93DF93CDB7DEB722970FB6F894DEBFC7
:10E5C0000FBECDBF9A019A838983AB01BE016F5FF5
:10E5D0007F4F88EB92E70E94097322960FB6F8945A
:10E5E000DEBF0FBECDBFDF91CF910895CF93DF93F4
:10E5F000DC01EC01EA81FB81309719F4ED81FE81A9
:10E6000003C00788F08DE02DCD010995DF91CF91F2
:10E6100008952F923F924F925F926F927F928F92C6
:10E620009F92AF92BF92CF92DF92EF92FF920F93A1
:10E630001F93CF93DF93CDB7DEB763970FB6F894F0
:10E64000DEBF0FBECDBF3C015B015B8B4A8B490136
:10E650003324432C232CEA89FB890191FB8BEA8B21
:10E66000002309F4BBC1802F99270E94E77D009702
:10E6700099F041E050E0BE016F5E7F4FC501F301AC
:10E680000995019741F7898999270E94E77D892B90
:10E6900081F711E0212EDFCF053289F0222059F4D5
:10E6A00041E050E0BE016F5E7F4FC501F301099567
:10E6B000019709F0D1C089898017C9F08FC1EA8913
:10E6C000FB891191FB8BEA8B153299F4222059F4C6
:10E6D00041E050E0BE016F5E7F4FC501F301099537
:10E6E000019709F0B9C08989853209F077C12224E0
:10E6F000B2CF7C0100E01A3211F4026019C01C365E
:10E7000011F4016015C0212F332710531A30B0F4D3
:10E71000C701B3E0880F991FBA95E1F78E0D9F1DD1
:10E72000E80EF91EE20EF31E80ED9FEFE80EF91ED3
:10E73000EA89FB891191FB8BEA8BDDCFAAE05A2E87
:10E7400013E02F36310521F12037310574F42336DB
:10E75000310529F12436310524F4232B09F47FC037
:10E7600063C02936310591F05FC02537310509F4C2
:10E770005BC02637310524F42337310529F054C016
:10E780002837310541F050C012E04EC055244CC02E
:10E79000F8E05F2E49C00061E0E15E2E45C0E11463
:10E7A000F10419F471E0E72EF12C01FF2AC0F1E128
:10E7B000EF16F104B0F0222061F440E150E0BE0118
:10E7C0006F5F7F4FC501F3010995181619060CF00C
:10E7D00043C080EF9FEFE80EF91E91E1E916F104C6
:10E7E00050F7E114F104F1F02220E1F4A701BE0199
:10E7F0006F5F7F4FC501F30109951816190694F054
:10E800002BC0222071F4F40182E090E0880E991E62
:10E81000A70160817181C501F301099518161906D8
:10E82000DCF44394222402C1222051F441E050E060
:10E83000BE016F5E7F4FC501F3010995019761F439
:10E84000222410C041E050E0BE016F5E7F4FC50141
:10E85000F3010995019731F0332009F0BFC08FEF24
:10E860009FEFE6C0898999270E94E77D892B51F7A0
:10E87000123009F047C0E114F10419F46FEFE62EED
:10E88000F62E01FF1AC012C00894E108F108E11445
:10E89000F10409F4CBC041E050E0BE016F5E7F4F50
:10E8A000C501F3010995019709F0C0C0898999272D
:10E8B0000E94E77D892B41F3B9C0F40182E090E02A
:10E8C000880E991EC080D18013C0F60111936F018C
:10E8D0000894E108F108E114F10489F041E050E006
:10E8E000BE016F5E7F4FC501F3010995019739F4B1
:10E8F0001989812F99270E94E77D892B31F3F60131
:10E90000108293C0133009F0A6CEC70101970F976C
:10E9100018F05FE0E52EF12C0C626E010894C11C2A
:10E92000D11CE114F10409F456C09989903349F4DB
:10E93000552019F448E0542E006105FF20C0037DE6
:10E9400035C0892F8153873018F45520C1F406C093
:10E95000892F8853823048F4552019F43AE0532E19
:10E960000EC0F8E0F515B8F50AC0892F815486303D
:10E9700018F08052863028F48AE0851560F5037E11
:10E9800015C09D3211F09B3221F402FF24C00B7F91
:10E990000DC0983711F0983531F404FF1CC020E108
:10E9A000522E0F7E03C081E0282E15C0F6019193F0
:10E9B0006F01F2E0EF16F10450F041E050E0BE01CB
:10E9C0006F5E7F4FC501F3010995019721F408940B
:10E9D000E108F108A6CF112703FF03C0842D992772
:10E9E00027C0B8016270707001FD20C0F60110826E
:10E9F000852D9927AC01CE0101960E94C47B94011C
:10EA00002E5F3F4F00FF0AC0F40149010190F081E1
:10EA1000E02D608371838283938307C0F4014901F1
:10EA20000190F081E02D718360834394339413CE81
:10EA300063960FB6F894DEBF0FBECDBFDF91CF91C6
:10EA40001F910F91FF90EF90DF90CF90BF90AF900C
:10EA50009F908F907F906F905F904F903F902F90FE
:10EA60000895CF93DF93CDB7DEB78F819885AE0140
:10EA7000475F5F4FBC018D819E810E946B75DF9166
:10EA8000CF910895EF92FF920F931F938C017B011A
:10EA90000E94F37CAC01B801F701808191810E9452
:10EAA000A4751F910F91FF90EF900895CF93DF937E
:10EAB000CDB7DEB7E5E0F0E0EC0FFD1F819191915D
:10EAC000AF01BC0180915104909152040E946B757A
:10EAD000DF91CF910895AF92BF92CF92DF92EF92E4
:10EAE000FF920F931F93CF93DF935C017B016A0129
:10EAF000CB010E94F37C8C010F5F1F4FC8010E9465
:10EB00006408EC01009719F40FEF1FEF11C0A80182
:10EB1000B7010E94DF7C9601AE01F5016081718131
:10EB200080EF99E10E943B1A8C01CE010E94EA0815
:10EB3000C801DF91CF911F910F91FF90EF90DF906F
:10EB4000CF90BF90AF900895CF93DF93DC01EC019D
:10EB5000EA81FB81309719F4E985FA8503C0038CBB
:10EB6000F48DE02DCD010995DF91CF9108950F939C
:10EB70001F9300E010E023E030E046E050E0B801F1
:10EB8000C8010E94DB79909365158093641581E03C
:10EB9000809363151F910F910895CF92DF92EF92AA
:10EBA000FF920F931F93CF93DF93EC01EE24FF248A
:10EBB00087010E94B775CE010A978B35910510F039
:10EBC000CAE0D0E0CC24DD24CC16DD0694F480919C
:10EBD0006415909165150E94F479AA27BB27E80E69
:10EBE000F91E0A1F1B1F0E94B4070894C11CD11CE8
:10EBF000EBCFC801B70128EC39E140E050E00E94BA
:10EC00004E7DDC01CB019E01442737FD4095542FFA
:10EC1000BC01CD010E94AE7DDA01C9012AE0B595A3
:10EC2000A795979587952A95D1F7DF91CF911F9159
:10EC30000F91FF90EF90DF90CF9008952F923F9229
:10EC40004F925F926F927F928F929F92AF92BF92FC
:10EC5000CF92DF92EF92FF920F931F93CF93DF93A8
:10EC6000CDB7DEB7C456D0400FB6F894DEBF0FBEA6
:10EC7000CDBF4424552432015301420180916315D4
:10EC8000882311F40E94B775CC24DD2451E3E52ECE
:10EC9000F12C1E010894211C311C8601020D131D4C
:10ECA00080916415909165150E94F479F801918323
:10ECB00080830E94B4070894E108F10882E090E0A4
:10ECC000C80ED91EF7FEE5CFF1019E012D593F4F29
:10ECD00081919191AA27BB27880E991EAA1EBB1E5F
:10ECE0002E173F07ACF7C501B40122E330E040E046
:10ECF00050E00E94AE7D49015A01CA01B90128ECD9
:10ED000039E140E050E00E944E7DDC01CB014AE059
:10ED1000B595A795979587954A95D1F7845F9140CA
:10ED2000A040B0402CF1810132E6E32EF12CE20C40
:10ED3000F31CF801819191918F01AA27BB27A501AE
:10ED40009401281B390B4A0B5B0BCA01B9010E94C5
:10ED50004E7DDC01CB01480E591E6A1E7B1EE0165B
:10ED6000F1063CF7F2E34F165104610471041CF400
:10ED700081E090E002C080E090E0CC59DF4F0FB618
:10ED8000F894DEBF0FBECDBFDF91CF911F910F91E1
:10ED9000FF90EF90DF90CF90BF90AF909F908F90BB
:10EDA0007F906F905F904F903F902F9008958823B1
:10EDB00021F0813011F0823019F40E94A54B0895A2
:10EDC000833011F40E94A54B0895882321F08130EF
:10EDD00011F0823019F40E94B24B0895833011F47F
:10EDE0000E94B24B08950E949F4B80E00E94E576FE
:10EDF00081E00E94E57682E00E94E57683E00E9451
:10EE0000E57608950F931F938B019C01CA01AA27F1
:10EE1000BB27800F911FA21FB31F80509D4CA240A3
:10EE2000B04018F081E090E002C080E090E01F91D7
:10EE30000F910895DC01CB01BC01CD0120E03FEE34
:10EE400040E050E00E948C7DDA01C9018F5F992774
:10EE50000895DC01CB01BC01CD0120E03FEE40E094
:10EE600050E00E948C7DDC01CB0180509F4E0895C4
:10EE7000DC01CB01BC01CD0120E03FEE40E050E0E1
:10EE80000E948C7DDC01CB0120E03FEE281B390B7A
:10EE9000C90108958F929F92AF92BF92CF92DF9255
:10EEA000EF92FF920F931F93CF93DF936C017A0140
:10EEB0008B01E901A901C801B7010E9402778823EB
:10EEC00009F083C0C801B7010E941A77982ECE01BD
:10EED000AA27BB278E0D9F1DA01FB11FBC01CD010E
:10EEE0000E941A77882EC801B7010E9429775C0119
:10EEF000981411F48E010EC0292D3327882D9927DF
:10EF000001972817390709F060C0C801B7010E94AE
:10EF100038778C01E92CFF2482E0E816F104A1F097
:10EF200083E0E816F1042CF481E0E816F10431F0F6
:10EF30004CC083E0E816F10469F047C0A801B601AF
:10EF4000C5010E9477790BC0A801B601C5010E94D6
:10EF5000877905C0A801B601C5010E949779282DBF
:10EF60003327C9010197E816F90691F522303105DA
:10EF7000B1F02330310524F42130310529F025C0CA
:10EF800023303105B9F021C0C01BD10BC00ED11EFA
:10EF9000AE01B60180E091E10E94777919C0C01BF3
:10EFA000D10BC00ED11EAE01B60180E091E10E94EE
:10EFB00087790EC0C01BD10BC00ED11EAE01B601A9
:10EFC00080E091E10E94977903C081E090E002C067
:10EFD00080E090E0DF91CF911F910F91FF90EF9033
:10EFE000DF90CF90BF90AF909F908F9008958F92B9
:10EFF0009F92AF92BF92CF92DF92EF92FF920F93C8
:10F000001F93CF93DF935C017A018B01E901A90182
:10F01000C801B7010E940277882309F083C0C801A4
:10F02000B7010E941A77982ECE01AA27BB278E0D12
:10F030009F1DA01FB11FBC01CD010E941A77882E11
:10F04000C801B7010E9429776C01981411F48E0150
:10F050000EC0292D3327882D9927019728173907A6
:10F0600009F060C0C801B7010E9438778C01E92C13
:10F07000FF2482E0E816F104A1F083E0E816F10431
:10F080002CF481E0E816F10431F04CC083E0E8167E
:10F09000F10469F047C0A801B601C5010E94A97931
:10F0A0000BC0A801B601C5010E94B97905C0A8012D
:10F0B000B601C5010E94C979282D3327C9010197DE
:10F0C000E816F90691F522303105B1F0233031050B
:10F0D00024F42130310529F025C023303105B9F061
:10F0E00021C0C01BD10BAE0160E071E1C501800FF2
:10F0F000911F0E94A97919C0C01BD10BAE0160E01D
:10F1000071E1C501800F911F0E94B9790EC0C01B2B
:10F11000D10BAE0160E071E1C501800F911F0E942B
:10F12000C97903C081E090E002C080E090E0DF9107
:10F13000CF911F910F91FF90EF90DF90CF90BF90F4
:10F14000AF909F908F9008954F925F926F927F92B1
:10F150008F929F92AF92BF92CF92DF92EF92FF92E7
:10F160000F931F93CF93DF93CDB7DEB7E2970FB620
:10F17000F894DEBF0FBECDBFDC01CB0139014A01DF
:10F1800044245524AC01BD01461557056805790591
:10F1900008F04BC082E3A82EB12CC12CD12CA40EB8
:10F1A000B51EC61ED71ED601C5016A147B048C0489
:10F1B0009D0410F4D401C3017C018D01E41AF50A09
:10F1C000060B170B9701CE0101960E94F77720E0FE
:10F1D00030E0E114F1040105110521F1FE01319641
:10F1E00081914826842D82958425082E86958695C2
:10F1F0008025082E869580258770042C452C8695C1
:10F2000007948795502C48260694879550244826C5
:10F210002F5F3F4FC901AA27BB278E159F05A00767
:10F22000B107F0F2B601A501AFCFC201E2960FB669
:10F23000F894DEBF0FBECDBFDF91CF911F910F912C
:10F24000FF90EF90DF90CF90BF90AF909F908F9006
:10F250007F906F905F904F900895EF92FF920F9381
:10F260001F937B018C01DA01C9010296A11DB11D1A
:10F270009C01AD01C801B7010E94A478009711F06C
:10F2800081E090E01F910F91FF90EF900895EF9231
:10F29000FF920F931F93CF93DF93CDB7DEB72297E3
:10F2A0000FB6F894DEBF0FBECDBFDC01CB017901F4
:10F2B0008A01BC01CD010E94A4788983FE013196A8
:10F2C000892F9927818322E030E0B801A701CF017F
:10F2D0000E944A7722960FB6F894DEBF0FBECDBFCC
:10F2E000DF91CF911F910F91FF90EF900895FB0157
:10F2F000DC01E89447F4689406C0F8940190C79A3A
:10F300000D92C798789441505040B8F70895FB018A
:10F31000DC01E89447F4689406C0F8940190C69A1A
:10F320000D92C698789441505040B8F70895FB016B
:10F33000DC01E89457F4689408C0F8940190C79AE7
:10F34000C69A0D92C798C698789441505040A8F735
:10F350000895FB01DC01E89447F4689406C0F89432
:10F36000C79A0190C7980D92789441505040B8F7D1
:10F370000895FB01DC01E89447F4689406C0F89412
:10F38000C69A0190C6980D92789441505040B8F7B3
:10F390000895FB01DC01E89457F4689408C0F894E0
:10F3A000C79AC69A0190C798C6980D927894415012
:10F3B0005040A8F708950F931F93682B642B822F5A
:10F3C000802B0FB6F8940F92379866B987B9379AA1
:10F3D0000F900FBE9927382F2227862F9927822B2F
:10F3E000932B1F910F910895AC01692F77270FB6CA
:10F3F000F8940F9287B126B12F76861711F424174F
:10F4000021F0379846B967B9379A369A3699FECFC0
:10F4100084B1282F332785B19927982F8827282B47
:10F42000392B0F900FBEC9010895AF92BF92CF92B2
:10F43000DF92FF920F931F93CF93DF936C015B01D9
:10F440008A01EC01FF24452BF9F0F501EF0DF11DC8
:10F45000808199279F938F938DED93E19F938F9355
:10F46000DF93CF930E942F19C80FD91F8DB79EB776
:10F4700006960FB6F8949EBF0FBE8DBFF3948F2DE6
:10F4800099278017910708F3C601DF91CF911F914B
:10F490000F91FF90DF90CF90BF90AF900895FC0147
:10F4A000808199279F938F93818199279F938F9331
:10F4B000828199279F938F93838199279F938F931D
:10F4C000848199279F938F93858199279F938F9309
:10F4D00083EE93E19F938F930E946E588DB79EB7F2
:10F4E0000E960FB6F8949EBF0FBE8DBF08950F9372
:10F4F0001F93FC01808199279F938F938181992786
:10F500009F938F93828199279F938F9383819927CC
:10F510009F938F93848199279F938F9385819927B8
:10F520009F938F9383EE93E19F938F9306E615E16C
:10F530001F930F930E942F198DB79EB740960FB659
:10F54000F8949EBF0FBE8DBFC8011F910F91089503
:10F550006F927F928F929F92BF92CF92DF92EF92A3
:10F56000FF920F931F93CF93DF933C014B01EC016C
:10F570008881803211F42196FBCF95E0B92E85E089
:10F58000C82ED12CC80CD91C0881E02EFF24E7FC22
:10F59000F094C7010E94DD7D892B89F11981812FAB
:10F5A000992787FD90950E94DD7D892B41F10A33D3
:10F5B0001CF4802F805304C0C7010E94F67D87553C
:10F5C000082F0295007F1A331CF4812F805307C047
:10F5D000812F992787FD90950E94F67D8755802B76
:10F5E000F601808322961B1424F488818A3339F42F
:10F5F0002196BA940894C108D108B7FEC5CFB7FCCC
:10F600000AC0F401A1E2B4E186E00D9001928150BC
:10F61000E1F7C30101C0CE01DF91CF911F910F919E
:10F62000FF90EF90DF90CF90BF909F908F907F9052
:10F630006F900895AF92BF92CF92DF92FF920F9397
:10F640001F93CF93DF935C01EB01FF24C42EDD24D5
:10F65000C6010197181619060CF043C08E010F0D54
:10F66000111DC5010E942F1841E050E0B8010E9411
:10F67000F672F8010081083011F00F3761F4FF20B5
:10F6800041F181E094E19F938F930E946E58FA9428
:10F690000F900F901EC00A3011F00D3049F485E034
:10F6A00094E19F938F930E946E580F900F9019C012
:10F6B000802F992787FD90959F938F9387E094E102
:10F6C0009F938F930E946E58F3940F900F900F901A
:10F6D0000F902F2D3327C6010197281739070CF4F7
:10F6E000BDCFCF0DD11D1882F3948F2D9927DF91B7
:10F6F000CF911F910F91FF90DF90CF90BF90AF906F
:10F700000895EF92FF921F93CF93DF93CDB7DEB7AB
:10F7100024970FB6F894DEBF0FBECDBF7C01AE01BB
:10F720004F5F5F4F6AE071E00E94831989819A817F
:10F73000AB81BC8187709070A070B0700097A105FC
:10F74000B10599F01981177087E090E0A0E0B0E072
:10F7500089839A83AB83BC83AE014F5F5F4F69E0BF
:10F7600071E0C7010E94831901C010E0812F992721
:10F7700024960FB6F894DEBF0FBECDBFDF91CF91B8
:10F780001F91FF90EF9008954F925F926F927F923A
:10F790008F929F92AF92BF92CF92DF92EF92FF92A1
:10F7A0000F931F93CF93DF938C012B01EA01EE247B
:10F7B0006115710519F0FB0191838083209749F051
:10F7C000CE010297839728F060E070E080E090E03F
:10F7D000E5C0F801F1908F018F2D99270E94E77DF8
:10F7E000892BB9F7FDE2FF1619F441E0E42E03C0BE
:10F7F000FBE2FF1619F4F801F1908F01209719F040
:10F80000C031D10591F4F0E3FF1679F4F80180815D
:10F81000883711F0883549F4F801F1800E5F1F4FE9
:10F82000C0E1D0E0F2E0EF2A0AC0209741F480E383
:10F83000F81619F4C8E0D0E002C0CAE0D0E0C83041
:10F84000D105E9F0C930D10524F4C230D105E9F081
:10F8500022C0CA30D10521F0C031D10551F01BC002
:10F860003CECA32E3CECB32E3CECC32E3CE0D32E60
:10F870001FC0A12CB12CC12C28E0D22E19C0A12C64
:10F88000B12CC12C90E1D92E13C0A12CB12CC12CCC
:10F8900080E4D82E0DC09E01442737FD4095542F9B
:10F8A00060E070E080E090E80E948C7D59016A0180
:10F8B00020E030E040E050E060E03E01882477FC4A
:10F8C0008094982C8F2D80538A3010F4F82E0DC020
:10F8D0008F2D81548A3118F4E9ECFE0E06C08F2D6D
:10F8E00081568A3148F5F9EAFF0E8F2D99278C173A
:10F8F0009D0714F567FD1CC0A216B306C406D50605
:10F90000A0F0CA01B901A40193010E944E7D9B01A0
:10F91000AC012F0D311D411D511D213080E03807F4
:10F9200080E0480780E8580710F06FEF01C061E001
:10F93000F801F1908F01C6CF4114510461F06623A4
:10F9400019F00150104004C0E1FE05C00250104003
:10F95000F201118300838E2D992767FF07C080FF76
:10F9600011C020E030E040E050E810C080FF08C047
:10F9700050954095309521953F4F4F4F5F4F0CC0AC
:10F9800057FF0AC02FEF3FEF4FEF5FE782E290E0B3
:10F990009093E8158093E715CA01B901DF91CF91E3
:10F9A0001F910F91FF90EF90DF90CF90BF90AF909D
:10F9B0009F908F907F906F905F904F900895FB0184
:10F9C000DC0140FF05C002C005900D9205900D922C
:10F9D00042505040C8F70895FB01DC0105900D929C
:10F9E0000020E1F70895FC0105900020E9F78095DB
:10F9F00090958E0F9F1F0895FC014150504030F0AC
:10FA000001900616D1F73197CF01089588279927DD
:10FA10000895FB01DC0140FF05C002C001900D927A
:10FA200001900D9242505040C8F70895DC0140FF0C
:10FA300003C001C06D936D9342505040D8F70895B4
:10FA4000FB01DC018D910190801911F40020D1F7A8
:10FA5000990B0895FB01DC0101900D920020E1F764
:10FA60000895FB01DC014150504030F08D91019030
:10FA7000801919F40020B9F7881B990B0895FB0130
:10FA8000DC014150504048F001900D920020C9F730
:10FA900001C01D9241505040E0F70895629FD0018F
:10FAA000739FF001829FE00DF11D649FE00DF11D39
:10FAB000929FF00D839FF00D749FF00D659FF00DE8
:10FAC0009927729FB00DE11DF91F639FB00DE11DD5
:10FAD000F91FBD01CF0111240895991B79E004C0DD
:10FAE000991F961708F0961B881F7A95C9F780957D
:10FAF000089597FB092E07260AD077FD04D049D038
:10FB000006D000201AF4709561957F4F0895F6F79E
:10FB1000909581959F4F0895A1E21A2EAA1BBB1BB9
:10FB2000FD010DC0AA1FBB1FEE1FFF1FA217B307C9
:10FB3000E407F50720F0A21BB30BE40BF50B661FDF
:10FB4000771F881F991F1A9469F7609570958095A3
:10FB500090959B01AC01BD01CF01089597FB092E43
:10FB600005260ED057FD04D0D7DF0AD0001C38F48C
:10FB700050954095309521953F4F4F4F5F4F0895D9
:10FB8000F6F790958095709561957F4F8F4F9F4FB9
:10FB90000895AA1BBB1B51E107C0AA1FBB1FA617D4
:10FBA000B70710F0A61BB70B881F991F5A95A9F726
:10FBB00080959095BC01CD010895082E8062813614
:10FBC00024F087360CF408952BC0802D36C0911197
:10FBD00027C0803251F08A3041F08C3031F08D30C6
:10FBE00021F0893011F08B3099F708958F931DD053
:10FBF0008F9109F080620895E199FECFBFBBAEBB43
:10FC0000E09A11960DB20895E199FECFBFBBAEBB4D
:10FC10000DBA11960FB6F894E29AE19A0FBE0895C4
:10FC200099278827089585FDFBCF80629111F8CF31
:10FC30008136ECF38B37DCF708959111F1CF8053C7
:06FC40008A50E0F7089570
:10FC4600722B000A23202D2D2D2D2D2D2D2D2D2D02
:10FC56002D2D2D2D2D2D2D2D2D2D2D2D2D2D2D2DCE
:10FC66002D2D2D2D2D2D2D2D2D2D2D2D2D2D2D2DBE
:10FC76002D2D2D2D2D2D2D2D2D2D2D2D000A232015
:10FC860057656C636F6D6520746F2042546E757492
:10FC960020286329203230303620455448205A75B2
:10FCA600726963680032303037303332382D31357F
:10FCB600323500232062742D636D642070726F6785
:10FCC60072616D2076657273696F6E3A2025730ACC
:10FCD600002449643A2062742D636D642E632C7689
:10FCE60020312E343820323030362F31322F313514
:10FCF6002031323A32343A31332079756563656C96
:10FD06006D20457870202400232025730A002320C7
:10FD160072756E6E696E6720402025752E2530340B
:10FD260075204D487A2C204E7574467265713D25B6
:10FD3600756C20487A0A0023202D2D2D2D2D2D2D72
:10FD46002D2D2D2D2D2D2D2D2D2D2D2D2D2D2D2DDD
:10FD56002D2D2D2D2D2D2D2D2D2D2D2D2D2D2D2DCD
:10FD66002D2D2D2D2D2D2D2D2D2D2D2D2D2D000A0D
:10FD7600626F6F74696E6720426C7565746F6F741D
:10FD860068206D6F64756C652E2E2E00426C75654D
:10FD9600746F6F7468204D414320616464726573AB
:10FDA600733A20252E34783A252E34783A252E3487
:10FDB600780A004843492076657273696F6E3A2067
:10FDC600255820252E345820255820252E345820F5
:10FDD600252E34580A004C4D5020666561747572A4
:10FDE60065733A20252E325820252E325820252E8E
:10FDF600325820252E325820252E325820252E32D4
:10FE06005820252E325820252E32580A004C6F6372
:10FE1600616C206E616D653A20272573270A0062A2
:10FE2600742D636D642064656D6F00686974207459
:10FE3600616220747769636520666F722061206C49
:10FE4600697374206F6620636F6D6D616E647300F5
:10FE56005B62742D636D6440252E32783A252E320E
:10FE6600785D242000FF6D61696E006574686572B7
:10FE76006E75740069646C650000000000890C00F2
:10FE8600007561727430000000000500000000007B
:10FE96006203646D4770D86D9E6FA66FD76FAE6FA5
:10FEA600AC7100000000000000000000000000002F
:10FEB600000000000000000000000000000000003C
:10FEC600000000000000000000000000000000002C
:10FED60000000000000000F0101211D010D2106EC9
:10FEE600105110500E030EAC0E8F0EFC0EE80E3C99
:10FEF6000F320F9A0F5A0F1A100710000075617211
:10FF0600743100000000050100000000DE03646D8E
:10FF16004770D86D9E6FA66FD76FAE6FAC7100003D
:10FF260000000000000000000000000000000000CB
:10FF360000000000000000000000000000000000BB
:10FF460000000000000000000000000000000000AB
:10FF5600000000B115B4158A15901528150B15E18A
:10FF6600129112421323139A138613DA13D0133AFB
:10FF760014F813C614B11400000000FC15000000AC
:10FF860000B01600000000171700000000771701E8
:10FF96000002000300000000000000000000003026
:10FFA600303030303030303030303030303030205B
:10FFB6002020202020202020202020202020202833
:10FFC6006E756C6C2900303132333435363738393A
:10FFD60041424344454600303132333435363738B2
:10FFE60039616263646566003132333400425453CA
:0AFFF6007461636B00722B005F550D
:020000021000EC
:1000000041525472656164206572726F72210A00F8
:100010006672616D696E67206572726F720A006246
:100020007566666572206F76657272756E20657290
:10003000726F720A00706172697479206572726FF2
:10004000720A005F55415254777269746520657277
:10005000726F72210A007061636B6574206F757432
:10006000206F662073796E6320746F204254207570
:10007000617274210A00307825580A0073656D6139
:100080002025703A2025640A0073656D6100000127
:100090000F4C4544000A0000004C6F674576740021
:1000A000545F5445524D494E414C00252E32783A0A
:1000B000252E32783A252E32783A252E32783A2576
:1000C0002E32783A252E327800446576696365735E
:1000D0003A2025640A004465766963652020202063
:1000E000202020202062745F6164647220636F644A
:1000F0002020202020202020525353490A005B2535
:10010000645D3A2000203078252E386C78202564F4
:100110000A0062743A206572726F722075736167AB
:10012000653A0A20627420616464720A2062742055
:10013000636F6E7461626C650A206274207561720F
:10014000746465627567203C303D6F66662C2031B3
:100150003D6F6E3E0A20627420636874696D656F3E
:100160007574203C68616E646C653E203C74696DFA
:10017000653E0A20627420636F6E203C696E712DAB
:10018000696E6465783E207C2078783A78783A7891
:10019000783A78783A78783A78780A2062742064E5
:1001A0006973636F6E203C68616E646C653E0A2003
:1001B000627420696E71756972790A002062742018
:1001C0006E616D650A20627420636F640A20627438
:1001D00020726E616D650A20627420726F6C6520FA
:1001E0003C68616E646C653E0A20627420726F6CBC
:1001F00065736574203C68616E646C653E203C6D7F
:10020000795F726F6C653A4D3D3020533D313E0A47
:100210002062742066656174757265730A20627469
:100220002076657273696F6E0A0025752575006307
:1002300068616E676520646973632074696D656FBA
:10024000757420666F722068616E646C6520256429
:100250000A00636874696D656F75743A206572721F
:100260006F723D256C640A00636874696D656F7513
:1002700074206368616E676564210A0073796E6338
:10028000002575005374617274696E672073796E0E
:100290006320696E717569727920666F72202564BA
:1002A000207365633A0A006173796E6300506C6570
:1002B0006173652063616C6C2066697273742027BA
:1002C000627420696E717569727920726573756CDC
:1002D0007427210A005374617274696E6720617318
:1002E000796E6320696E7175697279210A20557380
:1002F00065206E6578742027627420696E71756957
:10030000727920636865636B2720616E642F6F725A
:100310002027627420696E71756972792072657325
:10032000756C74272E0A00636865636B00496E71F3
:100330007569727920646F6E65210A00496E717566
:10034000697279207374696C6C2072756E6E696E57
:1003500067210A00726573756C7400506C65617377
:10036000652063616C6C2066697273742027627407
:1003700020696E7175697279206173796E632721C6
:100380000A00696E71756972793A206572726F72CE
:100390003A2075736167653A0A20696E71756972F2
:1003A000792073796E63205B74696D6520696E20B6
:1003B0007365635D0A20696E717569727920617376
:1003C000796E63205B74696D6520696E2073656367
:1003D0005D0A20696E717569727920726573756C3A
:1003E000740A20696E717569727920636865636B40
:1003F0000A002532783A2532783A2532783A253281
:10040000783A2532783A2532780068257500726E80
:10041000616D653A206572726F723A20646576206C
:10042000696E646578206F7574206F6620626F75E1
:100430006E64730A0067657474696E6720726E611A
:100440006D65206F6620000A00726E616D653A204E
:100450006572726F723A206E6F20636F6E207769DB
:1004600074682068616E646C652025640A00726E91
:10047000616D653A206572726F723A20252E32786E
:10048000210A0072656D6F7465206E616D653A2793
:1004900000270A00726E616D653A206572726F7294
:1004A0003A2075736167653A0A20726E616D652046
:1004B00078783A78783A78783A78783A78783A78F2
:1004C000780A20726E616D65203C696E712D696ECF
:1004D0006465783E0A20726E616D6520683C6861D3
:1004E0006E646C653E0A00636F6E3A206572726FCF
:1004F000723A2064657620696E646578206F757441
:10050000206F6620626F756E64730A006F70656E8F
:1005100020636F6E20746F2000636F6E3A206572E7
:10052000726F723A2028256C78290A006E65772050
:10053000636F6E212068616E646C6520256C640AAF
:1005400000646973636F6E3A206572726F723A204D
:100550006E6F20636F6E20776974682068616E64C7
:100560006C652025640A00646973636F6E3A2065C8
:1005700072726F723A2063616E6E6F742067657479
:100580002062745F61646472206F662068616E64CB
:100590006C652025640A00646973636F6E20636F65
:1005A0006E6E656374696F6E20746F20006469738A
:1005B000636F6E3A206572726F723A2063616E6E7D
:1005C0006F7420646973636F6E6E65637420636F0C
:1005D0006E6E656374696F6E2077697468206861F8
:1005E0006E646C652025640A00646973636F6E6EC7
:1005F0006563746564210A004552524F5220726F40
:100600006C65206368616E67653A206572726F720F
:1006100020636F64653D256C640A00726F6C6573BE
:1006200065742068616E646C652025643A206D797C
:1006300020726F6C6520697320004D415354455200
:100640000A00534C4156450A00726F6C657365741D
:100650003A206572726F723A2075736167653A0A63
:1006600020726F6C65736574203C68616E646C65A4
:100670003E203C6D795F726F6C653A4D3D30205382
:100680003D313E0A006D7920726F6C6520746F20D9
:10069000636F6E20776974682068616E646C652092
:1006A000256420697320000A48646C204D68646CDE
:1006B000204164647220202020202020202020203F
:1006C000202020537461746520526F6C65204D6F3B
:1006D00064650A0025336400252034642000202549
:1006E00035642000253464002061637469766500F8
:1006F00020686F6C640020736E696666002070610C
:10070000726B0020696E76616C69640073657400B9
:100710004552524F522077726974696E67206C6F30
:1007200063616C206E616D65210A004C6F63616CC2
:10073000206E616D6520736574210A006765740021
:100740004552524F522061736B696E67206C6F6324
:10075000616C206E616D65210A004C6F63616C20D5
:100760006E616D653A20272573270A006E616D65FD
:100770003A206572726F723A2075736167653A0A42
:10078000206E616D6520736574203C6E616D653E01
:100790000A206E616D65206765740A00256C75001E
:1007A0004552524F522077726974696E67206C6FA0
:1007B00063616C20434F44210A004C6F63616C20DD
:1007C000434F4420736574210A004552524F522012
:1007D00077726974696E67206C6F63616C20434F38
:1007E000443A20496C6C6567616C2076616C756574
:1007F0002028256C75292E0A004C6F63616C2043FC
:100800004F443A203078252E386C780A00636F64A4
:100810003A206572726F723A2075736167653A0AA1
:1008200020636F6420736574203C76616C75653E4F
:100830000A20636F64206765740A004C6F63616C03
:100840002062745F616464723A20004C6F63616C73
:10085000204843492076657273696F6E20696E6621
:100860006F3A20255820252E345820255820252E33
:10087000345820252E34580A004C6F63616C204C8C
:100880004D5020737570706F727465642066656179
:1008900074757265733A20252E325820252E3258F1
:1008A00020252E325820252E325820252E32582031
:1008B000252E325820252E325820252E32580A0057
:1008C0006164647200636F6E7461626C650075616F
:1008D0007274646562756700636874696D656F75CD
:1008E0007400636F6E00646973636F6E00696E718C
:1008F00075697279006E616D6500636F6400726E78
:10090000616D6500726F6C6573657400726F6C6504
:100910000066656174757265730076657273696FE0
:100920006E006274004261747465727920566F6C57
:10093000746167653A2025642E2530326420560A9A
:100940000D007061747465726E25752575257525A9
:1009500075007061747465726E636C72006F6E25E1
:1009600075006F66662575006862257525752575A5
:100970000075736167653A0A206C65642070617464
:100980007465726E203C73706565643A312D313048
:100990003E203C6475726174696F6E3E203C6E72DD
:1009A0003A312D383E205B6172675D0A206C6564C8
:1009B000207061747465726E636C720A206C656479
:1009C000206F6E203C6E723A302D333E0A206C65EB
:1009D00064206F6666203C6E723A302D333E0A20EA
:1009E0006C6564206862203C70617573653E203CD4
:1009F000342D626974207061747465726E3E203C9F
:100A00006475726174696F6E3E0A006C65640062A1
:100A1000617400746872656164730074696D6572F5
:100A2000730068656170006E7574000000010FFB53
:100A30000EF50EEF0E4442473A2000494E463A204A
:100A40000057524E3A20004552523A200025357543
:100A5000202531306C752043252E32642C202573DF
:100A6000006C6F672075736167653A0A0073686F81
:100A700077205B3C6E725F6D7367733E205B3C63F7
:100A80006C6173733E205B3C6D61736B5D5D5D0AF1
:100A900000676574205B3C69645F6E657765723ED4
:100AA000205B3C6E725F6D7367733E205B3C636CD2
:100AB0006173733E205B3C6D61736B3E5D5D5D5D9C
:100AC0000A00636C6561720A006C6F676D61736B1D
:100AD000203C636C6173733E205B3C6D61736B3EC5
:100AE0005D0A00766572626F73697479206F6E0AB1
:100AF00000766572626F73697479203C636C617310
:100B0000733E205B3C6D61736B3E5D0A00766572DF
:100B1000626F736974792070617573650A00766518
:100B200072626F7369747920726573756D650A00FE
:100B3000766572626F73697479206F66660A006FFA
:100B40006E00766572626F73697479206F6E210A28
:100B5000006661696C65643A206F74686572206C28
:100B60006F67206C697374656E6572207265676962
:100B7000737465726564210A006F6666007665723B
:100B8000626F73697479206F6666210A00706175FF
:100B9000736500766572626F736974792070617530
:100BA0007365642E0A00726573756D6500766572F3
:100BB000626F7369747920726573756D65642E0A4E
:100BC0000025642578006572723A20696E76616C42
:100BD0006964206C6F6720636C617373210A006C19
:100BE0006F6720636C6173732025692C20766572B2
:100BF000626F73697479206D61736B207365742003
:100C0000746F3A20252E32580A0073686F770025DA
:100C1000752575257800676574002575257525751A
:100C2000257800636C656172006C6F676D61736B32
:100C3000006C6F6720636C6173732025692C200042
:100C4000206C6F676D61736B2073657420746F3AED
:100C500020252E32580A00766572626F73697479A6
:100C6000006C6F6700656274206572726F72202D70
:100C70002075736167653A0A20686F6C640A207397
:100C80006E6966660A207061726B0A207363616E1A
:100C9000203C696E71756972795F7363616E3E2085
:100CA0003C706167655F7363616E3E0A20706F77A9
:100CB0006572205B307C315D0A2072657365740A51
:100CC00020636F6E736F6C65203C737472696E671E
:100CD0003E0A002575257500686F6C643A206D6FBB
:100CE0006465206368616E67653A20256420286921
:100CF0006E74657276616C202564290A0045525233
:100D00004F52206D6F6465206368616E67653A209D
:100D10006572726F7220636F64653D256C640A00B2
:100D2000686F6C64206572726F72202D207573611C
:100D300067653A20686F6C64203C68616E646C651E
:100D40003E203C74696D653E0A0025752575257544
:100D5000257500736E696666206572726F72202D4C
:100D60002075736167653A0A203C68616E646C6542
:100D70003E203C696E74657276616C3E203C617405
:100D800074656D70743E203C74696D656F75743E5A
:100D90000A203C68616E646C653E0A00736E696689
:100DA000663A206D6F6465206368616E67653A20FE
:100DB00025642028696E74657276616C202564292B
:100DC0000A007061726B206572726F72202D20753F
:100DD000736167653A0A203C68616E646C653E2009
:100DE0003C696E74657276616C2D736C6F74733EC2
:100DF0000A203C68616E646C653E0A007061726B2B
:100E00003A206D6F6465206368616E67653A2025DE
:100E1000642028696E74657276616C202564290AE5
:100E2000004552524F52206D6F6465206368616EB9
:100E3000676520286572726F7220636F64653D2557
:100E40006C64292E0A007363616E206572726F7282
:100E5000202D2075736167653A207363616E203CB5
:100E6000696E7175697279207363616E3A20303DE5
:100E70006F66662C20313D6F6E3E203C7061676569
:100E8000207363616E3A20303D6F66662C20313DE1
:100E90006F6E3E0A00636F6E736F6C6520657272D1
:100EA0006F72202D2075736167653A20656274202A
:100EB000636F6E736F6C65203C737472696E673E0E
:100EC0000A00686F6C6400736E6966660070617218
:100ED0006B007363616E00706F77657220007265DE
:100EE00073657400636F6E736F6C65006562740088
:100EF00054524D0052554E0052445900534C50002C
:100F0000AA13AE13B213B6135349474E414C45448E
:100F10000A004641494C004F4B005349474E414C53
:100F2000454400252E32782000252E32783A252E91
:100F300032783A252E32783A252E32783A252E32DA
:100F4000783A252E327800082008000A0025630030
:00000001FF
